S00F000078636F696E5F66772E73313988
S31508003000D0710020456301087D4201087F4201080E
S315080030108142010883420108854201080000000038
S315080030200000000000000000000000009B3F0108AF
S315080030308742010800000000553F0108894201083F
S31508003040C1660108C5660108C9660108CD6601089A
S31508003050D1660108D5660108D9660108DD6601084A
S31508003060E1660108E5660108E9660108ED660108FA
S31508003070F16601089D420108F5660108A7420108A4
S31508003080B1420108F9660108FD6601080000000062
S3150800309000000000000000000000000001670108B1
S315080030A005670108096701080D67010800000000A7
S315080030B01167010815670108196701081D670108E6
S315080030C02167010825670108296701082D67010896
S315080030D03167010835670108396701083D67010846
S315080030E04167010845670108000000004D670108AF
S315080030F0516701085567010800000000000000003C
S315080031004967010800000000596701085D67010862
S315080031106167010865670108696701086D67010845
S315080031207167010875670108BB42010879670108DC
S31508003130DFF8240B0078642801D1012000E0002084
S31508003140704780B5DFF8D00707F006FDDFF80C0BEF
S315080031500078002801D108F04DF83220DFF8FC1A73
S31508003160087001BD80B500224FF48051DFF8E407EE
S3150800317009F0EDFADFF8200B07F0EEFC01BD80B58B
S3150800318000224FF48051DFF8CC0709F0E0FADFF8A7
S315080031900C0B07F0E1FC01BD2DE9F843C0B00400B3
S315080031A00E0000254FF480775FF00008E946424696
S315080031B03900484609F00AFB300080B281281BDA3C
S315080031C0207850F48070ADF8000001273800C0B2AE
S315080031D0310080B289B2884209D23800C0B2205C78
S315080031E069463A00D2B221F812007F1CEEE7310098
S315080031F089B2684607F055FD41B0BDE8F0832DE970
S31508003200F843C0B004000E0000254FF480775FF045
S315080032100008E94642463900484609F0D7FA300020
S3150800322080B2812819DA2078ADF800000127380025
S31508003230C0B2310080B289B2884209D23800C0B221
S31508003240205C69463A00D2B221F812007F1CEEE7EC
S31508003250310089B2684607F024FD41B0BDE8F08325
S3150800326070B504000D0016002800C0B2412801DB25
S31508003270402005003000C0B2002806D02900C9B297
S3150800328089B22000FFF788FF05E02900C9B289B294
S315080032902000FFF7B4FF70BD10B50400200080B20F
S315080032A0C0F3002000283BD0DFF85C17DFF8680879
S315080032B002784020424301EB0200DFF85017DFF89E
S315080032C058281278895C4454DFF84007DFF8481814
S315080032D00978405C401CDFF83417DFF83C28127880
S315080032E088540120DFF82817DFF82C28127888542C
S315080032F00421DFF8200709F037FADFF81007DFF8AE
S3150800330018180978405C022836DB0020DFF8081711
S31508003310087000220121DFF80007FFF7A1FF2BE064
S31508003320DFF8E416DFF8F00702784020424301EBA5
S315080033300200DFF8D816DFF8E0271278895C4454D3
S31508003340DFF8C806DFF8D0170978405C401CDFF8BC
S31508003350BC16DFF8C42712788854DFF8B006DFF801
S31508003360B8170978405C402806DB3F20DFF89C1632
S31508003370DFF8A4271278885410BD30B403001878F3
S31508003380012422000D00EDB292B2ADB2AA4205D2D6
S31508003390220092B29A5C1018641CF2E7C0B230BCE4
S315080033A0704780B50820DFF8701608700820DFF827
S315080033B0681648700020DFF8641708800020DFF8D8
S315080033C04C1648700020DFF8481648700122022182
S315080033D0DFF84406FFF744FF01BD80B50920DFF892
S315080033E0381608700920DFF8301648700020DFF814
S315080033F02C1708800020DFF8141648700020DFF824
S315080034001016487001220221DFF80C06FFF728FF84
S3150800341001BD80B50A20DFF8001608700A20DFF81B
S31508003420F81548700020DFF8F41608800020DFF849
S31508003430DC1548700020DFF8D815487001220221F3
S31508003440DFF8D405FFF70CFF01BD80B50B20DFF8C8
S31508003450C81508700B20DFF8C01548700020DFF883
S31508003460BC1608800020DFF8A41548700020DFF895
S31508003470A015487001220221DFF89C05FFF7F0FE2F
S3150800348001BDF8B504000D0016001F000C20DFF87A
S3150800349088150870DFF880054470DFF87C058570AC
S315080034A0DFF87405C670DFF8700507710521DFF8C7
S315080034B06805FFF762FFDFF8601548710020DFF83E
S315080034C05C1608800020DFF8441548700020DFF8F5
S315080034D04015487001220621DFF83C05FFF7C0FEBB
S315080034E0F1BD10B504000D20DFF82C150870DFF8C3
S315080034F0280544700221DFF82005FFF73EFFDFF8B4
S31508003500181588700020DFF8141608800020DFF8E8
S31508003510FC1448700020DFF8F814487001220621D0
S31508003520DFF8F404FFF79CFE10BD70B500250024F3
S315080035300F20DFF8E4142A00D2B288546D1CFF204D
S31508003540DFF8D4142A00D2B288546D1C1720DFF88D
S31508003550C8142A00D2B288546D1C0020DFF8B814AB
S315080035602A00D2B288546D1C0020DFF8AC142A0059
S31508003570D2B288546D1C0020DFF89C142A00D2B2FF
S3150800358088546D1C0020DFF890142A00D2B28854A3
S315080035906D1C0020DFF880142A00D2B288546D1CF6
S315080035A00020DFF874142A00D2B288546D1C290052
S315080035B0C9B2DFF86404FFF7E0FE0600DFF8580436
S315080035C02900C9B246546D1C0020DFF85015088042
S315080035D00020DFF8381448700020DFF834144870EB
S315080035E001222900C9B2DFF83004FFF739FE70BDA1
S315080035F080B50F20DFF8201408700020DFF81814B3
S3150800360048700221DFF81004FFF7B7FEDFF8081448
S3150800361088700020DFF8041508800020DFF8EC1316
S3150800362048700020DFF8E813487001220321DFF80C
S31508003630E803FFF715FE01BD10B504000F20DFF8FB
S31508003640D81308700220DFF8D0134870DFF8C803D3
S3150800365084700321DFF8C003FFF78FFEDFF8B81385
S31508003660C8700020DFF8B41408800020DFF89C1327
S3150800367048700020DFF89813487001220421DFF80B
S315080036809803FFF7EDFD10BD80B50F20DFF888130E
S3150800369008700320DFF8801348700221DFF87803EA
S315080036A0FFF76BFEDFF8701388700020DFF86C14E4
S315080036B008800020DFF8541348700020DFF8501304
S315080036C0487001220321DFF85003FFF7C9FD01BD49
S315080036D080B50F20DFF8401308700420DFF8381390
S315080036E048700221DFF83003FFF747FEDFF828139A
S315080036F088700020DFF8241408800020DFF80C13F7
S3150800370048700020DFF80813487001220321DFF80B
S315080037100803FFF7A5FD01BD80B50F20DFF8F812F5
S3150800372008700520DFF8F01248700221DFF8E80279
S31508003730FFF723FEDFF8E01288700020DFF8DC13BD
S3150800374008800020DFF8C41248700020DFF8C01295
S31508003750487001220321DFF8C002FFF781FD01BD91
S31508003760F8B50600002400253000C0B2102819DA82
S31508003770DFF8D00A3100C9B2405CDFF8CC1A097804
S31508003780484309F093F800273900DFF8C02A127871
S31508003790C9B2914205D2DFF8081D09F099F87F1CD5
S315080037A0F2E700E00020F2BD80B530209A490870A3
S315080037B03020994948700020DFF8601308800020FF
S315080037C09249087000209249087001220221924805
S315080037D0FFF746FD01BD80B531208F4908703120BD
S315080037E08D4948700020DFF8341308800020874987
S315080037F00870002086490870012202218648FFF7D2
S315080038002FFD01BD80B533208349087033208249D6
S3150800381048700020C149088000207C4908700020B3
S315080038207B490870012202217B48FFF719FD01BD7B
S31508003830F8B504000D0016001F00342076490870FC
S3150800384075484470744885707348C6707248077125
S3150800385005217148FFF791FD6F4948710020AF496E
S31508003860088000206949087000206949087001220B
S3150800387006216948FFF7F4FCF1BD80B53520664995
S31508003880087000206449487002216348FFF775FDF7
S31508003890614988700020A149088000205B490870AA
S315080038A000205B490870012203215B48FFF7D8FC1A
S315080038B001BD80B535205849087001205649487021
S315080038C002215548FFF759FD53498870002093494E
S315080038D0088000204D49087000204D4908700122D3
S315080038E003214D48FFF7BCFC01BD80B536204A4987
S315080038F0087036204849487000208849088000200A
S3150800390042490870002042490870012202214248B3
S31508003910FFF7A6FC01BD00009456010880B53720C4
S315080039203D49087000203C49487002213A48FFF793
S3150800393024FD3949887000207849088000203349D9
S315080039400870002032490870012203213248FFF727
S3150800395087FC01BD000C0140F8B5060000240025CF
S315080039603000C0B2102819DADFF88C093100C9B264
S31508003970405CDFF888190988484308F097FF002754
S315080039803900DFF87C291278C9B2914205D2DFF8EE
S31508003990101B08F09DFF7F1CF2E700E00020F2BD37
S315080039A038B504000D0037201B490870FE201A4957
S315080039B0487030201849887000201749C870402080
S315080039C015490871144844712800C0B2002803D06C
S315080039D002201149887102E000200F4988710721E9
S315080039E00D48FFF7CAFC0C49C87100204B490880EE
S315080039F000200649087000200549087001220821A0
S31508003A000548FFF72DFC31BD78630020C86B002000
S31508003A10CC6B002000100140F06800202DE9F0472B
S31508003A2004000D00904600265FF000090027404676
S31508003A30C0B2202804DBDFF86C0A07F08DF84EE0E8
S31508003A403720DFF8001D3200D2B28854761CFC20DD
S31508003A50DFF8F01C3200D2B28854761C3020DFF82A
S31508003A60E41C3200D2B28854761CDFF8D80C310038
S31508003A70C9B24454761C5FF0000A50464146C0B2AB
S31508003A80C9B288420BD25046C0B2285CDFF8B41CD3
S31508003A903200D2B28854761C1AF1010AEDE73100D9
S31508003AA0C9B2DFF8A00CFFF768FC8146DFF8940C72
S31508003AB03100C9B200F80190761C00201749088029
S31508003AC00020DFF8E41908700020DFF8E019087014
S31508003AD001223100C9B2DFF86C0CFFF7C1FBBDE863
S31508003AE0F08780B51020DFF85C1C08701020DFF81E
S31508003AF0541C48700020094908800020DFF8A819DE
S31508003B0088700020DFF8A419887001220221DFF8E6
S31508003B10340CFFF7A5FB01BDA86C00205C6C0020E7
S31508003B2070B5002500241120DFF8181C2A00D2B22F
S31508003B3088546D1C0020DFF80C1C2A00D2B2885469
S31508003B406D1C0320DFF8FC1B2A00D2B288546D1CBA
S31508003B500020DFF8F01B2A00D2B288546D1C002022
S31508003B60DFF8E01B2A00D2B288546D1C0020DFF86B
S31508003B70D41B2A00D2B288546D1C2900C9B2DFF8BA
S31508003B80C40BFFF7FAFB0600DFF8B80B2900C9B229
S31508003B9046546D1C0020DFF8181908800020DFF84D
S31508003BA0081988700020DFF8041988700122290096
S31508003BB0C9B2DFF8900BFFF753FB70BD70B500254F
S31508003BC000241120DFF87C1B2A00D2B288546D1C11
S31508003BD00120DFF8701B2A00D2B288546D1CFF2022
S31508003BE0DFF8601B2A00D2B288546D1CFF20DFF86C
S31508003BF0541B2A00D2B288546D1C0020DFF8441BDF
S31508003C002A00D2B288546D1C0020DFF8381B2A001F
S31508003C10D2B288546D1C2900C9B2DFF8280BFFF709
S31508003C20ACFB0600DFF81C0B2900C9B246546D1C14
S31508003C300020DFF87C1808800020DFF86C188870F0
S31508003C400020DFF86818887001222900C9B2DFF859
S31508003C50F40AFFF705FB70BDA46C0020956C0020E4
S31508003C6080B51220DFF8DC1A08701220DFF8D41AA3
S31508003C7048700020DFF8381808800020DFF8281878
S31508003C8088700020DFF82418887001220221DFF8E6
S31508003C90B40AFFF7E5FA01BD1461010824610108B9
S31508003CA070B5002500241720DFF8981A2A00D2B22A
S31508003CB088546D1C0020DFF88C1A2A00D2B288546A
S31508003CC06D1C4E20DFF87C1A2A00D2B288546D1C6F
S31508003CD05920DFF8701A2A00D2B288546D1C582071
S31508003CE0DFF8601A2A00D2B288546D1C0020DFF86B
S31508003CF0541A2A00D2B288546D1C0020DFF8441AE0
S31508003D002A00D2B288546D1C0020DFF8381A2A001F
S31508003D10D2B288546D1C0020DFF8281A2A00D2B2C5
S31508003D2088546D1C0020DFF81C1A2A00D2B2885469
S31508003D306D1C0020DFF80C1A2A00D2B288546D1CBC
S31508003D400020DFF8001A2A00D2B288546D1C002021
S31508003D50DFF8F0192A00D2B288546D1C0020DFF86B
S31508003D60E4192A00D2B288546D1C0020DFF8D41951
S31508003D702A00D2B288546D1C0020DFF8C8192A0020
S31508003D80D2B288546D1C0020DFF8B8192A00D2B2C6
S31508003D9088546D1C0020DFF8AC192A00D2B288546A
S31508003DA06D1C0020DFF89C192A00D2B288546D1CBD
S31508003DB00020DFF890192A00D2B288546D1C002022
S31508003DC0DFF880192A00D2B288546D1C0020DFF86B
S31508003DD074192A00D2B288546D1C0020DFF86419C1
S31508003DE02A00D2B288546D1C0020DFF858192A0020
S31508003DF0D2B288546D1C0020DFF848192A00D2B2C6
S31508003E0088546D1C0020DFF83C192A00D2B2885469
S31508003E106D1C0020DFF82C192A00D2B288546D1CBC
S31508003E200020DFF820192A00D2B288546D1C002021
S31508003E30DFF810192A00D2B288546D1C0020DFF86A
S31508003E4004192A00D2B288546D1C0020DFF8F41831
S31508003E502A00D2B288546D1C2900C9B2DFF8E408DA
S31508003E60FFF78BFA0600DFF8DC082900C9B24654CA
S31508003E706D1C0020DFF8381608800020DFF82816A9
S31508003E8088700020DFF82416887001222900C9B23C
S31508003E90DFF8B008FFF7E4F970BD70B50025002417
S31508003EA01720DFF8A0182A00D2B288546D1C042007
S31508003EB0DFF890182A00D2B288546D1C0020DFF86B
S31508003EC084182A00D2B288546D1C0020DFF87418B2
S31508003ED02A00D2B288546D1C0020DFF868182A0020
S31508003EE0D2B288546D1C2020DFF858182A00D2B2A6
S31508003EF088546D1C2900C9B2DFF84808FFF73DFA57
S31508003F000600DFF840082900C9B246546D1C002097
S31508003F10DFF89C1508800020DFF88C1588700020D3
S31508003F20DFF88815887001222900C9B2DFF814085D
S31508003F30FFF796F970BD70B5002500241420DFF848
S31508003F4004182A00D2B288546D1C0020DFF8F41732
S31508003F502A00D2B288546D1C2900C9B2DFF8E407DA
S31508003F60FFF70BFA0600DFF8DC072900C9B246544A
S31508003F706D1C0020DFF8381508800020DFF82815AA
S31508003F8088700020DFF82415887001222900C9B23C
S31508003F90DFF8B007FFF764F970BD70B50025002497
S31508003FA01420DFF8A0172A00D2B288546D1C01200D
S31508003FB0DFF890172A00D2B288546D1C2900C9B2BE
S31508003FC0DFF88007FFF7D9F90600DFF87807290038
S31508003FD0C9B246546D1C0020DFF8D41408800020AE
S31508003FE0DFF8C41488700020DFF8C0148870012236
S31508003FF02900C9B2DFF84C07FFF732F970BD70B572
S31508004000002500241420DFF83C172A00D2B2885471
S315080040106D1C0220DFF82C172A00D2B288546D1CBA
S315080040202900C9B2DFF81C07FFF7A7F90600DFF871
S3150800403014072900C9B246546D1C0020DFF8701415
S3150800404008800020DFF8601488700020DFF85C1410
S31508004050887001222900C9B2DFF8E806FFF700F9DF
S3150800406070BD2DE9F04104000D000027002613203D
S31508004070DFF8D0163A00D2B288547F1C0020DFF849
S31508004080C4163A00D2B288547F1C200080B2000AB7
S31508004090DFF8B0163A00D2B288547F1CDFF8A406BF
S315080040A03900C9B244547F1C280080B2000ADFF8E0
S315080040B094163A00D2B288547F1CDFF88806390075
S315080040C0C9B245547F1C3900C9B2DFF87806FFF734
S315080040D054F98046DFF86C063900C9B200F8018049
S315080040E07F1C0020DFF8C81308800020DFF8B8130B
S315080040F088700020DFF8B413887001223900C9B22D
S31508004100DFF84006FFF7ACF8BDE8F08170B500258A
S3150800411000241320DFF82C162A00D2B288546D1C0E
S315080041200220DFF820162A00D2B288546D1CFF2020
S31508004130DFF810162A00D2B288546D1CFF20DFF86B
S3150800414004162A00D2B288546D1C2900C9B2DFF8B9
S31508004150F405FFF712F90600DFF8E8052900C9B2E9
S3150800416046546D1C0020DFF8481308800020CE490D
S3150800417088700020CD49887001222900C9B2DFF86D
S31508004180C405FFF76DF870BD70B50025002413202F
S31508004190DFF8B0152A00D2B288546D1C0320DFF868
S315080041A0A4152A00D2B288546D1C2900C9B2DFF8BA
S315080041B09405FFF7E2F80600DFF888052900C9B27A
S315080041C046546D1C0020BA4908800020B6498870FC
S315080041D00020B649887001222900C9B2DFF86405B3
S315080041E0FFF73EF870BD70B5002500241320DFF8F0
S315080041F054152A00D2B288546D1C0420DFF84415E1
S315080042002A00D2B288546D1C2900C9B2DFF83405D9
S31508004210FFF7B3F80600DFF82C052900C9B24654A3
S315080042206D1C0020A249088000209F498870002044
S315080042309E49887001222900C9B2DFF80805FFF7F0
S315080042400FF870BDBC6A0020716C0020726C0020EB
S315080042502DE9F04104000D00002700261320DFF8A1
S31508004260E4143A00D2B288547F1C0520DFF8D4142F
S315080042703A00D2B288547F1C200080B2000ADFF8C8
S31508004280C4143A00D2B288547F1CDFF8B804390047
S31508004290C9B244547F1C280080B2000ADFF8A4146F
S315080042A03A00D2B288547F1CDFF898043900C9B2A4
S315080042B045547F1C3900C9B2DFF88804FFF75DF85A
S315080042C08046DFF880043900C9B200F801807F1CF7
S315080042D000207749088000207349887000207349B8
S315080042E0887001223900C9B2DFF85804FEF7B8FF12
S315080042F0BDE8F08100000000CC6A00202E6C00208A
S31508004300766C002070B5FEF73AFF0020DFF88C15B2
S3150800431008700020DFF8881508800020DFF884156B
S3150800432008700020DFF8801508800020DFF87C156B
S3150800433008700020DFF86C1548700020DFF8681553
S3150800434048800020DFF8641548700020DFF854150F
S3150800435088700020DFF8501588800020DFF84C159B
S3150800436088700020DFF8481508700020DFF844152B
S3150800437008700020DFF8401508700020DFF83C15AB
S3150800438008700020DFF8381508700020DFF83415AB
S3150800439008700020DFF8301508700020DFF82C15AB
S315080043A008700020DFF8281508700020DFF82415AB
S315080043B008800020DFF8201508800020DFF81C158B
S315080043C008700020DFF8181508700020DFF81415AB
S315080043D008700020DFF8101508700020DFF80C15AB
S315080043E008700020DFF8081508700020DFF80415AB
S315080043F00870FF20DFF80015087020240025DFF874
S31508004400FC642A002100300008F0E0F90020DFF8FB
S31508004410F01408800020DFF8EC1408800020DFF88C
S31508004420E81408800020DFF8E41408800020DFF88C
S31508004430E01408700020DFF8DC1408700020DFF8AC
S31508004440D81408700020DFF8D41408700020DFF8AC
S31508004450D01408700020DFF8CC1408700020DFF8AC
S31508004460C8140870FF20DFF8C4140870FF20DFF8AE
S31508004470C0140870FF20DFF8BC140870FF20DFF8AE
S31508004480B81408700020DFF8B41408600020DFF8BC
S31508004490B01408600020DFF8AC14087070BD000086
S315080044A000002041AC460108C86B0020CC6B0020F8
S315080044B05C6C002070B50024DFF88C0406F04CFB19
S315080044C000252800C0B20F280ADADFF88004290080
S315080044D0C9B20844C17B82A006F03EFB6D1CF0E71A
S315080044E097A006F039FBDFF8680406F035FB0026CE
S315080044F03000C0B20F2809DADFF850043100C9B21B
S31508004500415C77A006F028FB761CF1E78CA006F044
S3150800451023FBDFF8400406F01FFB00242000C0B28E
S315080045200F280ADADFF824042100C9B20844817F7B
S315080045306BA006F011FB641CF0E781A006F00CFBEB
S31508004540DFF8140406F008FBDFF81004C178DFF87A
S31508004550100406F001FBDFF804040179DFF804040F
S3150800456006F0FAFADFF800040079002811D0DFF81F
S31508004570F803407900280CD0DFF8EC03807900288E
S3150800458007D071A006F0E8FADFF8E01354A006F0A9
S31508004590E3FADFF8DC0306F0DFFADFF8C003017898
S315080045A0DFF8BC0306F0D8FADFF8B0034178DFF885
S315080045B0B40306F0D1FADFF8BC0306F0CDFADFF84B
S315080045C09C038179DFF8980306F0C6FADFF88C03B6
S315080045D0C179DFF8900306F0BFFADFF89C0306F00E
S315080045E0BBFAB048407800280FD0022817D011D35C
S315080045F004281ED018D3062825D01FD308282CD067
S3150800460026D30A2833D02DD335E0DFF8700306F019
S31508004610A3FA30E0DFF8680306F09EFA2BE0DFF82D
S31508004620640306F099FA26E0DFF85C0306F094FACC
S3150800463021E0DFF8580306F08FFA1CE0DFF8500394
S3150800464006F08AFA17E0DFF84C0306F085FA12E05E
S31508004650DFF8440306F080FA0DE0DFF8400306F0C1
S315080046607BFA08E0DFF8380306F076FA03E0DFF8AD
S31508004670340306F071FADFF8300306F06DFA89485C
S31508004680007800280CD001280ED0022810D0032864
S3150800469012D0042814D0062816D0072818D01AE0F5
S315080046A0B64806F059FA16E0B54806F055FA12E08B
S315080046B0B44806F051FA0EE0B34806F04DFA0AE09F
S315080046C0BA4806F049FA06E0B24806F045FA02E0AA
S315080046D0B14806F041FA1AA006F03EFA70BD00008D
S315080046E025630000B248007801280FD1B148006858
S315080046F040F6C411884207D3AE48006840F6AD516B
S31508004700884201D2012008E0002006E0A848007887
S31508004710022801D1012000E00020704780B5A44896
S315080047200078022801D106F095FD0020A0490870FE
S315080047300020DFF85C1D087000209E49086001BD56
S315080047400D0A0000F06800202F00000080B5984888
S315080047500078002803D0022875D017D39DE0DFF82B
S31508004760300D007800280DD0934806F0F5F90020A2
S31508004770DFF81C1D087000208E49086001208C494E
S31508004780087002E000208B49086086E089480068C6
S31508004790401C88490860DFF8F80C007800283ED0ED
S315080047A08448006840F6C411884213D381480068DB
S315080047B040F6AD5188420DD2804806F0CDF900206A
S315080047C0DFF8CC1C087000207A4908600220784976
S315080047D0087037E07748006840F6C41188420AD264
S315080047E0774806F0B9F90020DFF8A41C0870002005
S315080047F07049086026E06F48006840F6AD51884267
S3150800480020D3704806F0A8F90020DFF8841C087049
S3150800481000206849086000206549087012E065486C
S31508004820006840F6AD5188420CD3664806F094F904
S315080048300020DFF85C1C087000205E490860002034
S315080048405B49087029E05B480068401C59490860C4
S31508004850DFF83C0C007800280AD05B4806F07CF9A3
S315080048600020DFF82C1C087000205249086014E06C
S315080048705048006842F2283188420ED3534806F061
S315080048806BF906F0E7FC0020DFF8041C087000202E
S315080048904849086000204649087001BDA36C0020FD
S315080048A05A6C0020C06B0020786B0020C46B002077
S315080048B0926C0020936C0020876C0020886C002086
S315080048C0896C00208A6C00208B6C00208C6C002080
S315080048D07E6C0020306C0020326C00207F6C00203B
S315080048E0806C0020816C0020826C0020836C002084
S315080048F08D6C00208E6C002080010020D869002075
S31508004900386C00203A6C00203C6C00203E6C00207D
S315080049108F6C0020906C0020796C00207A6C002047
S315080049207B6C00207C6C00207D6C0020AB6C00202A
S31508004930AC6C0020AF6C0020B06C0020D46B00205B
S31508004940D06B0020A66C0020D0590108A869002069
S31508004950E8590108B0560108B0640108586B0020F0
S31508004960046601080C660108646B0020686B002069
S3150800497034610108305D0108BC6401081466010849
S31508004980C864010844610108D4640108E0640108A8
S31508004990EC64010854610108445D0108646101087A
S315080049A0585D01086C5D0108F86401087461010826
S315080049B0BA6C0020DC6B00205C4801080C45010835
S315080049C048450108E446010884450108904801085D
S315080049D02DE9F84F040000250026DFF8100C210009
S315080049E0C9B2405C002836D0012845D0022800F01C
S315080049F08D80032800F0DE82042800F0DF86052873
S31508004A0000F06D87062801F06B80072801F0BF804B
S31508004A10082801F01F81092801F084820A2801F07C
S31508004A205F830B2801F04985122801F04D81132870
S31508004A3001F07281142801F09A81152801F0CD81C0
S31508004A40162801F0E9811E2800F0D1801F2800F001
S31508004A50E58101F050BDFEF7A4FC0120DFF88C1BB0
S31508004A602200D2B288540020DFF8841B2200D2B27A
S31508004A7021F8120001F03FBDDFF8780BDFF8781B4C
S31508004A800978405C00283DD00020DFF8681BDFF875
S31508004A90682B12788854DFF8641BDFF85C0B027801
S31508004AA040204243885C002826D1DFF8A40DDFF8B1
S31508004AB0481B0978405C01281ED1DFF8980D00785C
S31508004AC000280AD1DFF8900D06F046F8DFF88C0DBD
S31508004AD00078801CDFF8841D0870FEF7B6FC0220FB
S31508004AE0DFF8081B2200D2B288540020DFF8001B2A
S31508004AF02200D2B221F812006420DFF8581D08708F
S31508004B0001F0F9BCFEF74DFC01F0F5BCDFF8E40A4C
S31508004B10DFF8E41A0978405C002864D00020DFF842
S31508004B20D41ADFF8D42A127888546420DFF8241DB2
S31508004B300870DFF81C0DDFF8C01A0978405C0228F7
S31508004B4051DB19A006F008F8DFF8140D06F004F892
S31508004B500020DFF8101D0870DFF8080D0078DFF870
S31508004B60F01CDFF8942A1278895C884220D2DFF894
S31508004B708C1ADFF8840A02784020424301EB0200CF
S31508004B80DFF8E01C0978415CDFF8DC0C05F0E4FF8F
S31508004B9006A005F0E1FFDFF8CC0C0078401CDFF832
S31508004BA0C41C0870D8E700BF0D0A000020000000EA
S31508004BB0DFF8481ADFF8400A027840204243885C4A
S31508004BC00B2810D11E20DFF8241A2200D2B28854EE
S31508004BD00020DFF81C1A2200D2B221F81200FEF7D4
S31508004BE007FD01F088BCFEF730FC01F084BCDFF855
S31508004BF0040ADFF8041A0978405C002800F00C81E2
S31508004C000020DFF8F019DFF8F029127888546420BC
S31508004C10DFF8401C0870DFF8380CDFF8DC19097873
S31508004C20405C0228C0F2F8800C27DFF8D019DFF8BC
S31508004C30C80902784020424301EB020010F103083C
S31508004C40DFF8A41DDFF8B00902780F20424301EB14
S31508004C5002093A004146484607F0B8FEDFF8881DC3
S31508004C60DFF8940902780F20424301EB020007F0AF
S31508004C7005FF00281BD00F275FF00008DFF86C9DA2
S31508004C8042463900484607F0A1FD5FF00C09DFF8F7
S31508004C90581DDFF8640902780F20424301EB020A27
S31508004CA0DFF848BD4A465146584607F08FFEDFF8FA
S31508004CB04C19DFF8440902784020424301EB020010
S31508004CC0007EDFF82C1DDFF83029127801F8220063
S31508004CD0DFF82819DFF8200902784020424301EB63
S31508004CE00200407EDFF8081DDFF80C29127801EB78
S31508004CF082014870DFF80419DFF8FC0802784020C2
S31508004D00424301EB0200807EDFF8E41CDFF8E82866
S31508004D10127801EB820188700020DFF8D41CDFF8D6
S31508004D20D828127801EB8201C870DFF8D018DFF8AE
S31508004D30C80802784020424301EB0200C17EDFF832
S31508004D406C2DDFF8B408037803204343D154DFF809
S31508004D50AC18DFF8A40802784020424301EB0200B1
S31508004D60017FDFF8482DDFF89008037803204343D6
S31508004D7002EB030041700021DFF8302DDFF87808D8
S31508004D8003780320434302EB03008170DFF8600CCD
S31508004D90DFF86418097810F821004D2807D100209B
S31508004DA0DFF84C1CDFF85028127801F82200DFF8EB
S31508004DB0400CDFF84418097800EB81004078442855
S31508004DC008D10020DFF8281CDFF82C28127801EB20
S31508004DD082014870DFF8180CDFF81C18097800EB18
S31508004DE081008078422808D10020DFF8041CDFF80B
S31508004DF00828127801EB820188701F20DFF8EC176B
S31508004E002200D2B288540020DFF8E4172200D2B27A
S31508004E1021F81200FEF7E1FA01F06DBBDFF8D407BE
S31508004E20DFF8D4170978405C002800F0C18000201C
S31508004E30DFF8C017DFF8C027127888546420DFF837
S31508004E40141A0870DFF8080ADFF8AC170978405C0E
S31508004E500228C0F2AD80DFF8A417DFF89C070278B5
S31508004E604020424301EB02004078DFF8E01C08705E
S31508004E70DFF88817DFF8800702784020424301EB05
S31508004E8002008078DFF8C81C0870DFF87017DFF8B2
S31508004E90680702784020424301EB0200C078DFF839
S31508004EA04C1D0870DFF85417DFF84C0702784020CD
S31508004EB0424301EB02000079DFF8341D0870DFF881
S31508004EC02C0D0178DFF82C0D05F046FEDFF8200DD5
S31508004ED00178DFF8240D05F03FFE0020DFF81C1DE1
S31508004EE0087010275FF00008DFF8149D4246390065
S31508004EF0484607F06BFC072005002800C0B2DFF81B
S31508004F005019DFF8F4261278895C491E884237DA88
S31508004F10DFF8E816DFF8E00602784020424301EBA6
S31508004F2002002900C9B2405C002829D0DFF8CC1657
S31508004F30DFF8C40602784020424301EB020029004C
S31508004F40C9B2405CDFF8B81C3200D2B28854761C6D
S31508004F50701EC0B2FEF704FC07F0ACFD02000B00A1
S31508004F603100C9B2491EDFF89C0C05F0F5FDDFF8E3
S31508004F708C0C0078401CDFF8841C08706D1CBCE79C
S31508004F80DFF8840C0078012801D107F039F90120EF
S31508004F90DFF8781C08700320DFF850162200D2B21A
S31508004FA088540020DFF848162200D2B221F81200F1
S31508004FB001F0A1BADFF83C06DFF83C160978405C38
S31508004FC0002800F0F7830020DFF82816DFF82826E7
S31508004FD0127888546420DFF87C180870DFF87008A7
S31508004FE0DFF814160978405C0228C0F20983DFF856
S31508004FF00C16DFF80406027840204243885C10F05D
S31508005000F00F40F0B580DFF8080C0178DFF8EC25E2
S31508005010DFF8E405037840204343D05C814205D19C
S31508005020DFF8EC0B0078012840F0EA82BBA005F017
S3150800503093FDDFF82C0805F08FFDDFF8C015DFF8C3
S31508005040B8050278402042438F5C3800C0B2022877
S3150800505007DB3800C0B20E2803DA3800C0B206F003
S31508005060D4F8DFF89815DFF8900502784020424317
S31508005070885C012813D06FD303282BD025D30528A5
S3150800508032D02CD3072839D033D3092846D03AD37F
S315080050900B2853D04DD30D285AD054D35CE00120A9
S315080050A0DFF8EC130870FFF71DFB002806D0DFF8C1
S315080050B0640B05F051FD06F0C2F805E0DFF8580B61
S315080050C005F04AFD06F0B0F846E0DFF8500B05F0AB
S315080050D043FD41E0DFF8980D05F03EFD3CE0DFF8C2
S315080050E0940D05F039FD37E0DFF88C0D05F034FD39
S315080050F032E0DFF8880D05F02FFD2DE0DFF8800D92
S3150800510005F02AFD28E001220121DFF87C0D07F0D1
S315080051101EFBDFF8780D05F01FFD1DE001220121B9
S31508005120DFF8640D07F013FBDFF8640D05F014FDD6
S3150800513012E0DFF8600D05F00FFD0DE0DFF8580D01
S3150800514005F00AFD08E0DFF8540D05F005FD03E05B
S31508005150DFF84C0D05F000FDDFF8A014DFF8980421
S31508005160027840204243885CDFF8A41A087021E3DD
S315080051706AA005F0F1FCDFF8E80605F0EDFCDFF8BB
S315080051807C14DFF87404027840204243885C10F0EF
S31508005190F000C0B2402806D0502800F02D817028B3
S315080051A000F00C820FE2DFF8FC0C05F0D5FCDFF806
S315080051B04C14DFF84404027840204243885C10F01F
S315080051C00F00102880F20281DFF83C0A00780128D7
S315080051D05ED1DFF82814DFF8200402784020424325
S315080051E0885C10F00F00FEF7BBFA07F063FC0200BC
S315080051F00B00DFF80814DFF800040778402047435F
S31508005200C95D11F00F01DFF8A00C05F0A5FCDFF869
S315080052109C1CDFF8E823DFF8E003037840204343CB
S31508005220D25C12F00F02DFF8843CDFF8D073DFF8A7
S31508005230C80390F800C0402000FB0CFC17F80C00CF
S3150800524010F00F0033F81000401C21F81200DFF8A8
S31508005250641CDFF8A823DFF8A00303784020434343
S31508005260D25C12F00F02DFF84C3CDFF89073DFF8DF
S31508005270880390F800C0402000FB0CFC17F80C00CF
S3150800528010F00F0033F81000401C21F812009DE0C2
S31508005290DFF86813DFF86003027840204243885C31
S315080052A010F00F00FEF75CFA5FF07E5107F026FC5F
S315080052B012D1DFF8800D05F04FFCDFF87C0D008871
S315080052C0401CDFF8741D0880DFF8700D0088401C4C
S315080052D0DFF8681D088079E0C849C7480278402089
S315080052E04243885C10F00F00FEF73AFA5FF08041FF
S315080052F007F004FC14D1DFF8480D05F02DFCDFF8A3
S31508005300440D0088401CDFF83C1D0880DFF8380D86
S315080053100088401CDFF8301D088057E00D0A0000A1
S31508005320B649B548027840204243885C10F00F0021
S31508005330FEF716FADFF8141D07F0E0FB12D1DFF8C6
S31508005340100D05F009FCDFF80C0D0088401CDFF88D
S31508005350041D0880DFF8000D0088401CDFF8F81CE3
S31508005360088033E0A549A448027840204243885C77
S3150800537010F00F00FEF7F4F9DFF8E01C07F0BEFBAB
S3150800538012D1DFF8DC0C05F0E7FBDFF8D80C008853
S31508005390401CDFF8D01C0880DFF8CC0C0088401CC5
S315080053A0DFF8C41C088011E094499348027840202D
S315080053B04243885C10F00F00FEF7D2F907F07AFB3B
S315080053C002000B00DFF8A40C05F0C6FB8B498A48DF
S315080053D002784020424301EB0200417882A005F0A2
S315080053E0BBFBDFF88C0C05F0B7FBFFF797F906F067
S315080053F06BF806F0EBF9DDE1DFF8780C05F0ACFBAD
S315080054007E497D48027840204243885C10F00F00B0
S31508005410102880F2BD80DFF8F0070078012839D11E
S3150800542076497548027840204243885C10F00F00A0
S31508005430FEF796F907F03EFB02000B006F496E482F
S31508005440077840204743C95D11F00F01DFF8580A75
S3150800545005F082FBDFF8541A684A6748037840204B
S315080054604343D25C12F00F02DFF8403A634F6248BA
S3150800547090F800C0402000FB0CFC17F80C0010F058
S315080054800F0033F81000401C21F8120080E000BF1E
S31508005490B96C002059495848027840204243885C34
S315080054A010F00F00FEF75CF95FF07E5107F026FB5F
S315080054B00BD1DFF8800B05F04FFBDFF87C0B00887B
S315080054C0401CDFF8741B088062E04C494A480278A1
S315080054D040204243885C10F00F00FEF741F95FF068
S315080054E0804107F00BFB0BD1DFF8540B05F034FBBA
S315080054F0DFF8500B0088401CDFF8481B088047E09F
S315080055003E493D48027840204243885C10F00F002F
S31508005510FEF726F9DFF8341B07F0F0FA0BD1DFF8AF
S31508005520300B05F019FBDFF82C0B0088401CDFF860
S31508005530241B08802CE031492F480278402042433A
S31508005540885C10F00F00FEF70BF9DFF8101B07F068
S31508005550D5FA0BD1DFF8080B05F0FEFADFF8040BD5
S315080055600088401CDFF8FC1A088011E0234922480D
S31508005570027840204243885C10F00F00FEF7F0F8EE
S3150800558007F098FA02000B00DFF8E00A05F0E4FAE3
S315080055901A49194802784020424301EB0200417833
S315080055A011A005F0D9FADFF87C0D05F0D5FAFFF75A
S315080055B0B5F805F089FF06F009F9FBE0DFF8680D94
S315080055C005F0CAFAF6E0DFF8640D05F0C5FA0B49EE
S315080055D00948027840204243895CA34805F0BCFA92
S315080055E0A2A005F0B9FAE5E025640000C06B00202A
S315080055F0786B0020CC6B0020A86C00207863002014
S31508005600DFF82C0D0078002828D00027DFF8240DB5
S315080056100078DFF8241D91F8008058EA0018002069
S31508005620DFF80C1D08704046C0B2FDF75AFF00208F
S31508005630DFF8001D08700020DFF8FC1C0870122037
S31508005640DFF8B41D2200D2B288540020DFF8AC1D62
S315080056502200D2B221F8120000F04DBFDFF8A00DEB
S31508005660007801281BD10020DFF8941D0870DFF8A8
S31508005670940D0078002810D10220DFF88C1D0870E0
S315080056801520DFF8741D2200D2B288540020DFF8F6
S315080056906C1D2200D2B221F8120000F02CBFDFF8F0
S315080056A0C40D0078002823D00020DFF8B81D087044
S315080056B0DFF8B80D0078DFF8B81D0870DFF8AC0D14
S315080056C00078DFF8B01D0870DFF8A00D0078FDF748
S315080056D0B3FF0820DFF8201D2200D2B2885400202C
S315080056E0DFF8181D2200D2B221F8120000F003BF1D
S315080056F0DFF8840D0078002818D00020DFF8781D20
S31508005700087000230022FF21FF20FDF7BAFE0620BD
S31508005710DFF8E41C2200D2B288540020DFF8DC1C33
S315080057202200D2B221F8120000F0E5BEDFF84C0DD7
S315080057300078002818D00020DFF8401D08700023E4
S31508005740002200210020FDF79CFE0720DFF8A81C98
S315080057502200D2B288540020DFF8A01C2200D2B260
S3150800576021F8120000F0C7BEDFF8A0040078002870
S3150800577020D0DFF898040078401EDFF890140870EF
S31508005780DFF888040078002814D13220DFF87C146A
S315080057900870FDF7C1FF0420DFF85C1C2200D2B2B6
S315080057A088540020DFF8541C2200D2B221F81200D7
S315080057B000F0A1BEFDF749FE00F09DBEDFF8580DCA
S315080057C0DFF8581D0978405C002877D00020DFF8FC
S315080057D0481DDFF8482D1278885464201D49087042
S315080057E0DFF83C0D0178DFF83C2DDFF8300D037843
S315080057F040204343D05C81423DD0D2A005F0ACF9AD
S31508005800DFF8240D05F0A8F9002016490870154898
S3150800581000780F49DFF8042D1278895C884227D270
S31508005820DFF8001DDFF8F40C02784020424301EB54
S3150800583002000C490978415C0B4805F08DF9C2A0B5
S3150800584005F08AF907480078401C06490870DEE723
S31508005850C86B0020926C0020005A0108A66C002034
S3150800586084610108BB6C0020046601082900000059
S31508005870B4A005F071F9DFF8AC1CDFF8A00C0278CB
S3150800588040204243885C15280DD1DFF8981CDFF8C4
S315080058908C0C02784020424301EB02004078022833
S315080058A001D1FDF74EFCDFF87C1CDFF8700C02789E
S315080058B040204243885CDFF8681C0870FDF7A9FDA4
S315080058C00520DFF8341B2200D2B288540020DFF806
S315080058D02C1B2200D2B221F8120000F00CBEDFF811
S315080058E0380CDFF8381C0978405C002800F0F68090
S315080058F00020DFF8241CDFF8242C12788854642052
S31508005900DFF8281C0870C048007801282DD1202708
S315080059105FF00008DFF8189C42463900484606F052
S3150800592055FF002006003000C0B2102880F2C08063
S315080059303000C0B2FDF714FF002107F0EDF812D2CF
S31508005940DFF8E01BDFF8D40B02784020424301EB76
S3150800595002003100C9B208448078DFF8D41B32004F
S31508005960D2B221F81200761CDDE70020DFF8C81B4A
S3150800597008800020DFF8C41B08800020DFF8C01B61
S3150800598008800020DFF8BC1B0880002006003000D5
S31508005990C0B2102880F28C803000C0B2FDF7E0FE5D
S315080059A0002107F0B9F880F07E803000C0B2FDF71C
S315080059B0D7FE5FF07E5107F0A1F81BD1DFF8780B10
S315080059C00188DFF8602BDFF8540B03784020434347
S315080059D002EB03003200D2B2104480784118DFF897
S315080059E0580B01805FE000BFA8690020DC6A002030
S315080059F0646B00203000C0B2FDF7B2FE5FF0804154
S31508005A0007F07CF814D1DFF8340B0188DFF8142B83
S31508005A10DFF8080B03784020434302EB030032000B
S31508005A20D2B2104480784118DFF8100B01803AE0B2
S31508005A303000C0B2FDF794FEDFF8101607F05EF8E6
S31508005A4014D1DFF8FC0A0188DFF8D82ADFF8CC0A77
S31508005A5003784020434302EB03003200D2B21044DD
S31508005A6080784118DFF8D80A01801CE03000C0B2FF
S31508005A70FDF776FEDFF8E41507F040F813D1DFF8F6
S31508005A80C40A0188DFF89C2ADFF8900A03784020C8
S31508005A90434302EB03003200D2B210448078411827
S31508005AA0DFF8A00A0180761C71E700BF586B00205A
S31508005AB0DFF854090078002803D10120DFF84819D7
S31508005AC008700320DFF830192200D2B2885400206B
S31508005AD0DFF828192200D2B221F8120000F00BBD17
S31508005AE0DFF8340ADFF8341A0978405C00284CD00D
S31508005AF00020DFF8241ADFF8242A12788854642054
S31508005B00DFF8281A0870DFF81C1ADFF8100A02787E
S31508005B1040204243885C00281CD1DFF82C0ADFF8B5
S31508005B20FC190978405C012814D10120DFF8D41843
S31508005B30087004A005F010F8DFF8100A05F00CF854
S31508005B4014E000BF0D0A000020000000706C002061
S31508005B506F6C002001220121CB4806F0F8FDC9A090
S31508005B6004F0FAFFDFF8E80904F0F6FF05F089FE0D
S31508005B700320DFF884182200D2B288540020DFF808
S31508005B807C182200D2B221F8120000F0B4BCDFF86B
S31508005B908809DFF888190978405C002858D0002061
S31508005BA0DFF87419DFF87429127888546420DFF84E
S31508005BB07C190870DFF86C19DFF860090278402054
S31508005BC04243885C00282BD1DFF87C09DFF84C19A2
S31508005BD00978405C012823D10020DFF828180870CE
S31508005BE0DFF8700904F0B8FF23E000BF716C0020ED
S31508005BF0726C0020CC560108E8560108736C002028
S31508005C00BC6A0020185A01087E010020A96C0020F1
S31508005C10AB6C0020805D010894610108945D010861
S31508005C2001220121984806F092FDDFF82C0904F0BC
S31508005C3093FF05F026FE0320DFF8BC172200D2B238
S31508005C4088540020DFF8B4172200D2B221F81200D7
S31508005C5000F051BCDFF8C008DFF8C0180978405CCE
S31508005C6000282FD00020DFF8B018DFF8B028127807
S31508005C7088546420DFF8B418087082A004F06CFF1A
S31508005C80DFF8D80804F068FFDFF8E407017888A091
S31508005C9004F062FFDFF8C80804F05EFFFDF718FDA0
S31508005CA04FF4FA70DFF8BC1808600920DFF84817C7
S31508005CB02200D2B288540020DFF840172200D2B260
S31508005CC021F8120000F017BCDFF84C08DFF84C1872
S31508005CD00978405C00281ED00020DFF83C18DFF861
S31508005CE03C28127888546420DFF84018087065A0AC
S31508005CF004F032FFDFF8700804F02EFF1320DFF8F7
S31508005D00F8162200D2B288540020DFF8F0162200D6
S31508005D10D2B221F81200EEE35AA004F01DFFDFF814
S31508005D204C0804F019FFFDF790FB4FF4FA70DFF802
S31508005D30341808604B20DFF8381808600020DFF8B0
S31508005D40D817DFF8D827127888546420DFF8DC17CC
S31508005D5008701420DFF8A0162200D2B2885400205A
S31508005D60DFF898162200D2B221F81200C3E3DFF852
S31508005D70A807DFF8A8170978405C00282CD0DFF8B8
S31508005D80F0070068002827D06420DFF8A0170870FD
S31508005D90DFF8DC070068401EDFF8D4170860DFF874
S31508005DA0D0070068002817D136A004F0D5FEDFF822
S31508005DB0C40704F0D1FE022005F0BAFD0320DFF87F
S31508005DC038162200D2B288540020DFF83016220096
S31508005DD0D2B221F812008EE38DE30020DFF83817DF
S31508005DE0DFF83827127888546420DFF840170870DF
S31508005DF0FDF79BFB4B20DFF8801708601620DFF8BD
S31508005E00F8152200D2B288540020DFF8F0152200D7
S31508005E10D2B221F812006EE3DFF8FC06DFF8FC16B2
S31508005E200978405C002847D00020DFF8EC16DFF838
S31508005E30EC26127888546420DFF8F0160870DFF82C
S31508005E403C0704F089FE012005F081FD0020DFF8FB
S31508005E50B81508700320DFF8A0152200D2B28854BE
S31508005E600020DFF898152200D2B221F8120042E38A
S31508005E7004650108305A0108A4610108A85D0108F3
S31508005E80106501080D0A000000100140BC5D0108FC
S31508005E90D05D0108B4610108E45D01081C650108CC
S31508005EA010520108C4610108F85D0108F86900206C
S31508005EB025640000186A0020DFF8BC060068002880
S31508005EC02FD06420DFF864160870DFF8AC06006887
S31508005ED0401EDFF8A4160860DFF89C060068002854
S31508005EE01FD1DFF89C0604F037FE012005F02FFDD0
S31508005EF00020DFF82416DFF82426127888540020BC
S31508005F00DFF8041508700320DFF8EC142200D2B27B
S31508005F1088540020DFF8E4142200D2B221F81200D7
S31508005F20E9E2E8E2DFF8F005DFF8F0150978405C09
S31508005F30002800F0A5800020DFF8DC15DFF8DC2556
S31508005F40127888546420DFF8E4150870DFF8D41551
S31508005F50DFF8C805027840204243885C002826D12D
S31508005F60DFF8E405DFF8B4150978405C01281ED18E
S31508005F700020DFF8F8140870DBA004F0EDFDDFF868
S31508005F80040604F0E9FDFDF77FFB0020DFF8D415D1
S31508005F9008600A20DFF860142200D2B28854002074
S31508005FA0DFF858142200D2B221F81200A3E2DFF873
S31508005FB07415DFF86805027840204243885C00289B
S31508005FC05AD0DFF8AC040178DFF85825DFF84C051D
S31508005FD0037840204343D05C091ADFF89404017023
S31508005FE0C1A004F0B9FDDFF8740504F0B5FDDFF8CB
S31508005FF080040178CAA004F0AFFDDFF8640504F058
S31508006000ABFDDFF86C04007805F0B0FCDFF864043B
S315080060100078DFF85C140978884204D04FF4FA70E7
S31508006020DFF840150860DFF848040078DFF8441404
S31508006030087025E01C660108406C0020486C0020AA
S3150800604024660108426C00204A6C00200000A0402B
S315080060502C660108446C00204C6C0020000020418E
S3150800606034660108466C00204E6C00203C66010828
S3150800607044660108286501086420DFF8B014087032
S31508006080DFF8E0040068002827D105F07EFC002030
S31508006090DFF88414DFF88424127888546420DFF843
S315080060A08C1408700020DFF8BC1408608EA004F079
S315080060B053FDDFF8D40404F04FFDDFF8D00404F0F4
S315080060C04BFD0B20CC492200D2B288540020CB4984
S315080060D02200D2B221F812000DE2FDF7F9FA0AE21F
S315080060E0DFF83404DFF834140978405C002800F03F
S315080060F04D81DFF85404DFF824140978405C102831
S31508006100C0F244810020DFF81014DFF8102412785A
S3150800611088546420DFF81414087073A004F01CFD7A
S31508006120DFF86C0404F018FD0020DFF86814087026
S31508006130DFF860040078DFF81014DFF8E02312783F
S31508006140895C88421BD2DFF8DC13DFF8D0030278BB
S315080061504020424301EB0200DFF838140978415C1D
S31508006160DFF8340404F0F8FCBFA004F0F5FCDFF80F
S3150800617024040078401CDFF81C140870D8E7DFF800
S315080061801C040078012844D110275FF00008DFF8C6
S31508006190109442463900484606F018FBDFF8040416
S315080061A004F0DAFC002006003000C0B2102825DA18
S315080061B03000C0B2FDF7D4FA002106F0ADFC1BD2C0
S315080061C0DFF86013DFF8540302784020424301EBFE
S315080061D002003100C9B2405CDFF8C4133200D2B203
S315080061E08854DFF8BC033100C9B2425C3100C9B239
S315080061F0DFF8B40304F0B0FC761CD5E73AA004F047
S31508006200ABFCDFF8A8030178DFF8940305F0C8FBB8
S31508006210AAE00020DFF8981308700020DFF894132E
S3150800622008700020DFF8901308700020DFF88C1340
S315080062300870002006003000C0B2102880F27E8068
S315080062403000C0B2FDF78CFA002106F065FC64D276
S315080062503000C0B2FDF784FA5FF07E5106F04EFCBE
S3150800626011D1DFF84C030178AE4AAC4803784020D8
S31508006270434302EB03003200D2B2805C4118DFF8D8
S315080062803003017049E03000C0B2FDF769FA5FF0EB
S31508006290804106F033FC0FD1C6480178A14A9F48D1
S315080062A003784020434302EB03003200D2B2805CFD
S315080062B04118C048017030E03000C0B2FDF750FA0E
S315080062C0BF4906F01BFC11D1BB480178954A934893
S315080062D003784020434302EB03003200D2B2805CCD
S315080062E04118B548017018E00D0A00003000C0B228
S315080062F0FDF736FAB34906F001FC0ED1AF4801782E
S31508006300884A864803784020434302EB030032005C
S31508006310D2B2805C4118A9480170761C8BE700BF91
S31508006320256400004C6601083465010854660108B6
S31508006330796C00207B6C00207A6C00209F480078DE
S3150800634000909D4803789B480278994801789E48B2
S3150800635004F002FC99480378974802789548017832
S315080063609348007805F04AFB00230022002100200C
S31508006370FDF787F8072020492200D2B2885400206A
S315080063801E492200D2B221F81200B4E062486349DD
S315080063900978405C002800F08F8000205E495F4A3B
S315080063A01278885464206149087062A004F0D4FB0E
S315080063B0864804F0D1FB00207649087075480078B5
S315080063C06149564A1278895C88421FD25549534812
S315080063D002784020424301EB02006E490978415C8D
S315080063E06D4804F0B9FB20A004F0B6FB69480078B4
S315080063F0401C68490870E1E7C06B0020786B0020F4
S31508006400786C00208F6C00208101002010275FF037
S315080064100008DFF88C9142463900484606F0D6F95E
S31508006420002063490870002062490870002062490C
S3150800643008700020614908706048007800905E483E
S3150800644003785C4802785A4801785F4804F084FB70
S3150800645052480078012813D154480178504805F06D
S315080064609FFA17E07C6C0020200000007D6C00205D
S31508006470B16C0020B26C0020876C00208A6C00206A
S315080064804E4803784C4802784A48017848480078CC
S3150800649005F0B4FA0023002200210020FCF7F1FFE2
S315080064A007204B492200D2B28854002049492200CD
S315080064B0D2B221F812001EE01DE0174817490978E4
S315080064C0405C002815D000201349144A12788854D5
S315080064D0642016490870FDF7D7F80A203C492200BF
S315080064E0D2B2885400203B492200D2B221F81200C9
S315080064F001E0FDF7EDF83848007800280AD036485C
S315080065000078401E3449087033480078002801D1C5
S3150800651005F08FFABDE8F18FCC6B0020A86C00203F
S31508006520AF6C002078630020D4610108926C0020CB
S31508006530D86900200D0A0000386C00203A6C00204B
S315080065403C6C00203E6C0020C86B00200C5E0108E5
S31508006550485A01080457010820570108205E010817
S315080065605C660108D46B0020605A0108345E010895
S31508006570D86B0020485E0108D06B00203052010815
S31508006580505201085C5E0108705E01083C5701081C
S31508006590785A0108BB6C0020046601087E010020B9
S315080065A0EC6A0020E461010840650108736C00206C
S315080065B0B36C0020B46C0020B56C0020B66C0020CB
S315080065C00000A04000002041704B010870520108ED
S315080065D0C06B0020786B0020956C00202DE9F84FE1
S315080065E0040000250026DFF81C0C2100C9B2405C17
S315080065F000285DD001286CD0022800F0B780032857
S3150800660000F09082042800F0DA86062800F0108749
S31508006610072800F062871E2800F017811F2800F05F
S315080066209E81C82800F0AC87C92800F0C287CA280E
S3150800663001F09D80CB2801F0B780CC2801F07F813E
S31508006640CD2801F09981D22801F06D82D32801F076
S315080066509682D42801F0DC82D52801F0FE82DC2857
S3150800666001F03383DD2801F0AE83DE2801F074845F
S31508006670DF2801F01785E62801F02F85E72801F0C5
S315080066804D85E82801F00086F02801F03E86F128BD
S3150800669001F05186FA2801F09686FB2801F0DB8680
S315080066A0FC2801F0FF86FF2801F0418701F04CBF66
S315080066B0FDF77AF80120DFF84C1B2200D2B2885485
S315080066C00020DFF8441B2200D2B221F8120001F0A4
S315080066D03BBFDFF8380BDFF8381B0978405C002829
S315080066E040D00020DFF8241BDFF8242B12788854CA
S315080066F0DFF8201BDFF8180B027840204243885C3D
S31508006700002829D1DFF8880DDFF8041B0978405CDA
S31508006710012821D1DFF87C0D007800280DD1E4A0EE
S3150800672004F01AFADFF8700D04F016FADFF86C0DAB
S315080067300078401CDFF8641D0870FDF763F8022036
S31508006740DFF8C01A2200D2B288540020DFF8B81A3F
S315080067502200D2B221F812006420DFF8381D087032
S3150800676001F0F2BEFDF720F801F0EEBEDFF89C0A54
S31508006770DFF89C1A0978405C002862D00020DFF810
S315080067808C1ADFF88C2A127888546420DFF8041DE6
S315080067900870DFF8FC0CDFF8781A0978405C0228E4
S315080067A04FDBC3A004F0D8F9DFF88C0D04F0D4F958
S315080067B00020DFF8881D0870DFF8800D0078DFF804
S315080067C0D01CDFF84C2A1278895C88421BD2DFF885
S315080067D0441ADFF83C0A02784020424301EB0200E3
S315080067E0DFF8581D0978415CDFF8540D04F0B4F958
S315080067F0CBA004F0B1F9DFF8440D0078401CDFF8AF
S315080068003C1D0870D8E7AAA004F0A6F9DFF8041A18
S31508006810DFF8FC09027840204243885C062810D13C
S315080068201E20DFF8E0192200D2B288540020DFF8D3
S31508006830D8192200D2B221F81200FDF76FF801F03C
S3150800684083BEFCF7DFFF01F07FBEDFF8C009DFF883
S31508006850C0190978405C002800F07F800020DFF826
S31508006860AC19DFF8AC29127888546420DFF8241CA8
S315080068700870DFF81C0CDFF898190978405C0228C4
S315080068806BDB0F275FF00008DFF8B81CDFF880091C
S3150800689002780F20424301EB020942463900484676
S315080068A005F094FF5FF00C09DFF86819DFF8600956
S315080068B002784020424301EB020010F1030ADFF898
S315080068C0841CDFF84C0902780F20424301EB020BC7
S315080068D04A465146584606F079F8DFF83819DFF87F
S315080068E0300902784020424301EB0200C17EDFF8FE
S315080068F0582CDFF81C09037803204343D154DFF8EA
S315080069001419DFF80C0902784020424301EB020013
S31508006910017FDFF8342CDFF8F808037803204343B7
S3150800692002EB030041700021DFF81C2CDFF8E008B9
S3150800693003780320434302EB030081701F20DFF82E
S31508006940C4182200D2B288540020DFF8BC182200EE
S31508006950D2B221F81200FCF73EFF01F0F5BDDFF8D0
S31508006960AC08DFF8AC180978405C002800F0D6803F
S315080069700020DFF89818DFF89828127888546420E1
S31508006980DFF8CC1C0870DFF8080BDFF884180978E4
S31508006990405C0228C0F2C280DFF87818DFF8700879
S315080069A002784020424301EB02004078DFF8A41C3D
S315080069B00870DFF86018DFF858080278402042436C
S315080069C001EB02008078DFF8901C0870DFF84418A5
S315080069D0DFF83C0802784020424301EB0200C07809
S315080069E0DFF8781C0880DFF8740C0188DFF82428A3
S315080069F0DFF81C0803784020434302EB03000079C4
S31508006A0050EA0120DFF8541C0880DFF80818DFF880
S31508006A10000802784020424301EB02004079DFF883
S31508006A20401C0870DFF8340C0188DFF8380C04F0D5
S31508006A3093F8DFF82C0C0178DFF82C0C04F08CF8AE
S31508006A400020DFF8281C087010275FF00008DFF820
S31508006A50209C42463900484605F0B8FE0B20050042
S31508006A602800C0B2DFF8281ADFF8A4271278895C54
S31508006A70491E88423ADADFF89C17DFF8940702784D
S31508006A804020424301EB02002900C9B2405C0028BD
S31508006A902CD0DFF88017DFF87807027840204243C9
S31508006AA001EB02002900C9B2405CDFF8C41B01E013
S31508006AB00D0A00003200D2B28854761C701EC0B28D
S31508006AC0FCF74AFF05F0F6FF02000B003100C9B2D9
S31508006AD0491EDFF8A00B04F03FF8DFF8900B0078AA
S31508006AE0401CDFF8881B08706D1CB9E7DFF8880BB7
S31508006AF00078012801D105F0C7FB0120DFF87C1BCF
S31508006B0008700320DFF8FC162200D2B28854002051
S31508006B10DFF8F4162200D2B221F8120001F014BDF3
S31508006B2020000000DFF8E406DFF8E4160978405C88
S31508006B30002800F040840020DFF8D016DFF8D026C1
S31508006B40127888546420DFF84C190870DFF8400979
S31508006B50DFF8BC160978405C0228C0F22A83DFF801
S31508006B60B416DFF8AC06027840204243885C10F081
S31508006B70F00F40F09380DFF8080B0178DFF89426D1
S31508006B80DFF88C06037840204343D05C814200F04E
S31508006B901083C2A003F0E0FFDFF89C0903F0DCFFD6
S31508006BA0DFF87016DFF868060278402042438F5CEB
S31508006BB03800C0B2002807D03800C0B20D2803DA62
S31508006BC03800C0B204F040FFDFF84816DFF8400688
S31508006BD0027840204243885C012812D052D3032809
S31508006BE019D013D3052826D01AD307282DD027D392
S31508006BF0092834D02ED30B283BD035D30C283DD0CA
S31508006C0040E0DFF8840A03F0A7FF3BE0DFF87C0AE0
S31508006C1003F0A2FF36E0DFF8780A03F09DFF31E0C3
S31508006C2001220121DFF86C0A05F091FDDFF8680AF8
S31508006C3003F092FF26E0DFF8640A03F08DFF21E0F7
S31508006C40DFF85C0A03F088FF1CE0DFF8580A03F057
S31508006C5083FF17E0DFF8500A03F07EFF12E0DFF843
S31508006C604C0A03F079FF0DE0DFF8440A03F074FFDD
S31508006C7008E0DFF8400A03F06FFF03E0DFF8380AA0
S31508006C8003F06AFFDFF88C15DFF8840502784020E8
S31508006C904243885CDFF8E81908708CE37FA003F0AC
S31508006CA05BFFDFF8940803F057FF0020DFF88C1825
S31508006CB00870DFF888080078DFF8D417DFF8502561
S31508006CC01278895C88421BD2DFF84815DFF8400540
S31508006CD002784020424301EB0200DFF86018097889
S31508006CE0415CDFF85C0803F037FFA9A003F034FF26
S31508006CF0DFF848080078401CDFF840180870D8E725
S31508006D00DFF81015DFF80805027840204243885C52
S31508006D1010F0F000C0B2802815D0902800F03A8113
S31508006D20A02800F02282B02800F02A82C02800F0AD
S31508006D302C82D02800F02E82E02800F03082F0283D
S31508006D4000F0328237E3DFF8280D03F005FFDFF89D
S31508006D50C414DFF8BC04027840204243885C10F073
S31508006D600F00102880F21381DFF80C09007801283B
S31508006D704DD1DFF8A014DFF898040278402042438A
S31508006D80885C10F00F00FCF7E7FD05F093FE0200A3
S31508006D900B00DFF88014DFF87804077840204743B3
S31508006DA0C95D11F00F01DFF8CC0C03F0D5FEDFF852
S31508006DB06414DFF85C04027840204243885C10F0D3
S31508006DC00F00DFF8B41C0870DFF8B01CDFF84424A5
S31508006DD0DFF83C04037840204343D25C12F00F02EC
S31508006DE0DFF8983CDFF82C74DFF8240490F800C02C
S31508006DF0402000FB0CFC17F80C0010F00F0033F8CD
S31508006E001000401C21F8120004F05EFBBFE0DFF81A
S31508006E100414DFF8FC03027840204243885C10F033
S31508006E200F00FCF799FDDFF8581C05F067FE11D135
S31508006E30DFF8500C03F090FE0020DFF83C1C0870C9
S31508006E40DFF8440C0088401CDFF83C1C088004F07E
S31508006E503BFB9CE0DFF8BC13DFF8B4030278402064
S31508006E604243885C10F00F00FCF776FDDFF81C1C27
S31508006E7005F044FE14D1DFF8180C03F06DFE01206E
S31508006E80DFF8F41B0870DFF80C0C0088401CDFF8EC
S31508006E90041C088004F018FB79E000BF0D0A000006
S31508006EA0DFF87013DFF86803027840204243885CF5
S31508006EB010F00F00FCF750FDDFF8DC1B05F01EFE96
S31508006EC011D1DFF8D80B03F047FE0220DFF8A81B24
S31508006ED00870DFF8CC0B0088401CDFF8C41B08805C
S31508006EE004F0F2FA53E0CB49C948027840204243FD
S31508006EF0885C10F00F00FCF72FFDDFF8A81B05F0E3
S31508006F00FDFD11D1DFF8A00B03F026FE0320DFF804
S31508006F10681B0870DFF8940B0088401CDFF88C1B90
S31508006F20088004F0D1FA32E0BA49B948027840201C
S31508006F304243885C10F00F00FCF70EFDDFF8701B6B
S31508006F4005F0DCFD11D1DFF86C0B03F005FE04201B
S31508006F50DFF8241B0870DFF8600B0088401CDFF898
S31508006F60581B088004F0B0FA11E0AA49A84802782C
S31508006F7040204243885C10F00F00FCF7EDFC05F05A
S31508006F8099FD02000B00DFF87C0D03F0E5FD12E227
S31508006F9020000000DFF8700D03F0DEFD9D499C48D7
S31508006FA0027840204243885C10F00F00102880F2D7
S31508006FB0DB80DFF8C406007801282AD19549944871
S31508006FC0027840204243885C10F00F00FCF7C4FCAE
S31508006FD005F070FD02000B008E498D4807784020A9
S31508006FE04743C95D11F00F01DFF8880A03F0B4FDC5
S31508006FF088498748027840204243885C10F00F0091
S31508007000DFF8741A0870DFF8700A007804F02BFDB0
S31508007010AAE080497E48027840204243885C10F006
S315080070200F00FCF799FCDFF8581A05F067FD0DD13B
S31508007030DFF8500A03F090FD0020DFF83C1A0870CC
S31508007040DFF8340A007804F00EFD8DE071497048C7
S31508007050027840204243885C10F00F00FCF77CFC65
S31508007060DFF8281A05F04AFD0DD1DFF8240A03F0E7
S3150800707073FD0120DFF8001A0870DFF8FC090078B4
S3150800708004F0F1FC70E0634961480278402042430D
S31508007090885C10F00F00FCF75FFCDFF8FC1905F0C0
S315080070A02DFD0DD1DFF8F40903F056FD0220DFF8B7
S315080070B0C8190870DFF8C009007804F0D4FC53E05A
S315080070C054495348027840204243885C10F00F0028
S315080070D0FCF742FCDFF8CC1905F010FD0DD1DFF8FE
S315080070E0C80903F039FD0320DFF88C190870DFF8AA
S315080070F08809007804F0B7FC36E046494448027827
S3150800710040204243885C10F00F00FCF725FCDFF8AE
S31508007110A01905F0F3FC0DD1DFF8980903F01CFD62
S315080071200420DFF854190870DFF84C09007804F0D9
S315080071309AFC19E037493648027840204243885C71
S3150800714010F00F00FCF708FC05F0B4FC02000B0079
S31508007150DFF8B00B03F000FD0120DFF8B01B087064
S31508007160FE20DFF81419087025E1DFF8A40B03F0F8
S31508007170F3FCFF20DFF80019087004F083FC1AE11D
S31508007180DFF8900B03F0E8FC15E1DFF88C0B03F051
S31508007190E3FC10E1DFF8840B03F0DEFC0BE1DFF81B
S315080071A0800B03F0D9FC06E1DFF8780B03F0D4FC7A
S315080071B001E1DFF8740B007800280CD00020DFF816
S315080071C0681B0870DFF8B0080078FF2803D0FCF7C2
S315080071D070FB01F0B9B9DFF8340B007800281BD032
S315080071E00020DFF8281B0870DFF88C080078FF28D5
S315080071F012D0FF20DFF880180870FCF73EFB01F07C
S31508007200A3B900BFC06B0020786B0020CC6B0020B0
S31508007210A86C002078630020DFF8100B007800289F
S3150800722018D00020DFF8041B0870FF23FF22FF2177
S31508007230FF20FCF7FDFA0620DFF8F41A2200D2B286
S3150800724088540020DFF8EC1A2200D2B221F8120086
S3150800725001F07AB9DFF8E00A0078002818D0002093
S31508007260DFF8D41A08700023002200210020FCF75A
S31508007270DFFA0720DFF8B81A2200D2B288540020B5
S31508007280DFF8B01A2200D2B221F8120001F05CB978
S31508007290DFF8A80A007800286CD00020DFF8A01ACA
S315080072A008600020DFF89C1A0870A649DFF8140D5C
S315080072B002780F204243885C30280AD1A149DFF8BA
S315080072C0040D02780F20424301EB0200407836286D
S315080072D027D09C49DFF8EC0C02780F204243885CE3
S315080072E000280AD19749DFF8DC0C02780F204243C0
S315080072F001EB02004078002813D09249DFF8C40C4D
S3150800730002780F204243885C202824D18D49DFF873
S31508007310B40C02780F20424301EB02004078202883
S3150800732019D10020DFF8641D08700020DFF8101A54
S3150800733008600020DFF80C1A0870FB20DFF8F01947
S315080073402200D2B288540020DFF8E8192200D2B20F
S3150800735021F812000CE0C820DFF8D4192200D2B2B6
S3150800736088540020DFF8CC192200D2B221F8120086
S3150800737001F0EAB8C148007800281CD0BF48007858
S31508007380401EBE490870BD480078002813D1322037
S31508007390BA490870FCF7A9FA0420DFF89419220004
S315080073A0D2B288540020DFF88C192200D2B221F814
S315080073B0120001F0C9B8FCF725FA01F0C5B8DFF8E4
S315080073C0D00CDFF8001C0978405C00282ED000207D
S315080073D0DFF8BC1CDFF8EC2B1278885464202D49A2
S315080073E00870DFF8BC1DDFF8DC0B0278402042434A
S315080073F0885CDFF8A01C0870DFF8A41DDFF8C40B52
S3150800740002784020424301EB02004078DFF8881CEE
S3150800741008700320DFF818192200D2B28854002019
S31508007420DFF810192200D2B221F8120001F08CB848
S31508007430DFF85C0CDFF88C1B0978405C00284AD022
S315080074400020DFF84C1CDFF87C2B12788854642067
S3150800745010490870DFF8481DDFF8680B02784020ED
S315080074604243885C00281BD10948DFF8581B097875
S31508007470405C012814D10120DFF8281D0870E1A01E
S3150800748003F06AFBDFF8140C03F066FB14E000BF98
S31508007490C86B0020936C0020F4610108A66C0020DC
S315080074A0012201217B4805F052F9D6A003F054FBCE
S315080074B0DFF8EC0B03F050FB04F0E3F90320DFF8E8
S315080074C070182200D2B288540020DFF8681822000B
S315080074D0D2B221F8120001F037B8DFF8B40BDFF8A2
S315080074E0E41A0978405C002848D00020DFF8A01B81
S315080074F0DFF8D02A127888546420DFF8C41D087093
S31508007500DFF89C1CDFF8BC0A027840204243885CFE
S3150800751000281BD1DFF8AC0DDFF8A81A0978405C03
S31508007520012813D10020DFF87C1C0870DFF8980DBD
S3150800753003F012FB13E000BF04620108BB6C0020D5
S3150800754004660108A8690020586B00200122012161
S31508007550504805F0FCF8DFF8740D03F0FDFA04F066
S3150800756090F90320DFF8C8172200D2B28854002009
S31508007570DFF8C0172200D2B221F8120000F0E4BFEB
S31508007580DFF84C0D03F0E8FAFCF725F90020DFF8E0
S31508007590B0170860C920DFF898172200D2B28854BD
S315080075A00020DFF890172200D2B221F8120000F06E
S315080075B0CBBFDFF8DC0ADFF80C1A0978405C002834
S315080075C000F095800020DFF8C81ADFF8F82912784D
S315080075D088546420DFF8E81C0870DFF8E80CDFF848
S315080075E0E4190978405C1C28C0F2BF8085A003F026
S315080075F0B3FADFF8E00C03F0AFFA0020DFF8D81C86
S315080076000870DFF8D40C0078DFF8B81CDFF8B42966
S315080076101278895C884251D2DFF8841BDFF8A40906
S3150800762002784020424301EB0200DFF8AC1C0978DF
S31508007630415CDFF8A80C03F08FFA12A003F08CFA6D
S31508007640DFF8940C0078401CDFF88C1C0870D8E72B
S31508007650926C0020756C0020746C00202E6C002043
S31508007660766C00205857010874570108776C00207B
S31508007670CC6A0020905A01087E010020AA6C0020DE
S31508007680AC6C002020000000146201082462010886
S315080076903462010800100140845E0108985E010802
S315080076A0AC5E01084462010890570108C05E0108F3
S315080076B0A85A0108546201089052010851A003F023
S315080076C04BFA0020DFF8781608600020DFF87416F9
S315080076D00870CA20DFF858162200D2B28854002053
S315080076E0DFF850162200D2B221F812003DE0DFF88A
S315080076F050060068B0F57A7F37D30020DFF84016C9
S315080077000860DFF840060078401CDFF83816087075
S31508007710DFF83006007803281ADB0020DFF86C193A
S3150800772008700020DFF8181608600020DFF8141625
S315080077300870FB20DFF8F8152200D2B28854002022
S31508007740DFF8F0152200D2B221F8120000F0FCBED4
S31508007750C820DFF8DC152200D2B288540020DFF8F2
S31508007760D4152200D2B221F8120000F0EDBE002096
S31508007770DFF8C41508700F2300220F210020FCF73C
S3150800778057F80020DFF8B8150860CB20DFF8A015F9
S315080077902200D2B288540020DFF898152200D2B20F
S315080077A021F8120000F0D0BEDFF8E408DFF814185C
S315080077B00978405C002800F082800020DFF8D018A5
S315080077C0DFF80028127888546420DFF8F41A087065
S315080077D0DFF8CC19DFF8EC07027840204243885CD2
S315080077E0002829D1DFF8DC0ADFF8D8170978405CC9
S315080077F0012821D10120DFF8AC190870DFF8740CD4
S3150800780002E000BF0D0A000003F0A6F90020DFF829
S31508007810301508600020DFF82C150870CC20DFF83A
S3150800782010152200D2B288540020DFF8081522006D
S31508007830D2B221F8120080E001220121DFF80C0DF6
S3150800784004F085FFDFF8080D03F086F90020DFF85D
S31508007850F0140860DFF8EC040078401CDFF8E41444
S315080078600870DFF8E004007803281ADB0020DFF848
S315080078701C1808700020DFF8C81408600020DFF81C
S31508007880C4140870FB20DFF8A8142200D2B288546A
S315080078900020DFF8A0142200D2B221F8120000F06E
S315080078A053BECA20DFF888142200D2B288540020BA
S315080078B0DFF880142200D2B221F812003DE0DFF88A
S315080078C080040068B0F57A7F37D30020DFF870149B
S315080078D00860DFF870040078401CDFF86814087048
S315080078E0DFF86004007803281ADB0020DFF89C170D
S315080078F008700020DFF8481408600020DFF84414F8
S315080079000870FB20DFF828142200D2B28854002021
S31508007910DFF820142200D2B221F8120000F014BEBB
S31508007920CA20DFF80C142200D2B288540020DFF8EF
S3150800793004142200D2B221F8120000F005BE00207D
S31508007940DFF8F41308700023002200210020FBF75B
S315080079506FFF0020DFF8E8130860CD20DFF8D013AA
S315080079602200D2B288540020DFF8C8132200D2B20F
S3150800797021F8120000F0E8BDDFF81407DFF8441616
S315080079800978405C002800F099800020DFF800178D
S31508007990DFF83026127888546420DFF82419087036
S315080079A0DFF8FC17DFF81C06027840204243885CA3
S315080079B0002823D1DFF80C09DFF808160978405C9F
S315080079C001281BD10020DFF8DC170870DFF8840BCC
S315080079D003F0C2F80020DFF86C1308700020DFF807
S315080079E060130860D220D2492200D2B288540020FF
S315080079F0D0492200D2B221F8120092E001220121D8
S31508007A00DFF8480B04F0A3FEDFF84C0B03F0A4F8EC
S31508007A100020CB490860CB480078401CC94908704B
S31508007A20C8480078032816DB0020DFF860160870BF
S31508007A300020C34908600020C2490870FB20BC49E1
S31508007A402200D2B288540020BA492200D2B221F8C4
S31508007A50120000F079BDCC20B5492200D2B2885474
S31508007A600020B4492200D2B221F8120059E000BF22
S31508007A70646201087462010880010020386A0020E7
S31508007A800000A04164660108506C002000004842CE
S31508007A906C660108526C00200000C8427466010832
S31508007AA0546C00200000FA437C660108566C0020DE
S31508007AB000007A4484660108586C0020A0480068D3
S31508007AC0B0F57A7F2DD300209D4908609D4800783F
S31508007AD0401C9C4908709B480078032816DB002048
S31508007AE0DFF8A81508700020954908600020954918
S31508007AF00870FB208E492200D2B2885400208D4996
S31508007B002200D2B221F8120000F01EBDCC2088490E
S31508007B102200D2B28854002086492200D2B221F827
S31508007B20120000F011BD40275FF00008DFF82C9A1C
S31508007B3042463900484604F049FE0020DFF8201A7C
S31508007B400870DFF8200A0068401CDFF8181A086079
S31508007B50DFF8100A016889B2002004F02BFB002028
S31508007B6077490860D32072492200D2B2885400208F
S31508007B7070492200D2B221F8120000F0E5BCDFF805
S31508007B80E0090078002811D000206D49086000201F
S31508007B906C490870D52066492200D2B28854002064
S31508007BA064492200D2B221F812002FE06448006826
S31508007BB0B0F57A7F2AD363480078401C614908707B
S31508007BC060480078032816DB0020DFF8C014087028
S31508007BD000205B49086000205A490870FB20544978
S31508007BE02200D2B28854002052492200D2B221F88B
S31508007BF0120000F0A9BCD4204D492200D2B2885404
S31508007C0000204C492200D2B221F8120000F09CBC98
S31508007C1040275FF00008DFF8449942463900484695
S31508007C2004F0D4FD0020DFF838190870DFF83409AD
S31508007C30016889B2002004F0BDFA002040490860B6
S31508007C40D3203B492200D2B2885400203949220069
S31508007C50D2B221F8120000F077BCDFF808090068F4
S31508007C60401EFF21B0FBF1F201FB1200002815D1DE
S31508007C70DFF8F40802F070FF0020314908600020A0
S31508007C8030490870DC202A492200D2B288540020E4
S31508007C9028492200D2B221F8120014E0DFF8CC08F5
S31508007CA002F05AFF0020264908600020254908707E
S31508007CB0E6201F492200D2B2885400201D4922001E
S31508007CC0D2B221F8120000F03FBCDFF8980800682D
S31508007CD0FE30DFF89C180968884204D20021FF208C
S31508007CE0FBF75EFE5DE0DFF87C080068FE30DFF833
S31508007CF080180968884227D10121FF20FBF750FE2A
S31508007D004FE000BF8C660108D45E01088E6C002027
S31508007D1084620108E85E0108C05A0108B0520108E9
S31508007D2094620108D05201088D6C0020886C0020EE
S31508007D30C06B0020786B00208B6C00209F6C0020A5
S31508007D40B46B00209E6C0020DFF824080068DFF87A
S31508007D5014180968884218D20020CC4908700020F7
S31508007D60DFF8101808600020DFF80C180870FB20F0
S31508007D70DFF808182200D2B288540020DFF800186D
S31508007D802200D2B221F81200DEE30121DFF8E00773
S31508007D900068DFF8D0271268801AFF38C0B2FBF7F0
S31508007DA0FFFD0020DFF8CC170860DD20DFF8CC17D0
S31508007DB02200D2B288540020DFF8C4172200D2B2BB
S31508007DC021F81200C0E3B2487E490978405C0028D1
S31508007DD000F085800020AE497A4A127888546420DB
S31508007DE0DFF8DC140870DFF8B8137648027840200C
S31508007DF04243885C002820D1DFF8C8047149097815
S31508007E00405C012819D10020DFF898130870DFF8C4
S31508007E10740702F0A1FE0020DFF858170860DE207C
S31508007E20DFF858172200D2B288540020DFF850171E
S31508007E302200D2B221F812008DE0DFF864136148FF
S31508007E40027840204243885CFF2840F08480DFF8AF
S31508007E5074045C490978405C01287CD1012201211F
S31508007E60DFF8E80604F073FCDFF81C0702F074FE7E
S31508007E700020DFF800170860DFF8FC060078401CD1
S31508007E80DFF8F4160870DFF8F0060078032818DB28
S31508007E9000207E4908700020DFF8D8160860002008
S31508007EA0DFF8D4160870FB20DFF8D0162200D2B20D
S31508007EB088540020DFF8C8162200D2B221F8120032
S31508007EC042E3DC20DFF8B4162200D2B28854002040
S31508007ED0DFF8AC162200D2B221F812003BE0DFF838
S31508007EE094060068B0F57A7F35D30020DFF884164B
S31508007EF00860DFF884060078401CDFF87C160870F6
S31508007F00DFF874060078032818DB00205F4908703C
S31508007F100020DFF8601608600020DFF85C1608709D
S31508007F20FB20DFF858162200D2B288540020DFF86A
S31508007F3050162200D2B221F8120005E3DC20DFF841
S31508007F403C162200D2B288540020DFF834162200EC
S31508007F50D2B221F81200F7E24D481A490978405C76
S31508007F60002849D0DFF85C0316490978405C0428E4
S31508007F707BDB8B491348027840204243885C1E28E5
S31508007F8073D187490F4802784020424301EB02002B
S31508007F904078002869D182490A480278402042433D
S31508007FA001EB0200807830285FD17D4905480278C8
S31508007FB04020424301EB0200C0784E2855D1DFF835
S31508007FC0CC0501E0A86C002002F0C6FD0020DFF811
S31508007FD0A41508600020DFF8A0150870DF20DFF878
S31508007FE09C152200D2B288540020DFF8941522008E
S31508007FF0D2B221F8120038E0DFF87805006841F2BD
S315080080008831884231D3DFF870050078401CDFF8E4
S3150800801068150870DFF860050078032818DB00206B
S315080080201A4908700020DFF84C1508600020DFF8B0
S3150800803048150870FB20DFF844152200D2B2885490
S315080080400020DFF83C152200D2B221F812007BE2AC
S31508008050DC20DFF828152200D2B288540020DFF889
S3150800806020152200D2B221F812000A20DFF80415E2
S315080080700968DFF800251268B2FBF0F200FB12105F
S31508008080002801D1FBF7BEFB5EE200BFB76C0020FB
S31508008090CC6B0020866C0020856C0020FC5E0108F5
S315080080A0105F0108DFF8CC0400680A2814D3002002
S315080080B0DFF8C01408600020DFF8BC140870E6205A
S315080080C0DFF8B8142200D2B288540020DFF8B014C2
S315080080D02200D2B221F8120036E2DFF888040068DE
S315080080E0401EFF231F22DFF87414B0FBF3F703FBCF
S315080080F01700C0B2FBF792FC0020DFF8781408607E
S31508008100E720DFF878142200D2B288540020DFF87E
S3150800811070142200D2B221F8120015E2DFF87004BA
S31508008120DFF870140978405C002873D00020DFF867
S315080081306014DFF860241278885464206049087057
S315080081401749DFF85004027840204243885C00282B
S3150800815023D15C48DFF83C140978405C01281CD11F
S31508008160002010490870DFF8300402F0F5FC002002
S31508008170DFF8001408600020DFF8FC130870E82018
S31508008180DFF8F8132200D2B288540020DFF8F01383
S315080081902200D2B221F8120075E0DFF8000403E0ED
S315080081A078630020906C002002F0D6FCDFF8C80344
S315080081B00078401CDFF8C0130870DFF8BC030078AD
S315080081C0032819DB0020DFF8D81308700020DFF831
S315080081D0A41308600020DFF8A0130870FB20DFF85E
S315080081E09C132200D2B288540020DFF89413220090
S315080081F0D2B221F81200A7E1E620DFF880132200A8
S31508008200D2B288540020DFF878132200D2B221F8BF
S31508008210120038E0DFF85C030068B0F57A7F32D3E5
S31508008220DFF854030078401CDFF84C130870DFF8B9
S3150800823048030078032819DB0020DFF86413087068
S315080082400020DFF8301308600020DFF82C130870D0
S31508008250FB20DFF828132200D2B288540020DFF86A
S3150800826020132200D2B221F812006DE1E620DFF8D1
S315080082700C132200D2B288540020DFF8041322001F
S31508008280D2B221F812005FE1B6480068B849096819
S31508008290884225D1DFF80C0302F05EFC0020B549C0
S315080082A008600020B4490870F020B4492200D2B210
S315080082B088540020B2492200D2B221F8120023E0E5
S315080082C0936C0020C86B0020D85A0108AC570108E7
S315080082D0F052010810530108BB6C0020046601081F
S315080082E0B14802F039FC0020A24908600020A249E2
S315080082F00870D220A1492200D2B288540020A04991
S315080083002200D2B221F812001EE10020A749087007
S315080083100021002003F062FF002096490860F12042
S3150800832096492200D2B28854002095492200D2B23A
S3150800833021F8120008E19D480078002811D0002095
S315080083408C49086000208C490870FA208B49220065
S31508008350D2B2885400208A492200D2B221F81200EB
S3150800836030E084480068B0F57A7F2BD30020814935
S31508008370086081480078401C7F4908707E4800786C
S31508008380032814DB00208649087000207949086014
S31508008390002079490870FA2078492200D2B2885418
S315080083A0002077492200D2B221F81200CCE0F02052
S315080083B072492200D2B28854002071492200D2B2F2
S315080083C021F81200C0E0724872490978405C00281A
S315080083D017D0774802F0C0FB0120714908700020C9
S315080083E064490860002064490870FB20634922003C
S315080083F0D2B28854002062492200D2B221F8120073
S315080084001BE05C4800686B49884216D36A4802F04C
S31508008410A3FB002062490870002056490860002026
S3150800842055490870FB2055492200D2B288540020CD
S3150800843053492200D2B221F812000A204D49096890
S315080084404C4A1268B2FBF0F200FB1210002801D168
S31508008450FBF7D8F978E000205849087050480078AA
S31508008460002809D0564802F077FB0121002003F0C6
S31508008470B5FE08E0C8570108524802F06DFB022114
S31508008480002003F0ABFE00203A490860FC203B4977
S315080084902200D2B28854002039492200D2B221F8EB
S315080084A0120051E041480078002811D000203149D7
S315080084B00860002030490870FF2030492200D2B2F7
S315080084C0885400202E492200D2B221F812002DE04D
S315080084D028480068B0F57A7F28D300202549086027
S315080084E025480078401C244908702348007803284A
S315080084F011DB00201F49086000201F490870FF2073
S315080085001E492200D2B2885400201D492200D2B248
S3150800851021F8120018E0FB2018492200D2B288542C
S31508008520002017492200D2B221F812000CE01148A7
S31508008530006841F27071884206D300200D49086030
S3150800854004F0FCFA04F012FBBDE8F18F00100140BC
S3150800855030530108E457010850530108B068002059
S31508008560A26C0020B86B0020C0450108204E010807
S31508008570BC6B0020B46B00209E6C0020C06B0020F2
S31508008580786B0020784F0108C44801089C4F010801
S31508008590CC6B0020A86C002070530108FC4501082C
S315080085A0B76C00208C430108804C0108A06C0020A1
S315080085B0AC4C010878E0010038460108A16C00209F
S315080085C0D84C0108A04B0108F8B50400DFF85C0D8B
S315080085D02100C9B2405C002833D0012848D00228BF
S315080085E000F0AA80032800F0AE81042800F0688312
S315080085F0052800F09783062800F050850B2800F020
S31508008600AD850C2801F030830D2801F0BD830E28B6
S3150800861001F045840F2801F0EF84102801F06885E1
S31508008620112801F02C86122801F0C086132801F0C3
S31508008630BD86142801F05C85152801F07D8702F0B7
S315080086400EB8FBF74EFA0120DFF8E01C2200D2B282
S3150800865088540020DFF8541D2200D2B221F81200F7
S315080086600020DFF8BC1D2200D2B2885401F0F7BF03
S31508008670DFF8B00DDFF8B01D0978405C002857D048
S315080086800020DFF8A81D08700020DFF8981DDFF825
S31508008690982D12788854DFF8981DDFF88C0D02782B
S315080086A040204243885C00283CD1DFF8880DDFF87B
S315080086B0781D0978405C012834D1DFF87C0D0078F4
S315080086C0002812D1D5A002F047FADFF8700D02F0A3
S315080086D043FADFF86C0D0078400706D4DFF8600D22
S315080086E00078001DDFF8581D0870FBF7B9FA00205E
S315080086F0DFF8501D08700020DFF84C1D08700220B6
S31508008700DFF8281C2200D2B288540020DFF89C1C0F
S315080087102200D2B221F812000020DFF8041D220040
S31508008720D2B288546420DFF8101D087001F097BF94
S31508008730FBF7D7F901F093BFDFF8E80CDFF8E81C80
S315080087400978405C002800F0E1800020DFF8D41C9E
S31508008750DFF8D42C127888546420DFF8DC1C087003
S31508008760DFF8D00CDFF8C01C0978405C02286BDB08
S31508008770AAA002F0F1F9DFF8D40C02F0EDF9002016
S31508008780DFF8CC1C0870DFF8C80C0078DFF8A41CEA
S31508008790DFF8942C1278895C88421BD2DFF8901C8B
S315080087A0DFF8840C02784020424301EB0200DFF830
S315080087B0A01C0978415CDFF89C0C02F0CDF9DCA01E
S315080087C002F0CAF9DFF8880C0078401CDFF8801C34
S315080087D00870D8E791A002F0BFF9DFF8541CDFF85B
S315080087E0480C027840204243885C002840F08E807E
S315080087F0DFF83C1CDFF8300C02784020424301EBDE
S3150800880002004078002840F081800320DFF81C1B16
S315080088102200D2B288540020DFF8901B2200D2B280
S3150800882021F812000020DFF8F81B2200D2B2885483
S31508008830FBF776F90020DFF80C1C08700020DFF83B
S31508008840081C087001F00BBFDFF8D40B2100C9B271
S31508008850405C062843DADFF8000C02F07DF90020B8
S31508008860DFF8EC1B0870DFF8E80B0078DFF8C41BAC
S31508008870DFF8B42B1278895C884218D2DFF8B01B6F
S31508008880DFF8A40B02784020424301EB0200DFF830
S31508008890C01B0978415CDFF8C00D02F05DF9DFF80E
S315080088A0B00B0078401CDFF8A81B0870DBE75BA05C
S315080088B002F052F90020DFF8F41A2200D2B221F8A9
S315080088C01200DFF85C0B2100C9B2405C401CDFF8DF
S315080088D0501B2200D2B28854FBF7C2F916E0FBF708
S315080088E000F90120DFF8441A2200D2B28854002089
S315080088F0DFF8B81A2200D2B221F812000020DFF8F9
S31508008900201B2200D2B2885401F0A9BEDFF8340B2E
S315080089100078401CDFF82C1B0870DFF8280B00785D
S3150800892005280ADB0020DFF81C1B08706420DFF826
S31508008930081B0870FBF794F903E06420DFF8F81ABF
S31508008940087001F08CBEDFF8DC0ADFF8DC1A09785B
S31508008950405C002800F086810020DFF8C81ADFF89E
S31508008960C82A127888546420DFF8CC1A0870DFF811
S31508008970C40ADFF8B41A0978405C0228C0F22181DB
S3150800898026A002F0E9F8DFF8D40C02F0E5F800209A
S31508008990DFF8BC1A0870DFF8B80A0078DFF8941A0E
S315080089A0DFF8842A1278895C88421BD2DFF8801A9D
S315080089B0DFF8740A02784020424301EB0200DFF830
S315080089C0901A0978415CDFF88C0A02F0C5F858A0BD
S315080089D002F0C2F8DFF8780A0078401CDFF8701A4F
S315080089E00870D8E70DA002F0B7F8DFF8441ADFF8E8
S315080089F0380A027840204243885C012840F05E81AC
S31508008A00DFF82C1ADFF8200A02784020424301EBEF
S31508008A1002004078DFF8241D02E000BF0D0A0000BE
S31508008A200870DFF80C1ADFF8000A02784020424383
S31508008A3001EB02008078DFF8081D0870DFF8F019EE
S31508008A40DFF8E40902784020424301EB0200C078CF
S31508008A50DFF8F01C0870DFF8D819DFF8CC090278BF
S31508008A604020424301EB02000079DFF8DC1C087065
S31508008A70DFF8BC19DFF8B00902784020424301EB61
S31508008A8002004079DFF8C41C0870DFF8A419DFF883
S31508008A90980902784020424301EB02008079DFF80A
S31508008AA0B01C0870DFF88819DFF87C0902784020C6
S31508008AB0424301EB0200C079DFF8981C0870DFF822
S31508008AC0800C007810F00F0007280AD1DFF8740C24
S31508008AD00078642805D104F031F8022104F04DF835
S31508008AE03DE0DFF85C0C007810F00F0007280AD18B
S31508008AF0DFF8500C0078022805D104F01FF803218E
S31508008B0004F03BF82BE0DFF8380C007810F00F0083
S31508008B1004280AD1DFF82C0C0078582805D104F06F
S31508008B200DF8042104F029F819E0DFF8140C01E027
S31508008B3020000000007810F00F0007280AD1DFF89F
S31508008B40040C0078842805D103F0F8FF052104F009
S31508008B5014F804E003F0F2FF002104F00EF803F025
S31508008B60EDFF04F008F80100C9B2DFF8EC0B01F0DC
S31508008B70F3FFDFF8E00B0078000703D50120DFF8E4
S31508008B80DC1B08700420DFF8A4172200D2B2885430
S31508008B900020DFF818182200D2B221F812000020AF
S31508008BA0DFF87C182200D2B28854FBF707F80020B9
S31508008BB0DFF8901808700020DFF88C18087001F0AC
S31508008BC04EBDDFF85C082100C9B2405C062875DA9C
S31508008BD07CA001F0C1FFDFF8880B01F0BDFF002083
S31508008BE0DFF86C180870DFF868080078DFF84418B2
S31508008BF0DFF834281278895C88421BD2DFF83018EF
S31508008C00DFF8240802784020424301EB0200DFF82F
S31508008C1040180978415CDFF83C0801F09DFF6AA01E
S31508008C2001F09AFFDFF828080078401CDFF82018C2
S31508008C300870D8E763A001F08FFF0020DFF86C17F3
S31508008C402200D2B221F81200DFF8D4072100C9B2F7
S31508008C50405C401CDFF8C8172200D2B28854FAF7E5
S31508008C60FFFF2BE0DFF8DC070078401CDFF8D4179D
S31508008C700870DFF8D0070078052816DB0020DFF833
S31508008C80C4170870DFF8C0070078032816DADFF87B
S31508008C90B8070078401CDFF8B01708706420DFF8C2
S31508008CA098170870FAF73CFF08E0DFF89C07007889
S31508008CB0032803DA6420DFF88017087001F0CFBCB8
S31508008CC0DFF86007DFF860170978405C002827D0CE
S31508008CD00020DFF85017DFF85027127888546420F0
S31508008CE0DFF8541708700520DFF840162200D2B2C4
S31508008CF088540020DFF8B4162200D2B221F81200F8
S31508008D000020DFF81C172200D2B28854FAF7C8FFF1
S31508008D100020DFF8301708700020DFF82C170870DD
S31508008D2001F09DBCDFF8FC06DFF8FC160978405C0C
S31508008D30002800F07D810020DFF8E816DFF8E82635
S31508008D40127888546420DFF8F0160870DFF8E40615
S31508008D50DFF8D4160978405C0228C0F2188119A0F9
S31508008D6001F0FAFEDFF8FC0901F0F6FE0020DFF854
S31508008D70E0160870DFF8D8060078DFF8B816DFF8CE
S31508008D80A8261278895C884220D2DFF8A416DFF874
S31508008D90980602784020424301EB0200DFF8B0163D
S31508008DA00978415CDFF8AC0601F0D6FE06A001F0B2
S31508008DB0D3FEDFF89C060078401CDFF8941608708E
S31508008DC0D8E700BF0D0A000020000000B2A001F09D
S31508008DD0C3FEDFF85C16DFF85006027840204243EF
S31508008DE0885C092840F056810C25DFF84416DFF820
S31508008DF0380602784020424301EB0200061DDFF8E0
S31508008E006819DFF8240602780F20424301EB0207AF
S31508008E102A003100380003F0D9FDDFF81416DFF810
S31508008E20080602784020424301EB0200007FDFF883
S31508008E303C198871DFF8F815DFF8EC050278402050
S31508008E40424301EB0200407FDFF82019C871DFF8C2
S31508008E50E015DFF8D40502784020424301EB020012
S31508008E60807FDFF80C190870DFF8C415DFF8B8053D
S31508008E7002784020424301EB0200C07FDFF8F01879
S31508008E804870DFF8AC15DFF8A005027840204243A9
S31508008E9001EB020090F82000DFF8D4188870DFF89C
S31508008EA09015DFF8840502784020424301EB020062
S31508008EB090F82100DFF8B818C87002F0DDFFDFF877
S31508008EC07015DFF8640502784020424301EB020082
S31508008ED040784E2820D1DFF85815DFF84C0502787F
S31508008EE04020424301EB02008078592814D1DFF86C
S31508008EF04015DFF8340502784020424301EB0200B2
S31508008F00C078582808D1DFF86C0801F025FE03F070
S31508008F1015FE012103F031FE0020DFF82815087040
S31508008F200020DFF82415087003F008FE03F023FE7E
S31508008F30052815D10620DFF8F4132200D2B288548A
S31508008F400020DFF868142200D2B221F812000020AF
S31508008F50DFF8CC142200D2B28854FAF79EFF14E048
S31508008F600B20DFF8C8132200D2B288540020DFF89D
S31508008F703C142200D2B221F812000020DFF8A01417
S31508008F802200D2B28854FAF76BFE01F068BBDFF80C
S31508008F9090042100C9B2405C06287BDA3EA001F0A5
S31508008FA0DBFDDFF8280D01F0D7FD0020DFF8A0145F
S31508008FB00870DFF89C040078DFF87814DFF8682476
S31508008FC01278895C88421BD2DFF86414DFF85804EB
S31508008FD002784020424301EB0200DFF87414097856
S31508008FE0415CDFF8700401F0B7FD8CA001F0B4FD18
S31508008FF0DFF85C040078401CDFF854140870D8E7E2
S3150800900025A001F0A9FD0020DFF8A0132200D2B2A6
S3150800901021F81200DFF808042100C9B2405C401CA0
S31508009020DFF8FC132200D2B28854FAF719FE31E0B1
S3150800903003F084FD03F09FFD04282BD1DFF8040418
S315080090400078401CDFF8FC130870DFF8F803007896
S31508009050052816DB0020DFF8EC130870DFF8E803B4
S315080090600078032816DADFF8E0030078401CDFF8FA
S31508009070D81308706420DFF8C0130870FAF710FEDA
S3150800908008E0DFF8C4030078032803DA6420DFF871
S31508009090A813087001F0E3BA0D0A0000DFF884038C
S315080090A0DFF884130978405C002855D0BEA001F08B
S315080090B053FDDFF8300D01F04FFD0020DFF8901367
S315080090C00870DFF88C030078DFF86813DFF8582398
S315080090D01278895C88421BD2DFF85413DFF84803FC
S315080090E002784020424301EB0200DFF86413097856
S315080090F0415CDFF8600301F02FFD48A001F02CFD6C
S31508009100DFF84C030078401CDFF844130870D8E7F2
S31508009110A5A001F021FD0020C249C34A127888544F
S315080091206420DFF8141308700B2080492200D2B29D
S31508009130885400209D492200D2B221F8120000204E
S31508009140B7492200D2B28854FAF78AFD0020BD49F1
S3150800915008700020BC49087001F081BAB148B249CC
S315080091600978405C002800F07B820020AD49AE4AB1
S31508009170127888546420B04908700020B1490870F4
S315080091800020B14908700120DFF85C1C0870A94866
S31508009190A5490978405C0228C0F2628282A001F0E3
S315080091A0DBFCAA4801F0D8FC0020A9490870A848A9
S315080091B00078A0499C4A1278895C884215D29C4955
S315080091C0994802784020424301EB0200A0490978F9
S315080091D0415CA04801F0C0FC10A001F0BDFC9C4811
S315080091E00078401C9A490870E1E76FA001F0B4FCCA
S315080091F0DFF8540D01788E4A8B48037840204343A4
S31508009200D05C81421AD1DFF8400D00780A2807D0D1
S31508009210DFF8380D01F0A0FC22E200BF20000000B4
S31508009220DFF82C0D0178824A7F48037840204343B3
S3150800923002EB03004078814200F012827C497A48AA
S31508009240027840204243885C002849D0012854D03F
S31508009250022857D0032862D0042869D0052872D07E
S31508009260062800F08880072800F08F80082800F07C
S315080092709380092800F09C800A2800F09E800B281D
S3150800928000F0EC800D2800F0F0800E2800F0FC803D
S315080092900F2800F00881102800F01481112800F02A
S315080092A02081122800F02C81132800F03881142818
S315080092B000F04481152800F050811B2800F05C81DD
S315080092C01C2800F068811D2800F074811E2800F013
S315080092D080811F2800F08C81FF2800F09881A5E185
S315080092E0DFF8D40C01F038FC51494F480278402089
S315080092F04243885C02F04CFEA2E1DFF8C00C01F0A4
S315080093002BFC9DE1DFF8B80C01F026FC48494648DD
S31508009310027840204243885C02F03AFE90E1DFF88A
S31508009320A40C01F019FC02F04DFE89E1C06B002087
S31508009330DFF8940C01F010FC02F054FE0120DFF86F
S315080093408C1C08707CE1DFF8880C01F005FC3849B4
S31508009350354802784020424301EB020082783449BE
S31508009360314803784020434301EB0300417801204C
S3150800937002F0DEFD64E1DFF85C0C01F0EDFB002293
S315080093800021002002F0D4FD5AE1DFF84C0C01F070
S31508009390E3FB02F03BFE53E1DFF8400C01F0DCFB97
S315080093A002F044FE4CE100BF0D0A0000786B002075
S315080093B0DFF82C0C01F0D0FB42E11D491A4802786F
S315080093C04020424301EB02004178DFF8700D01F0BE
S315080093D0C3FB1749144802784020424301EB0200B8
S315080093E04078DFF86C1B087011490F480278402056
S315080093F0424301EB0200417811F00F010C4A0A487A
S3150800940003784020434302EB03004078C0B20009CA
S3150800941002F01CFE0120DFF8B41B087010E100BF43
S31508009420C46B0020CC6B0020A86C0020A76C002021
S3150800943078630020C86B0020946C0020245F010824
S31508009440A66C0020BC6C0020BD6C0020385F0108AB
S31508009450BB6C00200466010890530108DFF8E00C95
S3150800946001F07AFB02F00CFEEAE0DFF8200D01F0CD
S3150800947073FBDFF81C1DDFF81C0D02784020424301
S31508009480885C02F085FDDBE0DFF80C0D01F064FB7B
S31508009490DFF8FC1CDFF8FC0C027840204243885CAD
S315080094A002F076FDCCE0DFF8F40C01F055FBDFF8AE
S315080094B0E01CDFF8E00C027840204243885C02F0AA
S315080094C067FDBDE0DFF8D80C01F046FBDFF8C01CED
S315080094D0DFF8C00C027840204243885C02F058FD51
S315080094E0AEE0DFF8C00C01F037FBDFF8A41CDFF8AC
S315080094F0A40C027840204243885C02F049FD9FE0B4
S31508009500DFF8A40C01F028FBDFF8841CDFF8840CD4
S31508009510027840204243885C02F03AFD90E0DFF88A
S315080095208C0C01F019FBDFF8681CDFF8680C027870
S3150800953040204243885C02F02BFD81E0DFF8700C86
S3150800954001F00AFBDFF8481CDFF8480C02784020D7
S315080095504243885C02F01CFD72E0DFF8580C01F00B
S31508009560FBFADFF82C1CDFF82C0C0278402042436B
S31508009570885C02F00DFD63E0DFF83C0C01F0ECFAC4
S31508009580DFF80C1CDFF80C0C027840204243885C9C
S3150800959002F0FEFC54E0DFF8240C01F0DDFADFF8F7
S315080095A0F01BDFF8F00B027840204243885C02F09B
S315080095B0EFFC45E0DFF8200D01F0CEFADFF8D01B0E
S315080095C0DFF8D00B027840204243885C02F0E0FCCA
S315080095D036E0DFF8080D01F0BFFADFF8B41BDFF854
S315080095E0B40B027840204243885C02F0D1FC27E0A5
S315080095F0DFF8EC0C01F0B0FADFF8941BDFF8940BF7
S31508009600027840204243885C02F0C2FC18E0DFF88A
S31508009610D40C01F0A1FADFF8781BDFF8780B027892
S3150800962040204243885C02F0B3FC09E0DFF8601B87
S31508009630DFF8600B027840204243885C02F0A8FC01
S31508009640DFF84C1BDFF84C0B027840204243885C5D
S31508009650DFF8F4180870D4E294660108B0530108DC
S3150800966003F06CFA03F087FA04282AD1DFF8780C9D
S315080096700078002825D0DFF870070078002820D069
S315080096800020DFF8641C08700020DFF85C170870FB
S31508009690FAF7A9FD0020DFF8001D08700020DFF8A2
S315080096A0FC1C08701420DFF8F81C2200D2B288547B
S315080096B00020DFF8F01C2200D2B221F8120000F0D8
S315080096C0CEBFDFF8E40C0078002805D003F036FAA0
S315080096D003F051FA04280FD1DFF8CC0C00780028E3
S315080096E04AD0DFF804070078002845D003F026FAA8
S315080096F003F041FA04283FD10020DFF8AC1C0870BB
S315080097000020DFF8E4160870FAF715FC0020DFF8E9
S31508009710881C08700020DFF8841C08700D20DFF80C
S31508009720801C2200D2B288540020DFF8781C220060
S31508009730D2B221F8120000F092BF00BF966C00204A
S31508009740976C0020986C0020996C00209A6C002079
S315080097509B6C00209C6C0020484E01089D6C0020E4
S31508009760C04F010800580108A8690020586B00205E
S31508009770B06B0020704E0108DFF8D80C007800287E
S3150800978005D003F0DBF903F0F6F904280FD1DFF86A
S31508009790C40C007800282BD0DFF84C060078002887
S315080097A026D003F0CBF903F0E6F9042820D10020EF
S315080097B0DFF8A01C08700020DFF82C160870FAF7EE
S315080097C0ECFB0020DFF8D01B08700020DFF8CC1B6C
S315080097D008700C20DFF8C81B2200D2B2885400207B
S315080097E0DFF8C01B2200D2B221F8120000F037BF02
S315080097F0DFF8640C0078002805D003F09FF903F021
S31508009800BAF904280FD1DFF8500C007800284DD09B
S31508009810DFF8D4050078002848D003F08FF903F064
S31508009820AAF9042842D10020DFF82C1C0870002071
S31508009830DFF8B4150870DFF8240C0078002804D087
S31508009840DFF8180C0078022817D1FAF774FB002005
S31508009850DFF8441B08700020DFF8401B08700D2055
S31508009860DFF83C1B2200D2B288540020DFF8341BF4
S315080098702200D2B221F8120016E0FAF785FC002081
S31508009880DFF8141B08700020DFF8101B087013207F
S31508009890DFF80C1B2200D2B288540020DFF8041B24
S315080098A02200D2B221F8120000F0D9BEDFF8DC0C93
S315080098B00078002805D003F041F903F05CF9042884
S315080098C00FD1DFF8C80C007800284FD0DFF818054C
S315080098D0007800284AD003F031F903F04CF904283F
S315080098E044D10020DFF8A41C08700020DFF8F81423
S315080098F0087003F023F903F03EF9052803D1002088
S31508009900DFF844160870DFF8140D0188DFF8100D2B
S315080099100088FAF7A6FBDFF8080D0088DFF8041DB3
S315080099200880DFF8F80C0088DFF8FC1C08800020A7
S31508009930DFF8EC1C08800020DFF8E01C0880002017
S31508009940DFF8541A08700020DFF8501A08700E2045
S31508009950DFF84C1A2200D2B288540020DFF8441AE5
S315080099602200D2B221F8120000F079BEDFF8F00C1E
S315080099700078002805D003F0E1F803F0FCF8042885
S315080099800FD1DFF8DC0C007800282BD0DFF858045C
S315080099900078002826D003F0D1F803F0ECF8042864
S315080099A020D10020DFF8B81C08700020DFF8381432
S315080099B00870FAF7ABFB0020DFF8DC190870002006
S315080099C0DFF8D81908700F20DFF8D4192200D2B2B0
S315080099D088540020DFF8CC192200D2B221F81200F0
S315080099E000F03DBEDFF8E4050078002805D003F056
S315080099F0A5F803F0C0F804280FD1DFF8D0050078E1
S31508009A0000282BD0DFF8E0030078002826D003F0E2
S31508009A1095F803F0B0F8042820D10020DFF8AC153B
S31508009A2008700020DFF8C0130870FAF7DCFB002086
S31508009A30DFF8641908700020DFF860190870102034
S31508009A40DFF85C192200D2B288540020DFF85419D6
S31508009A502200D2B221F8120000F001BEDFF8040C91
S31508009A600078002805D003F069F803F084F8042884
S31508009A700FD1DFF8F00B007800282AD0DFF868034A
S31508009A800078002825D003F059F803F074F8042864
S31508009A901FD10020DFF8CC1B08700020D2490870BF
S31508009AA0FAF7ADFA0020DFF8F01808700020DFF8A2
S31508009AB0EC1808701120DFF8E8182200D2B2885492
S31508009AC00020DFF8E0182200D2B221F8120000F0D8
S31508009AD0C6BDDFF8940B0078002805D003F02EF8F1
S31508009AE003F049F804280ED1DFF87C0B007800282B
S31508009AF029D0BD480078002825D003F01FF803F0C8
S31508009B003AF804281FD10020DFF85C1B08700020F3
S31508009B10B5490870FAF738FB0020DFF87C1808709A
S31508009B200020DFF8781808701220DFF87418220071
S31508009B30D2B288540020DFF86C182200D2B221F87D
S31508009B40120000F08CBDDFF8240B0078002805D041
S31508009B5002F0F4FF03F00FF804280ED1DFF80C0B1F
S31508009B60007800284DD0A0480078002849D002F097
S31508009B70E5FF03F000F8042843D10020DFF8EC1ACB
S31508009B80087000209849087002F0D8FF02F0F3FF29
S31508009B90052803D10020DFF8B0130870DFF8D00AD3
S31508009BA00188DFF8D00A0088FAF752FBDFF8C40A02
S31508009BB00088DFF8C41A0880DFF8B40A0088DFF8DE
S31508009BC0BC1A08800020DFF8AC1A08800020DFF8ED
S31508009BD0A01A08800020DFF8C01708700020DFF8F8
S31508009BE0BC1708701520DFF8B8172200D2B28854BF
S31508009BF00020DFF8B0172200D2B221F8120000F0D8
S31508009C002EBD02F09BFF02F0B6FF042828D1DFF82C
S31508009C1088070078401CDFF880170870DFF8780797
S31508009C200078052812DB0020DFF86C170870DFF8CB
S31508009C306C070078401CDFF864170870DFF85C07CB
S31508009C40007803280EDAFAF70BF80BE0DFF84C0772
S31508009C500078032806DA6420DFF8241A087001E081
S31508009C60F9F7FEFF00F0FBBCDFF8180ADFF8241549
S31508009C700978405C002853D00020DFF8081ADFF87E
S31508009C801425127888546420DFF8F4190870DFF870
S31508009C900015DFF80005027840204243885C00285A
S31508009CA016D1DFF8E409DFF8EC140978405C0128DE
S31508009CB00ED10120DFF8A4170870BEA000F04CFFF3
S31508009CC0DFF8C80900F048FF0FE000BFD0530108CD
S31508009CD001220121DFF8B80902F039FDB5A000F02C
S31508009CE03BFFDFF8B00900F037FF01F0CAFD00209E
S31508009CF03D4908700020DFF8A01608700020DFF83C
S31508009D009C1608700B20DFF898162200D2B28854E9
S31508009D100020DFF890162200D2B221F8120031E0B6
S31508009D2002F00CFF02F027FF04282BD1DFF86806A3
S31508009D300078401CDFF860160870DFF85C060078CB
S31508009D40052816DB0020DFF850160870DFF84C06E9
S31508009D500078032816DADFF844060078401CDFF896
S31508009D603C1608706420DFF818190870FAF715F918
S31508009D7008E0DFF828060078032803DA6420DFF80D
S31508009D800019087000F06BBCDFF8F808DFF8041457
S31508009D900978405C00284FD00020DFF8E818DFF883
S31508009DA0F423127888546420DFF8D4180870DFF892
S31508009DB0E013DFF8E003027840204243885C00287D
S31508009DC014D1DFF8C408DFF8CC130978405C012801
S31508009DD00CD10020DFF884160870DFF8BC0800F004
S31508009DE0BBFE0DE01C580108BE6C002001220121B3
S31508009DF0DFF89C0802F0ABFCDFF8A00800F0ACFE28
S31508009E0001F03FFD0020DFF8201B08700020DFF876
S31508009E10881508700020DFF8841508700B20DFF815
S31508009E2080152200D2B288540020DFF87815220067
S31508009E30D2B221F8120031E002F080FE02F09BFE59
S31508009E4004282BD1DFF850050078401CDFF84815A8
S31508009E500870DFF844050078052816DB0020DFF8CF
S31508009E6038150870DFF834050078032816DADFF8A5
S31508009E702C050078401CDFF8241508706420DFF8EC
S31508009E8000180870FAF757F808E0DFF810050078A8
S31508009E90032803DA6420DFF8E8170870DFE3DFF841
S31508009EA0E407BC490978405C002853D00020DFF855
S31508009EB0D417B84A127888546420DFF8C417087093
S31508009EC0B349B448027840204243885C00280BD145
S31508009ED0DFF8B407AF490978405C012804D1DFF8F8
S31508009EE0500A00F039FE09E001220121DFF8A00737
S31508009EF002F02DFCDFF83C0A00F02EFEDFF85C05C8
S31508009F000078002805D10120DFF85015087001F007
S31508009F10B8FC0020DFF8101A08700020DFF8781463
S31508009F2008700020DFF8741408700B20DFF870142E
S31508009F302200D2B288540020DFF868142200D2B278
S31508009F4021F8120057E000BFAD6C0020E44F01086D
S31508009F50AE6C002002F0F2FD02F00DFE04284AD194
S31508009F60DFF834040078401CDFF82C140870DFF89A
S31508009F7028040078052835DB0020DFF81C14087053
S31508009F80DFF818040078032835DADFF810040078BB
S31508009F90401CDFF8081408706420DFF8E41608701F
S31508009FA0DFF884060188DFF87C060088FAF759F896
S31508009FB021E000BF0D0A0000A4620108F05A01085A
S31508009FC04C5F0108B462010838580108816C00200A
S31508009FD0C4620108D4620108E46201084C650108FC
S31508009FE0F4620108DFF8B4030078032803DA642072
S31508009FF0DFF88C16087032E3DFF8880665490978B9
S3150800A000405C002849D00020DFF87816614A1278AB
S3150800A01088546420DFF8681608705D495D48027840
S3150800A02040204243885C00280BD1DFF85C0659497A
S3150800A0300978405C012804D1DFF8FC0800F08CFDA3
S3150800A04009E001220121DFF8480602F080FBDFF86B
S3150800A050EC0800F081FD0220DFF8001408700120EA
S3150800A060DFF8DC1808700020DFF8BC18087000203C
S3150800A070DFF8241308700020DFF8201308700B207F
S3150800A080DFF81C132200D2B288540020DFF814131C
S3150800A0902200D2B221F8120029E002F04FFD02F0A8
S3150800A0A06AFD042823D1BC480078401CBA490870C8
S3150800A0B0B9480078052812DB0020B7490870B74868
S3150800A0C00078032813DAB5480078401CB3490870AD
S3150800A0D06420DFF8AC150870FAF718F807E0AF48FF
S3150800A0E00078032803DA6420DFF894150870B6E2CE
S3150800A0F0DFF8900527490978405C002800F094802D
S3150800A1000020DFF88015234A127888546420DFF887
S3150800A110701508701E491F48027840204243885C23
S3150800A12000280FD1DFF860051A490978405C012834
S3150800A13008D1DFF8100800F00FFD4BE0F0530108D6
S3150800A1405458010812491348027840204243885C53
S3150800A150072835D10E490F4802784020424301EBC3
S3150800A1600200407807282BD1DFF81C050949097831
S3150800A170405C022824D1DFF8CC0700F0EDFCDFF8BC
S3150800A180C80700F0E9FC01F041FF23E0605F010821
S3150800A19078630020A86C0020745F0108085B01083A
S3150800A1A0885F01089C5F010810540108B05F010828
S3150800A1B0C45F010804630108D85F0108EC5F010861
S3150800A1C001220121DFF8C80402F0C1FADFF87C0792
S3150800A1D000F0C2FCA1480078002804D101209F495C
S3150800A1E0087001F04EFB6E482100C9B2405C142885
S3150800A1F002D101206C4908700020DFF82C1708707E
S3150800A2000020654908700020644908700B206449DD
S3150800A2102200D2B28854002062492200D2B221F824
S3150800A2201200F9F71DFD29E002F088FC02F0A3FCF4
S3150800A230042823D158480078401C574908705648C6
S3150800A2400078052812DB0020534908705348007827
S3150800A250032813DA51480078401C504908706420D6
S3150800A260DFF81C140870F9F7BEFF07E04B480078C2
S3150800A270032803DA6420DFF808140870EFE1DFF832
S3150800A2800404DFF8CC160978405C00285AD0002070
S3150800A290DFF8F013DFF8B826127888546420DFF860
S3150800A2A0E0130870DFF8AC16DFF8A4060278402041
S3150800A2B04243885C002819D1DFF8CC03DFF89016F2
S3150800A2C00978405C012811D1C4A000F045FCDFF8EC
S3150800A2D0880600F041FC16E00060010814600108D9
S3150800A2E028600108205B0108BF6C002001220121BB
S3150800A2F0DFF89C0302F02BFAB8A000F02DFCDFF87B
S3150800A3005C0600F029FC55480078002804D1012095
S3150800A3105249087001F0B5FA0020DFF80C160870EB
S3150800A32000201D49087000201C4908700B201C4994
S3150800A3302200D2B2885400201A492200D2B221F84B
S3150800A340120027E002F0FAFB02F015FC042821D1DE
S3150800A35011480078401C104908700F4800780528F5
S3150800A36011DB00200C4908700C480078032811DA24
S3150800A3700A480078401C094908706420C0490870DA
S3150800A380F9F73DFE06E005480078032802DA64205E
S3150800A390BB49087063E100BFBC6C0020BD6C00209F
S3150800A3A0C06B0020786B0020B86C0020B548DFF839
S3150800A3B0A0150978405C002800F08D800020B1497E
S3150800A3C0DFF88C25127888546420AD490870DFF8C8
S3150800A3D08415DFF87C05027840204243885C002813
S3150800A3E00ED1A948DFF868150978405C012807D11D
S3150800A3F07AA000F0B1FBDFF8680500F0ADFB0BE0D2
S3150800A40001220121A24802F0A2F974A000F0A4FBDF
S3150800A410DFF8500500F0A0FB0020DFF80C150870E7
S3150800A4200020DFF8441508700020DFF84015087092
S3150800A43002F084FB02F09FFB042823D1DFF83005E5
S3150800A4402100C9B2405C13280AD10120DFF824157F
S3150800A450087009E0896C00208C6C0020916C002043
S3150800A4600120DFF8DC1408700B20DFF80415220041
S3150800A470D2B288540020DFF800152200D2B221F8A3
S3150800A480120058E0DFF8E8042100C9B2405C13283E
S3150800A4900FD1F9F7A8FE1420DFF8D4142200D2B29F
S3150800A4A088540020DFF8D0142200D2B221F8120016
S3150800A4B041E00120DFF8881408700B20DFF8B0149B
S3150800A4C02200D2B288540020DFF8AC142200D2B29F
S3150800A4D021F812002FE002F031FB02F04CFB0428B1
S3150800A4E029D1DFF884040078401CDFF87C14087052
S3150800A4F0DFF874040078052815DB0020DFF86814F7
S3150800A5000870DFF868040078032814DADFF85C04BA
S3150800A5100078401CDFF85414087064205849087005
S3150800A520F9F732FE07E0DFF844040078032802DA78
S3150800A53064205349087092E05248DFF814140978E9
S3150800A540405C00284CD000204E49DFF804241278DD
S3150800A550885464204A490870DFF8F813DFF8F003D6
S3150800A560027840204243885C002811D14648DFF82B
S3150800A570E0130978405C01280AD1DFF8000400F0EE
S3150800A580EBFA012001F0F6FD0EE000BF7E6C00201C
S3150800A590012201213E4802F0DAF8DFF8E40300F070
S3150800A5A0DBFA022001F0E6FD0020DFF87C130870D4
S3150800A5B00020DFF8B41308700020DFF8B013087025
S3150800A5C00B20DFF8AC132200D2B288540020DFF843
S3150800A5D0A8132200D2B221F8120040E00D0A0000AA
S3150800A5E0DFF884030078401CDFF87C130870DFF876
S3150800A5F07803007805282ADB0020DFF86C1308703A
S3150800A600DFF868030078032810DBDFF8740300F02E
S3150800A610A3FA022001F0AEFD21E000BF326C002053
S3150800A620306C00205E6C0020606C0020DFF83C0374
S3150800A6300078401CDFF8341308706420104908704D
S3150800A6400E4801880C480088F9F702FE07E0DFF893
S3150800A6501C030078032802DA642009490870F1BD52
S3150800A6607F6C0020836C0020806C0020846C0020A6
S3150800A670366C0020346C0020626C0020646C00206C
S3150800A680946C0020CC6B0020C86B0020385B010856
S3150800A69000100140505B0108705801083054010849
S3150800A6A080B5DFF8E0020078002808D0012818D025
S3150800A6B0022826D0032868D0642872D076E0B248EB
S3150800A6C00088411CB04A118080B2B0F5167F07DBBE
S3150800A6D00120AC4908700020AB490880F8F742FD14
S3150800A6E064E0A9480088411CA74A118080B2B0F5E9
S3150800A6F0967F05DB0220A34908700020A24908803E
S3150800A70054E0A1480088401C9F4908809F4800786B
S3150800A710002809D000209C49088000208C49087030
S3150800A7200020FBF75BFF2FE097480088242802DB10
S3150800A73000209549088094480088002810D00428ED
S3150800A7400ED008280CD00C2811D010280FD01428A9
S3150800A7500DD0182812D01C2810D020280ED013E0AF
S3150800A76001207B4908700120FAF732F90CE0002035
S3150800A770774908700020FBF731FF05E0022074498D
S3150800A78008700220FDF720FF10E07F480088401C73
S3150800A7907D4908807C480088C82801DBF9F7B2FDA6
S3150800A7A004E0012201217A4801F0D1FF79480078B6
S3150800A7B0002838D075480078002834D175480078C4
S3150800A7C0401E744908707348007800282BD1002071
S3150800A7D06749487000206849488054A000F0BCF9D1
S3150800A7E06D4800F0B9F96D48007807281BD16C4808
S3150800A7F0007800280BD1012069490870F8F7BFFCDA
S3150800A80003206049087000205F4908800BE0012298
S3150800A81001215F4801F09BFF01F03FF9F8F7AFFC13
S3150800A8206420584908705F480078002835D0574892
S3150800A8300078002831D15B480078401E59490870D5
S3150800A84058480078002828D1002049490870002077
S3150800A85049490880544800F07FF95048007807288D
S3150800A8601BD14F48007800280BD101204C490870AD
S3150800A870F8F785FC03204349087000204249088000
S3150800A8800BE001220121424801F061FF01F005F9C0
S3150800A890F8F775FC64203B4908704448007800289E
S3150800A8A02DD03A480078002829D140480078401E23
S3150800A8B03E4908703D480078002820D100202C49E0
S3150800A8C0887000202C498880394800F045F93348BB
S3150800A8D00078072813D137480078002803D10120CB
S3150800A8E0344908700BE001220121294801F02FFFA5
S3150800A8F001F0D3F8F8F743FC64202249087023488E
S3150800A9000078002804D02C480068401C2A490860B2
S3150800A9102A480068002804D028480068401E2749AD
S3150800A9200860F9F713FF01BDBE6C00200D0A000090
S3150800A9308C58010850540108705401080850010841
S3150800A940816C00202C500108E4620108984E010829
S3150800A950A86C002078630020685B0108805B01080A
S3150800A960A858010890540108BC6C0020BD6C002052
S3150800A970C06B0020BF6C0020786B0020C45801080B
S3150800A980B0540108A36C00205A6C00209F6C00206C
S3150800A99000100140926C00203C600108A66C002063
S3150800A9A0A56C0020936C002050600108946C002070
S3150800A9B0985B0108A76C0020B46B0020D46B0020BC
S3150800A9C001B501226946DFF8940702F034F901BDA2
S3150800A9D080B500208DF80000DFF8800702F01AF92C
S3150800A9E000280FD101226946DFF8700702F048F9FE
S3150800A9F0002807D09DF8000002F03BFB00208DF8E8
S3150800AA000000EFE701BD70B504000D000026DFF871
S3150800AA10500702F0CBF8290089B2884214D35FF0B8
S3150800AA20FF31DFF84007006802F09EFF2A0092B265
S3150800AA302100DFF82C0702F0FEF8DFF82807006887
S3150800AA4002F0D1FF012024E03000461C80B26428C1
S3150800AA501EDA012002F053FF761CDFF8040702F025
S3150800AA60A5F8290089B28842EED35FF0FF31DFF8F6
S3150800AA70F406006802F078FF2A0092B22100DFF897
S3150800AA80E00602F0D8F8DFF8DC06006802F0ABFF53
S3150800AA90002070BDF8B5ADF5007D0024DFF8C006CE
S3150800AAA002F0B8F8002826D14FF4007500266F4644
S3150800AAB032002900380001F089FE5FF0FF31DFF827
S3150800AAC0A406006802F050FF4FF400726946DFF8EA
S3150800AAD0900602F0D5F80400DFF88806006802F050
S3150800AAE082FF4FF47A73220092B26946DFF878063D
S3150800AAF003F000F8D2E70DF5017DF0BD38B5040086
S3150800AB000D004FF47A732A0092B22100DFF8580636
S3150800AB1002F0F0FF012032BD80B54022DFF84C1666
S3150800AB20DFF8380602F02BF84FF40072DFF840160B
S3150800AB30DFF82C0602F023F801BD80B5FFF7ECFF1D
S3150800AB40DFF8240603F0D6F80122DFF82816DFF826
S3150800AB50180603F03BF801BD0EB42DE9F8410400D0
S3150800AB604FF480775FF00008DFF80C56424639004C
S3150800AB70280001F02BFE07AE32002100DFF8F805A9
S3150800AB8003F01CFA0500DFF8F025A4A1DFF8E805B4
S3150800AB9003F030FADFF8E00501F070FF010089B232
S3150800ABA0DFF8D405FFF72FFFBDE8F2015DF810FBCB
S3150800ABB01CB5040000208DF80000200080B2000AB1
S3150800ABC08DF8000001226946DFF8B00502F033F877
S3150800ABD020008DF8000001226946DFF8A00502F082
S3150800ABE02AF813BD2DE9F04104000D0000200026C7
S3150800ABF000275FF000084046290080B289B28842E3
S3150800AC0018D23000C0B2002807D1012006004046FD
S3150800AC1080B2205C0002070009E0002006004046DA
S3150800AC2080B2205C0743380080B2F8F735FB18F18C
S3150800AC300108E0E7BDE8F081F8B500208DF80000CE
S3150800AC4000244FF480750026DFF834753200290099
S3150800AC50380001F0BBFDDFF8240501F0DBFF002812
S3150800AC601ED101226946DFF8140502F009F800280A
S3150800AC7010D09DF80000DFF80815220092B288541B
S3150800AC80641C200080B2B0F5807F03DA00208DF8BE
S3150800AC900000E6E7210089B2DFF8E404FFF7A2FF27
S3150800ACA0F1BD38B504000D004FF47A732A0092B24C
S3150800ACB02100DFF8D00402F01DFF012032BD80B567
S3150800ACC04FF48072DFF8C014DFF8B00401F057FFC4
S3150800ACD001BD80B5FFF7F3FFDFF8A80403F00AF813
S3150800ACE00122DFF8A814DFF89C0402F06FFF01BD0B
S3150800ACF001B501226946DFF8980401F09CFF01BD01
S3150800AD0070B504000D000026DFF8880400780028D6
S3150800AD1017D0DFF88404FFF71FFF00200600300075
S3150800AD20290080B289B2884208D2300080B2215CFC
S3150800AD30DFF86804FFF710FF761CF0E795A0FFF729
S3150800AD400BFF290089B2200003F0CAF9290089B24D
S3150800AD50200003F021FA70BD80B500208DF80000B0
S3150800AD60DFF82C0401F056FF00280FD101226946AE
S3150800AD70DFF81C0401F084FF002807D0012168468B
S3150800AD80FFF7BEFF00208DF80000EFE701BD70B5A4
S3150800AD9004000D000026DFF8080401F007FF29006B
S3150800ADA089B2884214D35FF0FF31DFF8F8030068F0
S3150800ADB002F0DAFD2A0092B22100DFF8E40301F07E
S3150800ADC0DCFFDFF8E003006802F00DFE012024E056
S3150800ADD03000461C80B264281EDA012002F08FFD7E
S3150800ADE0761CDFF8BC0301F0E1FE290089B288422F
S3150800ADF0EED35FF0FF31DFF8AC03006802F0B4FD74
S3150800AE002A0092B22100DFF8980301F0B6FFDFF8B6
S3150800AE109403006802F0E7FD002070BD257300006A
S3150800AE20F8B5C0B00024DFF8780301F0F3FE002877
S3150800AE3075D1DFF874030078002870D14FF4807557
S3150800AE4000266F4632002900380001F0BFFC5FF08B
S3150800AE50FF31DFF85003006802F086FD6946DFF827
S3150800AE60400301F0D5FF0400DFF83803006802F05C
S3150800AE70BAFD9DF8020003F0EAFE00282CD0012056
S3150800AE80DFF8241308700020DFF81C1348709DF8BB
S3150800AE900200C54988702500EDB26E46C34F2A00E8
S3150800AEA03100380001F092FDBF4880F883405FF01A
S3150800AEB0FF31BF48006802F057FD4FF47A73BA486D
S3150800AEC090F8832092B2B949BA4802F013FEB848FE
S3150800AED0006802F088FDA6E75FF0FF31B148006818
S3150800AEE002F042FD6946AE4801F052FF0400AD4843
S3150800AEF0006802F078FD5FF0FF31AD48006802F0A7
S3150800AF0033FD4FF47A732200D2B292B26946A94849
S3150800AF1002F0F0FDA648006802F065FD83E741B03F
S3150800AF20F0BD2DE9F04104000D00207803F08CFEF9
S3150800AF3000282CD05FF0FF319A48006802F014FD13
S3150800AF4084260027DFF870823A003100404601F077
S3150800AF503DFC9A49924801F05BFF20789649497969
S3150800AF60884210D121789648FFF7F6FD8F498C481C
S3150800AF7001F00EFF84260027DFF82C823A00310004
S3150800AF80404601F023FC8748006802F02CFDBDE826
S3150800AF90F08100000D0A0000F8B500248248007808
S3150800AFA000285ED087480078401C86490870854886
S3150800AFB000780A2858DB0020824908707A484078C9
S3150800AFC002281EDA78484078401C774948705FF0B6
S3150800AFD0FF317748006802F0C7FC4FF47A7372486D
S3150800AFE090F8832092B27149724802F083FD704846
S3150800AFF0006802F0F8FC6C4841787348FFF7ACFD2E
S3150800B00032E07248FFF7A8FD0020040020006649D8
S3150800B01091F88310C0B2884209D263482100C9B2A8
S3150800B0200844C1786A48FFF797FD641CEEE769484B
S3150800B030FFF792FD5FF0FF315A48006802F094FC72
S3150800B0405A49574801F0A4FE84250026564F320077
S3150800B0502900380001F0BAFB5248006802F0C3FC28
S3150800B06002E0002057490870F1BD38B504000D000C
S3150800B0705FF0FF314E48006802F076FC4FF47A73B1
S3150800B0802A0092B221004B4802F034FD4848006875
S3150800B09002F0A9FC012032BD80B54FF480724E49FA
S3150800B0A03B4801F06CFD4FF480724C493C4801F076
S3150800B0B066FD01BD80B5FFF7EFFF3E4802F01AFEB8
S3150800B0C0012247493B4802F081FD01BD10B5040045
S3150800B0D020684449884207D126480078FFF770FC63
S3150800B0E000202449087016E020683F49884207D1A5
S3150800B0F026480088FFF75CFD0020244908800AE0FE
S3150800B10020683A49884206D135480078FFF7F0FDAD
S3150800B11000203349087010BD10B50400200002F065
S3150800B12025FE3349086020682E49884204D103F079
S3150800B13091FD03F09DFD10E020682B49884204D15B
S3150800B14003F09CFD03F0A8FD07E020682749884224
S3150800B15003D103F0A7FD03F0B3FD10BDFC6A002080
S3150800B1602C6B0020A46B0020F067002030690020BB
S3150800B170DC590020C46C0020786200200C6B00208B
S3150800B1807861002070680020785E00206A6C0020D4
S3150800B1901C6B00206D6C002034630108586501089B
S3150800B1A03C6B0020A86B0020C4640020C764002004
S3150800B1B0AC6B0020B0670020486500204B65002076
S3150800B1C0F8480108C66C00202C490108D04301083C
S3150800B1D064650108AC660108785F00207860002085
S3150800B1E0C56C00200038014000480040004C004073
S3150800B1F0246C002080B52D20DFF88C1D08700121F5
S3150800B200DFF8840D02F0B4FF01BD10B5040030204C
S3150800B210DFF8741D0870DFF8700D44700221DFF83E
S3150800B220680D02F0A5FF10BD80B52F20DFF8581D68
S3150800B23008700121DFF8500D02F09AFF01BD80B5B4
S3150800B2405020DFF8441D08700121DFF83C0D02F09C
S3150800B2508FFF01BD80B55120DFF82C1D0870012134
S3150800B260DFF8240D02F084FF01BD10B50024A120EB
S3150800B270DFF8141D2200D2B28854641CDFF87C0B58
S3150800B2800088DFF8041D2200D2B28854641CDFF857
S3150800B2906C0B008880B2000ADFF8EC1C2200D2B2E0
S3150800B2A08854641CDFF8580B0088DFF8DC1C220081
S3150800B2B0D2B28854641CDFF8480B008880B2000AB2
S3150800B2C0DFF8C41C2200D2B28854641CDFF8640B71
S3150800B2D00088DFF8B41C2200D2B28854641CDFF858
S3150800B2E0540B008880B2000ADFF89C1C2200D2B2F8
S3150800B2F08854641CDFF8400B0088DFF88C1C220099
S3150800B300D2B28854641CDFF8300B008880B2000A79
S3150800B310DFF8741C2200D2B28854641CDFF8440B90
S3150800B3200088DFF8641C2200D2B28854641CDFF857
S3150800B330340B008880B2000ADFF84C1C2200D2B217
S3150800B3408854641CDFF8200B0088DFF83C1C2200B8
S3150800B350D2B28854641CDFF8100B008880B2000A49
S3150800B360DFF8241C2200D2B28854641CDFF8FC0AD9
S3150800B3700088DFF8141C2200D2B28854641CDFF857
S3150800B380EC0A008880B2000ADFF8FC1B2200D2B261
S3150800B3908854641CDFF8D80A0088DFF8EC1B220002
S3150800B3A0D2B28854641CDFF8C80A008880B2000A42
S3150800B3B0DFF8D41B2200D2B28854641CDFF8B40A22
S3150800B3C00088DFF8C41B2200D2B28854641CDFF858
S3150800B3D0A40A008880B2000ADFF8AC1B2200D2B2A9
S3150800B3E08854641C2100C9B2DFF89C0B02F0C0FE29
S3150800B3F010BD38B500240021B120DFF88C2B2300BE
S3150800B400DBB2D054641CDFF8200B0078DFF8782B09
S3150800B4102300DBB2D054641C00200100DFF8082B9F
S3150800B4201278C9B291421BD2DFF8001B0200D2B2D1
S3150800B43031F81210DFF8502B2300DBB2D154641C0C
S3150800B440DFF8E81A0200D2B231F8121089B2090AF6
S3150800B450DFF8342B2300DBB2D154641C401CDCE734
S3150800B460DFF8281B0978DFF8202B2300DBB2D1543C
S3150800B470641C00252800DFF8141B0978C0B288422E
S3150800B4801BD2DFF83C0B2900C9B230F81100DFF8EF
S3150800B490F81A2200D2B28854641CDFF8240B29005B
S3150800B4A0C9B230F8110080B2000ADFF8DC1A2200AF
S3150800B4B0D2B28854641C6D1CDCE72100C9B2DFF8DF
S3150800B4C0C80A02F055FE31BD80B5DFF8380B0078A2
S3150800B4D001280AD1DFF8300B0078012802D1FFF7DE
S3150800B4E088FF41E0FFF7C1FE3EE02120DFF8981A09
S3150800B4F00870DFF808090088DFF88C1A4870DFF84A
S3150800B50000090088DFF8801A8870DFF828090088A3
S3150800B510DFF8741AC870DFF820090088DFF8681A9F
S3150800B5200871DFF840090088DFF85C1A4871DFF80F
S3150800B53038090088DFF8501A8871DFF83009008862
S3150800B540DFF8441AC871DFF828090088DFF8381AC6
S3150800B5500872DFF820090088DFF82C1A48720A21D9
S3150800B560DFF8240A02F004FE01BD2DE9F0410024AB
S3150800B570DFF888080088DFF8741B0D88451BDFF89C
S3150800B58080080088DFF8901B0E88861BDFF8A40861
S3150800B5900088DFF8881B0F88C71BDFF89C0800881F
S3150800B5A0DFF8A41BB1F80080B0EB0808A220DFF88A
S3150800B5B0D8192200D2B28854641CDFF8CC092100BD
S3150800B5C0C9B24554641C280080B2000ADFF8B819CD
S3150800B5D02200D2B28854641CDFF8AC092100C9B233
S3150800B5E04654641C300080B2000ADFF89C19220019
S3150800B5F0D2B28854641CDFF890092100C9B24754B6
S3150800B600641C380080B2000ADFF87C192200D2B226
S3150800B6108854641CDFF870092100C9B200F801805B
S3150800B620641C404680B2000ADFF85C192200D2B2D8
S3150800B6308854641CDFF8B40A0088DFF84C19220025
S3150800B640D2B28854641CDFF8A40A008880B2000AC3
S3150800B650DFF834192200D2B28854641CDFF8B80A1D
S3150800B6600088DFF824192200D2B28854641CDFF857
S3150800B670A80A008880B2000ADFF80C192200D2B2A4
S3150800B6808854641CDFF8940A0088DFF8FC18220046
S3150800B690D2B28854641CDFF8840A008880B2000A93
S3150800B6A0DFF8E4182200D2B28854641CDFF8980A3E
S3150800B6B00088DFF8D4182200D2B28854641CDFF858
S3150800B6C0880A008880B2000ADFF8BC182200D2B2C5
S3150800B6D08854641C2100C9B2DFF8AC0802F048FDA2
S3150800B6E0BDE8F08170B5002400200025B221DFF8FE
S3150800B6F098282300DBB2D154641CDFF82C1809788B
S3150800B700DFF884282300DBB2D154641C002108002A
S3150800B710DFF814281278C0B290421ED2DFF80C085F
S3150800B7200A00D2B230F81220DFF8D00A0B00DBB2DA
S3150800B73030F81300121A1500DFF84C082200D2B2AE
S3150800B7408554641C280080B2000ADFF83C282300D0
S3150800B750DBB2D054641C491CD9E700263000DFF858
S3150800B760C8170978C0B2884229D2DFF8C007310065
S3150800B770C9B230F81110DFF8840A3200D2B230F8B4
S3150800B7801200091A0D00DFF8740A3100C9B230F840
S3150800B7901100DFF8F4172200D2B28854641CDFF8CF
S3150800B7A05C0A3100C9B230F8110080B2000ADFF82D
S3150800B7B0D8172200D2B28854641C761CCEE7210022
S3150800B7C0C9B2DFF8C40702F0D3FC70BD80B5DFF854
S3150800B7D03408007801280AD1DFF82C0800780128F7
S3150800B7E002D1FFF77FFF4BE0FFF7BFFE48E02320BB
S3150800B7F0DFF894170870DFF804060188DFF8EC080C
S3150800B8000088091ADFF880074170DFF8F405018817
S3150800B810DFF804090088091ADFF86C078170DFF879
S3150800B82014060188DFF8F4080088091ADFF85807B3
S3150800B830C170DFF804060188DFF80C090088091AC8
S3150800B840DFF844070171DFF8A4080088DFF8381725
S3150800B8504871DFF8C4080088DFF82C178871DFF80C
S3150800B860BC080088DFF82017C871DFF8DC080088F4
S3150800B870DFF8141708720921DFF80C0702F078FCC4
S3150800B88001BD80B53120DFF800170870DFF8940A8B
S3150800B890007800280ED0DFF8900A0078002804D037
S3150800B8A00120DFF8E416487008E00020DFF8D81613
S3150800B8B0487003E0FF20DFF8D0164870DFF86C0AFE
S3150800B8C0007800280ED0DFF8680A0078002804D02F
S3150800B8D00120DFF8B416887008E00020DFF8A81603
S3150800B8E0887003E0FF20DFF8A0168870DFF8440AA6
S3150800B8F0007800280ED0DFF8400A0078002804D027
S3150800B9000120DFF88416C87008E00020DFF87816F2
S3150800B910C87003E0FF20DFF87016C8700020DFF853
S3150800B920681608710521DFF8600602F021FC01BDE2
S3150800B93010B504002020DFF850160870DFF8480616
S3150800B94044700221DFF8400602F012FC10BD10B563
S3150800B95004002A20DFF830160870DFF82C06447039
S3150800B9600221DFF8240602F003FC10BD10B504001E
S3150800B9702720DFF814160870DFF80C064470022139
S3150800B980DFF8040602F0F4FB10BD80B52920DFF8C5
S3150800B990F81508700121DFF8F00502F0E9FB01BD92
S3150800B9A0F8B504000D0000260020B321DFF8D825DD
S3150800B9B03300DBB2D154761CDFF86C150978DFF852
S3150800B9C0C8253300DBB2D154761C0027380029007D
S3150800B9D0C0B2C9B288420AD23800C0B2205CDFF8C9
S3150800B9E0A8153200D2B28854761C7F1CEEE73100C7
S3150800B9F0C9B2DFF8940502F0BBFBF1BDF8B5040047
S3150800BA000D0016001F002820DFF87C150870DFF8E7
S3150800BA1078054470DFF870058570DFF86C05C67028
S3150800BA20DFF8640507710521DFF85C0502F0A0FB65
S3150800BA30F1BD80B52E20DFF8501508700121DFF81A
S3150800BA40480502F095FB01BD10B504004920DFF852
S3150800BA5038150870DFF8300544700221DFF828052C
S3150800BA6002F086FB10BD10B504004020DFF818155B
S3150800BA700870DFF8140544700221DFF80C0502F09F
S3150800BA8077FB10BD80B54620DFF8FC14087003214B
S3150800BA90DFF8F40402F06CFB01BD80B53A20DFF84C
S3150800BAA0E81408700121DFF8E00402F061FB01BD2B
S3150800BAB010B50024A320DFF8D0142200D2B288548F
S3150800BAC0641CDFF878080088DFF8BC142200D2B2BC
S3150800BAD08854641CDFF86408008880B2000ADFF81E
S3150800BAE0A8142200D2B28854641CDFF854080088CF
S3150800BAF0DFF894142200D2B28854641CDFF8400898
S3150800BB00008880B2000ADFF880142200D2B2885476
S3150800BB10641CDFF830080088DFF86C142200D2B203
S3150800BB208854641CDFF81C08008880B2000ADFF815
S3150800BB3058142200D2B28854641CDFF80C08008816
S3150800BB40DFF844142200D2B28854641CDFF8F807E0
S3150800BB50008880B2000ADFF830142200D2B2885476
S3150800BB60641C2100C9B2DFF8200402F001FB10BDF5
S3150800BB7038B500240020B421DFF80C242300DBB2FA
S3150800BB80D154641CDFF8A0130978DFF8FC232300DE
S3150800BB90DBB2D154641C00252800DFF88C13097821
S3150800BBA0C0B288421BD2DFF8A4072900C9B230F810
S3150800BBB01100DFF8D4132200D2B28854641CDFF8CF
S3150800BBC08C072900C9B230F8110080B2000ADFF8E4
S3150800BBD0B8132200D2B28854641C6D1CDCE721001D
S3150800BBE0C9B2DFF8A40302F0C3FA31BD80B5DFF8A5
S3150800BBF01404007801280AD1DFF80C04007801281B
S3150800BC0002D1FFF7B5FF22E0FFF752FF1FE033200E
S3150800BC10DFF874130870DFF824070088DFF8681364
S3150800BC204870DFF81C070088DFF85C138870DFF8B7
S3150800BC3014070088DFF85013C870DFF80C0700886F
S3150800BC40DFF8441308710521CF4802F091FA01BDC7
S3150800BC5080B53520CC4908700121CB4802F088FA16
S3150800BC6001BD38B5002000243921C74A2300DBB2BC
S3150800BC70D154641CDFF8D8160978C34A2300DBB20E
S3150800BC80D154641CDFF8C8164978BF4A2300DBB2D2
S3150800BC90D154641CDFF8B816C978BB4A2300DBB256
S3150800BCA0D154641CDFF8A8160979B74A2300DBB219
S3150800BCB0D154641C00210800C0B2042824DADFF835
S3150800BCC094060A00D2B210440079302814DBDFF853
S3150800BCD084060A00D2B2104400793A280CDADFF852
S3150800BCE074060A00D2B2104400793038A64A2300F6
S3150800BCF0DBB2D054641C05E0FF20A34A2300DBB264
S3150800BD00D054641C491CD6E700221000C0B20C2887
S3150800BD100BDADFF844061100C9B2405C9A492300E1
S3150800BD20DBB2C854641C521CEFE700200100C9B2FC
S3150800BD300C290BDADFF824160200D2B2895C924A83
S3150800BD402300DBB2D154641C401CEFE7DFF8001671
S3150800BD5089798D4A2300DBB2D154641CDFF8F015CB
S3150800BD60C979894A2300DBB2D154641C002528000E
S3150800BD70C0B20C280CDADFF8E4052900C9B2084479
S3150800BD80807F81492200D2B28854641C6D1CEEE77C
S3150800BD902100C9B27C4802F0EBF931BD80B52620F6
S3150800BDA0794908700121784802F0E2F901BD80B5A9
S3150800BDB02B2075490870DFF8A80500787249487085
S3150800BDC00221714802F0D4F901BD80B5DFF8940567
S3150800BDD00078FF2806D142206B490870FF206A497F
S3150800BDE0487005E042206849087000206649487096
S3150800BDF00221654802F0BCF901BD0000406C002034
S3150800BE00426C002080B5DFF85C050078FF2806D173
S3150800BE1045205D490870FF205B49487005E04520CC
S3150800BE20594908700020584948700221564802F0BE
S3150800BE309FF901BD446C0020466C002080B548205F
S3150800BE4051490870DFF8200500784F494870DFF837
S3150800BE501C0500784C49887003214B4802F088F984
S3150800BE6001BD0000506C0020526C0020546C00206C
S3150800BE70566C0020586C002038B500200024632139
S3150800BE80414A2300DBB2D154641CDFF8E414097874
S3150800BE903D4A2300DBB2D154641CDFF8D814097874
S3150800BEA0394A2300DBB2D154641CDFF8CC14097874
S3150800BEB0354A2300DBB2D154641CDFF8C014097874
S3150800BEC0314A2300DBB2D154641CDFF8B414097874
S3150800BED02D4A2300DBB2D154641CDFF8A814097874
S3150800BEE0294A2300DBB2D154641CDFF89C14097874
S3150800BEF0254A2300DBB2D154641C00252800C0B2B1
S3150800BF0004280BDADFF884042900C9B2405C1E490C
S3150800BF102200D2B28854641C6D1CEFE72100C9B216
S3150800BF20194802F025F931BD736C0020F869002024
S3150800BF30F8B504000D00160000275A2012493A00E9
S3150800BF40D2B288547F1C2000C0B2002806D0012037
S3150800BF500D493A00D2B288547F1C05E000200A49F0
S3150800BF603A00D2B288547F1C07483900C9B24654F1
S3150800BF707F1C05483900C9B245547F1C3900C9B22F
S3150800BF80014802F0F5F8F1BDCC650020776C002079
S3150800BF9038B5040000255B20DFF8F4132A00D2B276
S3150800BFA088546D1CDFF8E8032900C9B244546D1C97
S3150800BFB02900C9B2DFF8D80302F0DAF831BD00006B
S3150800BFC0386A002010B500245C20DFF8C41322006C
S3150800BFD0D2B28854641C2100C9B2DFF8B40302F057
S3150800BFE0C7F810BD10B500245D20DFF8A4132200A1
S3150800BFF0D2B28854641C2100C9B2DFF8940302F057
S3150800C000B7F810BD7F0100207E01002010B500247E
S3150800C0105E20DFF87C132200D2B28854641C21000B
S3150800C020C9B2DFF86C0302F0A3F810BD10B50024FE
S3150800C0305F20DFF85C132200D2B28854641C21000A
S3150800C040C9B2DFF84C0302F093F810BD70B50400CE
S3150800C0500D0000266020CE493200D2B28854761CE4
S3150800C060CB483100C9B24454761CC9483100C9B21C
S3150800C0704554761C3100C9B2C54802F079F870BD3E
S3150800C08010B500246120C2492200D2B28854641C2B
S3150800C0902100C9B2BE4802F06BF810BD38B50400DD
S3150800C0A000256520BA492A00D2B288546D1CB848C2
S3150800C0B02900C9B244546D1C2900C9B2B44802F01B
S3150800C0C057F831BD38B5040000256720B0492A0065
S3150800C0D0D2B288546D1CAE482900C9B244546D1CAE
S3150800C0E02900C9B2AA4802F043F831BD486C0020BD
S3150800C0F038B5040000256920A5492A00D2B288541B
S3150800C1006D1CA3482900C9B244546D1C2900C9B244
S3150800C1109F4802F02DF831BD4A6C00204C6C002077
S3150800C12038B5040000256B2099492A00D2B28854F4
S3150800C1306D1C97482900C9B244546D1C2900C9B220
S3150800C140934802F015F831BD4E6C002038B504004E
S3150800C15000256D208E492A00D2B288546D1C8C4861
S3150800C1602900C9B244546D1C2900C9B2884801F097
S3150800C170FFFF31BD38B5040000256E2084492A002A
S3150800C180D2B288546D1C82482900C9B244546D1C29
S3150800C1902900C9B27E4801F0EBFF31BD10B5040095
S3150800C1A0F1207B4908707A4844700221784801F0EA
S3150800C1B0DFFF10BD38B504000D00F2207449087081
S3150800C1C073484470280080B2000A71498870704824
S3150800C1D0C57004216E4801F0CBFF31BD38B50400A7
S3150800C1E00D00F4206A4908706948447068488570EB
S3150800C1F00321674801F0BCFF31BD0000186A002022
S3150800C20038B5002400203C21614A2300DBB2D15412
S3150800C210641C604909785E4A2300DBB2D154641C69
S3150800C2205D4909785A4A2300DBB2D154641C5B493C
S3150800C2300978574A2300DBB2D154641C5849097857
S3150800C240534A2300DBB2D154641C56490978504A34
S3150800C2502300DBB2D154641C002528005149097813
S3150800C260C0B288420AD250482900C9B2405C48493F
S3150800C2702200D2B28854641C6D1CEEE72100C9B2B4
S3150800C280434801F075FF31BD38B5002400203E2132
S3150800C2903F4A2300DBB2D154641C444909783C4A1E
S3150800C2A02300DBB2D154641C41490978384A23007B
S3150800C2B0DBB2D154641C3F490988354A2300DBB2F6
S3150800C2C0D154641C3B49098889B2090A304A2300BB
S3150800C2D0DBB2D154641C384909782D4A2300DBB2F5
S3150800C2E0D154641C35490978294A2300DBB2D15454
S3150800C2F0641C0025280031490978C0B288420AD250
S3150800C3002F482900C9B2405C21492200D2B288547C
S3150800C310641C6D1CEEE72100C9B21D4801F028FF18
S3150800C32031BD0000926C00208F6C0020936C0020B9
S3150800C330906C0020946C0020916C0020386C0020D2
S3150800C3403A6C00203C6C00203E6C0020D869002026
S3150800C350586B0020646B0020DC6A0020A869002066
S3150800C3608101002080010020856C0020866C002059
S3150800C370966C0020976C0020986C0020996C002021
S3150800C3809A6C00209B6C00209C6C0020B06B0020EF
S3150800C390CC650020706C00206F6C0020716C00204A
S3150800C3A0726C0020736C0020BC6A0020756C00203B
S3150800C3B0746C00202E6C0020766C0020776C0020B0
S3150800C3C0CC6A00202DE9F84302005FF0000E5FF00A
S3150800C3D00008086830FA0EF0002800F013810120E2
S3150800C3E010FA0EF003000868184004009C4240F05A
S3150800C3F006814868002831D0012820D0022825D097
S3150800C40003283CD011281DD0122823D0DFF874C386
S3150800C410604523D0DFF870C360451FD0DFF86CC3D2
S3150800C42060451BD0DFF868C3604517D0DFF864C3E2
S3150800C430604513D0DFF860C360450FD022E0C868B6
S3150800C44080461FE0C868001D80461BE0C8680830A3
S3150800C450804617E0C8680C30804613E088680028D4
S3150800C46002D10420804609E08868012803D1082003
S3150800C4708046136102E008208046536102E00020EE
S3150800C4808046FFE7B4F5807F01D2160000E0161D4E
S3150800C490B4F5807F02D25FEA8E0702E0BEF1080794
S3150800C4A0BF00D6F800C00F20B8403CEA000C18FAC6
S3150800C4B007F050EA0C0CC6F800C04868C00040F106
S3150800C4C09E80DFF8D802006850F00100DFF8CCC281
S3150800C4D0CCF80000DFF8C402006810F001000090F4
S3150800C4E00098DFF8BC02F4465FEA9C0C50F82CC0B2
S3150800C4F05FF00F091EF00300C0B2800019FA00F9B8
S3150800C5003CEA090CA748824202D15FF000091FE005
S3150800C510A548824202D15FF0010919E0A348824288
S3150800C52002D15FF0020913E0A148824202D15FF00E
S3150800C53003090DE09F48824202D15FF0040907E033
S3150800C5409D48824202D15FF0050901E05FF00609C5
S3150800C55065461EF00300C0B2800019FA00F959EAD0
S3150800C56005058F48F4465FEA9C0C40F82C5048684D
S3150800C570C00307D5914800682043DFF840C2CCF8CD
S3150800C580000006E08D480068A043DFF830C2CCF80A
S3150800C59000004868800307D5894800682043DFF80B
S3150800C5A020C2CCF8000006E085480068A043DFF802
S3150800C5B010C2CCF800004868C00207D58148006858
S3150800C5C02043DFF800C2CCF8000006E07D4800688A
S3150800C5D0A043DFF8F0C1CCF800004868800207D510
S3150800C5E0794800682043DFF8E0C1CCF8000006E08F
S3150800C5F075480068A043DFF8D0C1CCF800001EF1EA
S3150800C600010EE6E6BDE8F183F0B503000027080051
S3150800C610F840002800F09A800120B840084002003F
S3150800C620002A00F091805E48BC465FEA9C0C50F8F0
S3150800C6302CC05FF00F0E17F00300C0B280001EFA80
S3150800C64000FE1EEA0C0C64465648834202D15FF08F
S3150800C650000C1FE05448834202D15FF0010C19E038
S3150800C6605248834202D15FF0020C13E050488342DD
S3150800C67002D15FF0030C0DE04E48834202D15FF011
S3150800C680040C07E04C48834202D15FF0050C01E038
S3150800C6905FF0060C17F00300C0B280001CFA00FC1D
S3150800C6A0644532D15FF00F0C17F00300C0B280006A
S3150800C6B01CFA00FC64463A48BC465FEA9C0C50F8F3
S3150800C6C02C00A043DFF8D8C0BE465FEA9E0E4CF8A1
S3150800C6D02E003A4800689043DFF8E0C0CCF8000026
S3150800C6E0374800689043DFF8D8C0CCF800003548D2
S3150800C6F000689043DFF8CCC0CCF8000032480068E8
S3150800C7009043DFF8C4C0CCF80000B2F5807F01D2B0
S3150800C7101D0000E01D1DB2F5807F01D2BE0002E0BB
S3150800C720B7F10806B60028685FF00F0C1CFA06FC7D
S3150800C73030EA0C005FF0040C1CFA06FC5CEA000008
S3150800C7402860D8689043D8607F1C60E7F0BD130066
S3150800C750DBB2002B03D00B009BB2036103E00B0096
S3150800C7609BB21B040361704710B4C2680B009BB2EE
S3150800C77013400C00A4B2944354EA0344046110BC69
S3150800C7807047000000001110000012100000211070
S3150800C790000022100000311000003210181002406C
S3150800C7A00800014000080140000C0140001001404B
S3150800C7B00014014000180140001C0140000401401B
S3150800C7C004040140080401400C04014062F30F22EE
S3150800C7D062F31F42401810F0030308D0C91A1FD38A
S3150800C7E0DB0748BF00F8012D28BF20F8022D1300EB
S3150800C7F030B414461546103928BF20E93C00FAD84B
S3150800C800490728BF20E90C0048BF40F8042D8900D5
S3150800C81028BF20F8022D48BF00F8012D30BC70470C
S3150800C820C91818BF00F8012DCB0728BF00F8012D3D
S3150800C8307047F0B40246106895681318506803EB01
S3150800C8405004C00721D54D441FE0F0BC02F10C008E
S3150800C850704713F8017B05F8017B491EF9D1A0B191
S3150800C860B60813F8011B06F00306032E08BF13F8D3
S3150800C870016B01EB06214942801C294405D011F8B9
S3150800C880016B05F8016B401EF9D1A342DDD013F800
S3150800C890016B16F0030104BF13F8011BC91C30090C
S3150800C8A00F28DAD113F8010B0F30D6E7C21750401C
S3150800C8B0801AB0FA80F10AD08840D1F19D01D207DA
S3150800C8C042EAC151020672F1004241EB102070475C
S3150800C8D010B5FF2313EAD0541DBF13EAD1529C4268
S3150800C8E09A4239E0A41ADA0780EA0103134042EAB9
S3150800C8F0012142EA0020421A3CBF641E01EB4202B3
S3150800C900090AB2FBF1FE01FB1E221202B2FBF1F08C
S3150800C91001FB10226EF30F201202B2FBF1FE4EEA63
S3150800C92000207F3406DDFE2C24DA53EA500050EB53
S3150800C930C45010BDD4F1020401FB1E2240F08071E0
S3150800C940192C1DDC21FA04F0C4F12004A14011437E
S3150800C95071F10042584110BD9C421ABF03EAD152F8
S3150800C9609A420FE080EA010E0EF00043400004D020
S3150800C970490016D143F0FF4010BD490008BFD34314
S3150800C980180010BD9C4205D1D21AF7D001F000411B
S3150800C990484010BD4A0212BF0846484000F0004011
S3150800C9A010BD4AB90902B1FA81F2914044B1A418FE
S3150800C9B0C00140F000409EE7C90141F000415242E3
S3150800C9C00002B0FA80F4A040141B94E762B38B0708
S3150800C9D008D0521E11F8013B00F8013B00F02480F4
S3150800C9E08B07F6D1830740F0208000BF103A07D3A3
S3150800C9F030B4B1E83810103AA0E83810F9D230BC93
S3150800CA00530724BFB1E80810A0E8081044BF51F83E
S3150800CA10043B40F8043BD20724BF31F8022B20F828
S3150800CA20022B44BF0B7803707047121F17D35B00A5
S3150800CA3009D151F8043B20F8023B1B0C121F20F8C1
S3150800CA40023BF6D20BE051F8043B00F8013B1B0A07
S3150800CA5020F8023B1B0C121F00F8013BF3D238BF2B
S3150800CA60121D521E24BF11F8013B00F8013BF8D8ED
S3150800CA7070470268531C03601170704700F1010388
S3150800CA80810704D010F8011B89B18107FAD1026821
S3150800CA90B2F10131914311F0803F04BF50F8042FE1
S3150800CAA0F6E710F8011B11B110F8011BFBE7C01AD5
S3150800CAB070472D00C0F3C75181B1FF2906D0C110B8
S3150800CAC0400721F0E04101F16051704741020CBF77
S3150800CAD040F4E0016FF000410020704700F000418B
S3150800CAE000020AD0B0FA80FC00FA0CF001F160519D
S3150800CAF0A1EB0C5101EBD0214005704740EA010C2F
S3150800CB001CEB0C0F07D0884205D14FEA400C1CF1EC
S3150800CB10807F98BF804270474FF0807C1CEB400FA7
S3150800CB2094BF1CEB410F05E040EA010C1CEB0C0F0F
S3150800CB3001D28142704718BF8842704770B50848CD
S3150800CB40007800280AD1012005490870022400252A
S3150800CB50044E2A0021003000FFF738FE014870BD58
S3150800CB60C16C0020666C0020007870470100012027
S3150800CB70087001207047407870474170704703007D
S3150800CB80002B02D15FF0FF300FE01960186800280B
S3150800CB9002D15FF0FF3008E018681044401E586064
S3150800CBA0186898609868D8600020704701000029C6
S3150800CBB002D00868002801D1002011E0C8688A68F8
S3150800CBC0904207D34A68C868101A8B680A689B1A85
S3150800CBD0181802E08A68C868101A002800D0401E93
S3150800CBE070470100002902D00868002802D15FF0CA
S3150800CBF0FF300EE0C8688A68904203D3C86889681F
S3150800CC00401A06E048688A68801ACA680968521A8B
S3150800CC10101870470100002902D00868002801D1C1
S3150800CC20012007E08868C968884201D1012000E030
S3150800CC300020C0B27047F8B504000E001500002C9D
S3150800CC4002D02068002801D1002018E02F0020001B
S3150800CC50FFF7ACFFB84201D2002010E0E1683800C7
S3150800CC60471E002809D030780870761C491C606871
S3150800CC708142F4D120680100F1E7E1602800F2BDA5
S3150800CC8070B504000E001500002C02D0206800289C
S3150800CC9001D100201BE02000FFF7A3FF01008D4211
S3150800CCA001D2290002E0A94200D20D00A2680800BC
S3150800CCB0411E002809D010783070521C761C606816
S3150800CCC08242F4D120680200F1E7A260280070BD14
S3150800CCD02DE9F841ADF5A06DB7B005000C001600BA
S3150800CCE01F00002C02D02068002801D1002040E057
S3150800CCF02800C0B2002807D12000FFF757FFB91C4B
S3150800CD00814214D3002034E02000FFF74FFFB91CFE
S3150800CD10814206D3012080466946200000F038F893
S3150800CD2001E0002080464046C0B20128ECD0E06809
S3150800CD300770401C6168884201D1216808003900E3
S3150800CD40090A0170421C6068824201D1206802000B
S3150800CD5039000800411E002809D030781070761C6A
S3150800CD60521C60688242F4D120680200F1E7E26052
S3150800CD7038000DF5BC6DBDE8F08170B504000D00F6
S3150800CD80160033002A0021000020FFF7A1FF70BD1E
S3150800CD902DE9F04104000D00002C02D0206800287F
S3150800CDA001D1002032E0A068E168884201D1002064
S3150800CDB02CE0A0680678401C6168884201D1216889
S3150800CDC00800017856EA0126471C6068874201D1A7
S3150800CDD020680700B0462000FFF703FF404505D24C
S3150800CDE02068A060A068E06000200FE03000461EC2
S3150800CDF0002809D0387828707F1C6D1C6068874227
S3150800CE00F4D120680700F1E7A7604046BDE8F08145
S3150800CE102DE9F04104000D00002C02D020680028FE
S3150800CE2001D1002031E0A068E168884201D10020E4
S3150800CE302BE0A0680678401C6168884201D1216809
S3150800CE400800017856EA0126471C6068874201D126
S3150800CE5020680700B0462000FFF7C3FE404505D20C
S3150800CE602068A060A068E06000200EE03000461E42
S3150800CE70002809D0387828707F1C6D1C60688742A6
S3150800CE80F4D120680700F1E74046BDE8F0813F008D
S3150800CE9001000800C0B23038092801D8012000E096
S3150800CEA00020704701000800C0B230282AD0312877
S3150800CEB02AD032282AD033282AD034282AD035280E
S3150800CEC02AD036282AD037282AD038282AD03928EE
S3150800CED02AD041282AD042282AD043282AD04428B2
S3150800CEE02AD045282AD046282AD061281ED062286A
S3150800CEF01ED063281ED064281ED065281ED066283A
S3150800CF001ED01FE000201EE001201CE002201AE0CF
S3150800CF10032018E0042016E0052014E0062012E09D
S3150800CF20072010E008200EE009200CE00A200AE09D
S3150800CF300B2008E00C2006E00D2004E00E2002E09D
S3150800CF400F2000E0002070470120704738B5002008
S3150800CF500025DFF8C4070C2101FB05F140580078CD
S3150800CF60002801D1002036E0DFF8AC070C2101FBD0
S3150800CF7005F1405800782D282BD000200400142CE9
S3150800CF8027D2DFF894070C2101FB05F14058005D14
S3150800CF9000280BD1A3A0FDF7DFFDDFF87C070C21E5
S3150800CFA001FB05F108448068804714E0DFF86C0748
S3150800CFB0005D00280DD0DFF860070C2101FB05F1A4
S3150800CFC04058005DDFF85417095D884201D1641C9A
S3150800CFD0D5E76D1CBDE732BD70B500240026DFF825
S3150800CFE04007FDF7B9FD0025DFF82C070C2101FBEA
S3150800CFF005F108448068002831D0DFF81C070C21A9
S3150800D00001FB05F1405800782D280BD1DFF80807F9
S3150800D0100C2101FB05F108444168DFF80807FDF714
S3150800D0209BFD10E0DFF8F0060C2101FB05F1084432
S3150800D0304268DFF8E4060C2101FB05F14158DFF8E8
S3150800D040E806FDF789FD641C2000C0B20A2804DB47
S3150800D05000200400642000F052FC6D1CC4E7012087
S3150800D06070BD80B5DFF8C416DFF8C406FDF774FD99
S3150800D07001BD01B59DF80000082802D00D2801D091
S3150800D08027E043E0DFF8AC060078002802D1FFF776
S3150800D090E8FF3BE00020DFF88416DFF898261278D0
S3150800D0A08854FFF753FF002804D0DFF88C06FDF7F5
S3150800D0B053FD07E0DFF88406FDF74EFDDFF880062E
S3150800D0C0FDF74AFD0020DFF86C160870FFF7C9FF68
S3150800D0D01CE0DFF860060078372813DA0121684675
S3150800D0E0FDF791FC9DF80000DFF83016DFF84426BE
S3150800D0F012788854DFF83C060078401CDFF83416AE
S3150800D100087003E0072168A0FDF726FD01BD80B57C
S3150800D110DFF83006FDF720FDFFF710FDFFF726FDC7
S3150800D120012002BD3EB56846DFF81C1691E81C00D2
S3150800D13080E81C006846FFF7A1FC441EDFF8DC0502
S3150800D1402100C9B2405CFFF7A3FE002801D10020E8
S3150800D15027E0DFF8C8052100C9B2405CFFF7A2FE48
S3150800D16005002800C0B2012809D02800C0B200284E
S3150800D17005D0DFF8D805FDF7EFFC002011E0280000
S3150800D180C0B2002804D10020DFF8C415087007E0F3
S3150800D1902800C0B2012803D10120DFF8B4150870B1
S3150800D1A001203EBD3EB56846DFF8A81591E81C008B
S3150800D1B080E81C006846FFF761FC441EDFF85C0542
S3150800D1C02100C9B2405CFFF763FE002801D10020A8
S3150800D1D027E0DFF848052100C9B2405CFFF762FE88
S3150800D1E005002800C0B2012809D02800C0B20028CE
S3150800D1F005D0DFF85805FDF7AFFC002011E0280040
S3150800D200C0B2002804D10020DFF84C15087007E0EA
S3150800D2102800C0B2012803D10120DFF83C150870A8
S3150800D22001203EBD0D0A00003EB56846DFF82C1504
S3150800D23091E81C0080E81C006846FFF71FFC441EA6
S3150800D240DFF8D8042100C9B2405CFFF721FE0028A8
S3150800D25001D1002027E0DFF8C4042100C9B2405CF0
S3150800D260FFF720FE05002800C0B2012809D02800D3
S3150800D270C0B2002805D0DFF8D404FDF76DFC002005
S3150800D28011E02800C0B2002804D10020DFF8D0142D
S3150800D290087007E02800C0B2012803D10120DFF892
S3150800D2A0C014087001203EBD256300001CB500248B
S3150800D2B0DFF8B004FDF750FCDFF8AC04FDF74CFCD2
S3150800D2C0F7F7F8F8DFF8A404FDF746FCDFF8A00442
S3150800D2D0007800280ED0DFF89C040078002804D0D7
S3150800D2E0DFF89404FDF738FC08E0DFF89004FDF752
S3150800D2F033FC03E0DFF88804FDF72EFCDFF884042E
S3150800D300007800280ED0DFF880040078002804D0C2
S3150800D310DFF87804FDF720FC08E0DFF87404FDF771
S3150800D3201BFC03E0DFF86C04FDF716FCDFF8680465
S3150800D3300078012856D1002004002000DFF85C148C
S3150800D3400978C0B2884216D22000C0B2F6F708FAA9
S3150800D350DFF84C142200D2B231F812100091FFF710
S3150800D360A9FB02000B002100C9B2DFF83804FDF75B
S3150800D370F3FB641CE1E7DFF83004FDF7EDFBDFF8AB
S3150800D3802C040078FE38012804D8DFF82404FDF7B9
S3150800D390E3FB0FE0DFF814040078F6F7DDFAFFF791
S3150800D3A089FB02000B00DFF804040178DFF80404A7
S3150800D3B0FDF7D2FBDFF80004FDF7CEFBDFF8FC0330
S3150800D3C00078000603D5DFF8F803FDF7C5FBDFF89C
S3150800D3D0F403017870A0FDF7BFFBDFF8EC03FDF757
S3150800D3E0BBFB68E0DFF8E403FDF7B6FBDFF8E00314
S3150800D3F0018869A0FDF7B0FBDFF8CC03FDF7ACFBAD
S3150800D400DFF8D003FDF7A8FBDFF8CC03018862A09C
S3150800D410FDF7A2FBDFF8B003FDF79EFBDFF8BC03C0
S3150800D420FDF79AFBDFF8B80301885BA0FDF794FBCC
S3150800D430DFF89403FDF790FBDFF8A803FDF78CFBF4
S3150800D440DFF8A403018854A0FDF786FBDFF878030C
S3150800D450FDF782FBDFF85003FDF77EFBDFF84C0390
S3150800D4600078002803D002280BD005D30EE0DFF899
S3150800D4707C03FDF771FB0CE0DFF87403FDF76CFB2A
S3150800D48007E0DFF87003FDF767FB02E0C848FDF721
S3150800D49063FBC948FDF760FBC8480078000602D55B
S3150800D4A0C748FDF759FBC74801783BA0FDF754FB71
S3150800D4B0C548FDF751FB012016BDB3480078012881
S3150800D4C001D1002003E00120CB49087001207047F4
S3150800D4D00120CA4908700120C94908700120C949B4
S3150800D4E00870012070470120C74908700120C74904
S3150800D4F008700120C6490870012070473EB5684685
S3150800D500C44991E81C0080E81C006846FFF7B6FA93
S3150800D510441E82482100C9B2405CFFF7B9FC0028C6
S3150800D52001D1002019E07D482100C9B2405CFFF70F
S3150800D530B9FC05002900C9B2B748FDF70DFB28005C
S3150800D540C0B2002808D02800C0B20A2804DAB348B6
S3150800D55005700120B249087001203EBD80B5934888
S3150800D5600078FF2804D1AF48FDF7F6FA002003E05B
S3150800D5700120AD490870012002BD80B58B480078AE
S3150800D580FF2804D1A748FDF7E7FA002003E00120A9
S3150800D590A6490870012002BD256400002DE9FE4356
S3150800D5A06846A34991E81C0080E81C0000246846E8
S3150800D5B0FFF764FA451E6846FFF760FA861E574865
S3150800D5C02900C9B2405CFFF763FC002807D053481E
S3150800D5D03100C9B2405CFFF75BFC002801D100208E
S3150800D5E02CE04E482900C9B2405CFFF75BFC0700F7
S3150800D5F04A483100C9B2405CFFF754FC8046C14630
S3150800D6005FFA89F90A213800C0B201FB09094946BF
S3150800D61089B28848FDF7A0FA484680B200280CD09F
S3150800D620484680B2642808DA8348A0F80090FF20AC
S3150800D630824908800120824908700120BDE8FE83DE
S3150800D6400120804908700120704701207E49087032
S3150800D6500120704701207D4908700120704701208C
S3150800D6607B490870012070472DE9F84384B0684665
S3150800D67078491022FFF7BAF900246846FFF7FEF941
S3150800D680451E6846FFF7FAF9861E24482900C9B2DE
S3150800D690405CFFF7FDFB002807D020483100C9B2DF
S3150800D6A0405CFFF7F5FB002801D100202CE01B4861
S3150800D6B02900C9B2405CFFF7F5FB0700174831009F
S3150800D6C0C9B2405CFFF7EEFB8046C1465FFA89F9AE
S3150800D6D00A213800C0B201FB0909494689B25E48E9
S3150800D6E0FDF73AFA484680B200280CD0484680B280
S3150800D6F0642808DA5948A0F80090FF20584908809D
S3150800D700012058490870012005B0BDE8F0830120C2
S3150800D71055490870012070470000002070690020F4
S3150800D7202C5C0108A4650108CC630108C4600108E3
S3150800D730AC6501086C6C0020D460010840590108EA
S3150800D740E460010858590108D863010870590108AE
S3150800D7506D6C0020E46301087C010020F063010879
S3150800D7607D010020B4650108605501088859010843
S3150800D770936C0020906C0020D0500108F0500108EE
S3150800D7807C550108926C00208F6C0020105101080E
S3150800D79030510108985501087E010020736C00205D
S3150800D7A0D869002050510108405C0108800100201A
S3150800D7B0BC650108545C0108F4600108866C002009
S3150800D7C0C4650108856C0020CC650108FC63010866
S3150800D7D0386C0020086401083A6C002014640108BB
S3150800D7E03C6C0020206401083E6C00202C64010873
S3150800D7F03864010844640108786C0020876C0020AE
S3150800D800886C0020896C00208A6C00208B6C0020B4
S3150800D8108C6C002050640108685C01087D6C00204F
S3150800D8207C6C00207C5C01088D6C00208E6C0020CE
S3150800D8305C640108905C0108306C0020326C0020A2
S3150800D8407E6C00207F6C0020836C0020806C00209A
S3150800D850816C002004610108A0590108346C00207D
S3150800D860366C0020846C0020826C002001000020A9
S3150800D8700A0012B2842A03D00A0012B2D21C101867
S3150800D8807047EFF30580002801D0012000E0002052
S3150800D890C0B2704780B501F019FE002002BD38B548
S3150800D8A084B004000D006069002813D0A069002820
S3150800D8B010D0B4F90800FFF7D9FFA1690291616990
S3150800D8C0019100902B0022692168606801F08CFCA8
S3150800D8D0039011E0B4F90800FFF7C8FF03A9019106
S3150800D8E000902B00226992B22168606801F0CAFC98
S3150800D8F0012801D0002000E0039805B030BD38B5F6
S3150800D90005000120B5FBF0F4002C01D0200000E052
S3150800D910012001F0B4FD002032BD7CB505000E00E3
S3150800D920686800280CD0012E08D1032000906B6887
S3150800D93000220021012002F0EBFA14E0002012E098
S3150800D940012E0FD103220021012002F041FB040021
S3150800D950002C05D0002300220021200002F07FFBC6
S3150800D960200000E0002076BD7CB504000D000020F4
S3150800D9700090002C01D1802034E0002615F1010F1B
S3150800D98003D15FF0FF30060009E0002D07D0012023
S3150800D990B5FBF0F00600002E01D101200600FFF7C6
S3150800D9A070FF002815D06A460021200002F05EFDAF
S3150800D9B0012801D0FF2015E00098002811D05FF05B
S3150800D9C08050DFF878100860BFF34F8FBFF36F8F72
S3150800D9D007E03100200002F076FC012801D0FF2084
S3150800D9E000E0002076BD38B5040000250020009030
S3150800D9F0FFF747FF002814D06946200002F002FC12
S3150800DA00012801D0FF2017E00098002813D05FF006
S3150800DA108050DFF828100860BFF34F8FBFF36F8F71
S3150800DA2009E0002300220021200002F018FB01284B
S3150800DA3001D0FF200500280032BD000004ED00E0FB
S3150800DA4010B50400002C01D1012033E0A06900289C
S3150800DA50FFD194F83900002805D1002084F8380051
S3150800DA60200002F04FFE242084F839002068C068A0
S3150800DA7030F400502168C860200000F02DFA2068B4
S3150800DA80006930F49040216808612068406930F0E8
S3150800DA902A00216848612068C06850F4005021684F
S3150800DAA0C8600020E063202084F83900202084F82C
S3150800DAB03A00002010BD10B50400002C01D1012049
S3150800DAC017E0242084F839002068C06830F4005034
S3150800DAD02168C860200002F07EFF0020E063002075
S3150800DAE084F83900002084F83A00002084F83800C9
S3150800DAF0002010BD2DE9FC4706000D0017009846CA
S3150800DB00002496F8390020285DD1002D03D038006E
S3150800DB1080B2002801D1012056E096F83800012885
S3150800DB2001D1022050E0012086F838000020F06379
S3150800DB30212086F8390002F0BFFF8146B784F784B2
S3150800DB40B068B0F5805F05D13069002802D100249D
S3150800DB50AA4602E02C005FF0000A002086F838008A
S3150800DB60F08C00281ED0CDF800804B46002280217C
S3150800DB70300000F053F9002801D0032024E0002CDF
S3150800DB8008D1BAF80000C005C00D316848601AF11E
S3150800DB90020A03E0207831684860641CF08C401E55
S3150800DBA0F084DDE7CDF800804B46002240213000A6
S3150800DBB000F034F9002801D0032005E0202086F87B
S3150800DBC03900002000E00220BDE8F68773B504009E
S3150800DBD0150094F83A00202851D10198002803D05E
S3150800DBE0280080B2002801D1012049E094F83800C5
S3150800DBF0012801D1022043E0012084F83800019869
S3150800DC00A062A5850020E063222084F83A000FF27E
S3150800DC106110616B88620FF29D10616BC8620FF22A
S3150800DC20A510616B08630020616B486301AE2B0089
S3150800DC309BB232682068011D606B02F0D6FF002097
S3150800DC40009020680068009020684068009000985E
S3150800DC50002084F838002068C06850F48070216875
S3150800DC60C8602068406950F0010021684861206852
S3150800DC70406950F0400021684861002000E0022019
S3150800DC8076BD70B50600002031684C69E40914F0C9
S3150800DC90010496F83910212910D1002C0ED03068CD
S3150800DCA0406930F0800031684861306B002802D046
S3150800DCB0306B02F0E6FF300000F0E7F8306845699F
S3150800DCC0AD0915F0010596F83A00222810D1002D65
S3150800DCD00ED03068406930F0400031684861706B9A
S3150800DCE0002802D0706B02F0CCFF300000F0D7F8A5
S3150800DCF0002070BD10B504002068C06830F490702C
S3150800DD002168C86020684069400840002168486169
S3150800DD102068406940061FD52068406930F04000F9
S3150800DD2021684861606B00280DD00FF29510616B71
S3150800DD304863606B02F0CCFF002815D0606B616BFE
S3150800DD40496B884710E00020E085202084F83A00D7
S3150800DD50200003F09DFA07E00020E085202084F8E3
S3150800DD603A00200003F094FA002010BDC06B7047FB
S3150800DD7038B50400656A20680068800616D4002055
S3150800DD80E8852868C06830F480702968C860286803
S3150800DD90406940084000296848612868406930F0B1
S3150800DDA0400029684861202085F83A002800FDF7D8
S3150800DDB08DF931BD38B50400656A280003F069FAA3
S3150800DDC031BD0000F8B506000020776A39684C694D
S3150800DDD0E40914F0010497F83910212906D1002C1A
S3150800DDE004D00020F884380000F04FF838684569F8
S3150800DDF0AD0915F0010597F83A00222806D1002D3D
S3150800DE0004D00020F885380000F049F8F86B50F087
S3150800DE101000F8633800FDF77FF9F1BD2DE9F041F0
S3150800DE2005000E0090461F00069C286800683040D2
S3150800DE30B04201D1012000E000204146C9B2884223
S3150800DE4020D114F1010FF0D0002C04D002F034FEDA
S3150800DE50C01B8442E9D22868C06830F4D0702968AB
S3150800DE60C860286840694008400029684861202041
S3150800DE7085F83900202085F83A00002085F8380012
S3150800DE80032000E00020BDE8F0810168C96831F090
S3150800DE90C0010268D160202180F8391070470168F6
S3150800DEA0C96831F490710268D16001684969490806
S3150800DEB0490002685161202180F83A107047000035
S3150800DEC038B50400656A0020E885202085F83A0000
S3150800DED0280003F0DDF931BD70B50400206801693A
S3150800DEE031F44051E068014320680161A568206962
S3150800DEF00543606905432068C1682E4801402943E7
S3150800DF002068C1602068416931F44071A069014305
S3150800DF102068416120682849884202D103F0FAFC4A
S3150800DF2001E003F0ECFC192101FB00F162689200A4
S3150800DF30B1FBF2F16422B1FBF2F2192101FB00F107
S3150800DF4063689B00B1FBF3F3192101FB00F16668D6
S3150800DF50B600B1FBF6F16426B1FBF6F6642101FBC7
S3150800DF601633190132316423B1FBF3F313F0F003CE
S3150800DF7013EB0213192101FB00F162689200B1FB51
S3150800DF80F2F2192101FB00F16668B600B1FBF6F161
S3150800DF906426B1FBF6F6642101FB16221101323123
S3150800DFA06422B1FBF2F111F00F01CB1821688B60E6
S3150800DFB070BD0000F3E9FFFF0038014016B50022E6
S3150800DFC082B00446009201940A4603AB01A90848A8
S3150800DFD078441C3003F0E4FC019900220A700028FA
S3150800DFE04EBF04460198041B204604B010BD00BF6E
S3150800DFF083EAFFFF0CB430B583B0044606A8029046
S3150800E0000A4600250194009502AB01A90848784400
S3150800E0101E3003F0C5FC01990D7000284EBF04465A
S3150800E0200198041B204603B030BC5DF80CFB00BF0A
S3150800E03043EAFFFF38B504000D0002216548FEF7E4
S3150800E04093FB65480078002803D021786348FCF7DD
S3150800E05083FD63480078002803D15CA0FCF77CFDAB
S3150800E06002E05BA0FCF778FD2900C9B2200000F0A9
S3150800E070C6FC31BDF8B504000D005A4800780028E2
S3150800E08013D000265848FCF767FD00273800C0B2B1
S3150800E090A84207DA3800C0B2215C5448FCF75CFD98
S3150800E0A07F1CF3E749A0FCF757FD2800010089B259
S3150800E0B02000FCF76CFEF1BD38B504000D0046489B
S3150800E0C00078002803D021784948FCF745FD280048
S3150800E0D0020092B221004748006804F095FB31BD62
S3150800E0E038B504000D002A0021004248006804F0F3
S3150800E0F001FC31BD38B504000D003748007800280A
S3150800E10003D021783548FCF727FD354800780028E4
S3150800E11003D12EA0FCF720FD02E02DA0FCF71CFD84
S3150800E1202900C9B2200000F0EBF831BDF8B50400AB
S3150800E1300D002C480078002813D000262E48FCF73E
S3150800E1400BFD00273800C0B2A84207DA3800C0B273
S3150800E150215C2648FCF700FD7F1CF3E71BA0FCF7B3
S3150800E160FBFC2800010089B22000FCF77EFFF1BD08
S3150800E17038B504000D0018480078002803D0217827
S3150800E1801E48FCF7E9FC2800020092B221001C4850
S3150800E190006804F039FB31BD38B504000D002A00CB
S3150800E1A021001748006804F0A5FB31BD80B5154B62
S3150800E1B0154A00210F48006804F004FB134B144A63
S3150800E1C000210F48006804F0FDFA01BD0D0A0000A1
S3150800E1D02C200000001001407C010020A45C0108EE
S3150800E1E07D0100206D6C0020B85C01086864010898
S3150800E1F07051010868010020CC5C0108B45501087B
S3150800E2006C01002075E0000835E000082DE10008E3
S3150800E210F5E0000801000800C0B230286BD00800FD
S3150800E220C0B2322867D00800C0B2342863D00800CC
S3150800E230C0B238285FD00800C0B220285BD00800DA
S3150800E240C0B2222857D00800C0B2242853D00800EC
S3150800E250C0B225284FD00800C0B22C284BD00800E1
S3150800E260C0B22A2847D00800C0B22B2843D00800DD
S3150800E270C0B241283FD00800C0B244283BD00800AD
S3150800E280C0B2472837D00800C0B2622833D0080089
S3150800E290C0B264282FD00800C0B266282BD0080068
S3150800E2A0C0B2682827D00800C0B26A2823D0080060
S3150800E2B0C0B26C281FD00800C0B2F0281BD00800D6
S3150800E2C0C0B2F12817D00800C0B2F22813D008004F
S3150800E2D0C0B2F3280FD00800C0B2F4280BD008004B
S3150800E2E0C0B2F52807D00800C0B23B2803D0080002
S3150800E2F0C0B23D2801D1012000E00020704700008F
S3150800E3002DE9F04704000D002078FFF783FF002869
S3150800E31000F073830421DFF8C007FEF725FA20789A
S3150800E320202800F07681222800F09F81242800F01A
S3150800E330A881252800F0B1812A2800F0D6812B284B
S3150800E34000F0EA812C2800F0BC81302831D0322830
S3150800E3503BD0342845D0382800F04F813B2800F0C0
S3150800E36034833D2800F03B83412800F0E3814428AC
S3150800E37000F0F581472800F00782622800F0108235
S3150800E380642800F01982662800F05882682800F090
S3150800E39076826A2800F093826C2800F0AD82F02815
S3150800E3A000F0DF82F32800F0EA82F52800F0068301
S3150800E3B01FE3DFF828070078002803D0DFF82007D6
S3150800E3C0FCF7CAFBFDF75DFA17E3DFF810070078DC
S3150800E3D0002803D0DFF80C07FCF7BEFBFDF706FCA8
S3150800E3E00BE3DFF8F806007800281ED0DFF8F806F9
S3150800E3F0FCF7B2FB6178DFF8F406FCF7ADFBA17811
S3150800E400DFF8E806FCF7A8FB2800C0B2042805DBFD
S3150800E410E178DFF8D806FCF79FFB03E0DFF8D006C3
S3150800E420FCF79AFBC2A0FCF797FBF4F781FE0028DD
S3150800E43002D0FDF732FBE0E2607800285FD0DFF813
S3150800E440B4060078002833D10020DFF8AC1608801F
S3150800E4500020DFF8A81608800020DFF8A416088038
S3150800E4600020DFF8A01608800020DFF89C16088038
S3150800E4700020DFF8981608800020DFF89416088038
S3150800E4800020DFF89016088020260027DFF8888607
S3150800E4903A0031004046FEF799F95FF020085FF030
S3150800E4A00009DFF878A64A4641465046FEF78EF937
S3150800E4B0DFF86C06007800281CD10020DFF8641607
S3150800E4C008800020DFF8601608800020DFF85C1658
S3150800E4D008800020DFF8581608800020DFF8541658
S3150800E4E0088020260027DFF850863A00310040468B
S3150800E4F0FEF76CF90120DFF84416087003E00120E6
S3150800E500DFF83C160870A07800285FD0DFF8E4052D
S3150800E5100078002833D10020DFF8DC1508800020B9
S3150800E520DFF8D81508800020DFF8D4150880002009
S3150800E530DFF8D01508800020DFF8CC150880002009
S3150800E540DFF8C81508800020DFF8C4150880002009
S3150800E550DFF8C015088020260027DFF8BC853A00BA
S3150800E56031004046FEF732F95FF020085FF00009F7
S3150800E570DFF8A8A54A4641465046FEF727F9DFF8D0
S3150800E580A005007800281CD10020DFF8981508801F
S3150800E5900020DFF8941508800020DFF89015088021
S3150800E5A00020DFF88C1508800020DFF88815088021
S3150800E5B020260027DFF880853A0031004046FEF71E
S3150800E5C005F90120DFF87C15087003E00120DFF863
S3150800E5D0781508702800C0B204280BDBE0780028FC
S3150800E5E004D00120DFF86415087003E00120DFF885
S3150800E5F060150870FDF72CFBFFE1DFF8E0040078F2
S3150800E600002803D0DFF84C05FCF7A6FAFDF729FB2E
S3150800E610F3E1DFF8C8040078002803D0DFF83805EE
S3150800E620FCF79AFADFF834050078012803D10020B0
S3150800E630FDF77EF918E06078DFF824150870A078F1
S3150800E64000280ED0A07810280BDAA078DFF8141569
S3150800E65008700120DFF8041508700120FDF768F935
S3150800E66002E00020FDF764F9C7E1DFF870040078DE
S3150800E670002803D0DFF8F004FCF76EFAFCF724FF55
S3150800E680BBE1DFF858040078002803D0DFF8DC0483
S3150800E690FCF762FAFDF79AF8AFE1DFF84004007874
S3150800E6A0002803D0DFF8C804FCF756FA6078DFF8CC
S3150800E6B0C41408700120DFF8C0140870FDF76EFB5B
S3150800E6C09BE1DFF818040078002803D0DFF8AC04D3
S3150800E6D0FCF742FADFF8A8040078002802D1FDF713
S3150800E6E0A8F901E0FCF786FD87E1DFF8F00300787A
S3150800E6F0002803D0DFF88C04FCF72EFADFF8F403C1
S3150800E7000078002804D10120DFF87C14087002E0A4
S3150800E7100220FDF71CF970E1DFF8C0030078002835
S3150800E72003D0DFF86804FCF717FAFDF740FB64E14D
S3150800E7300D0A0000DFF8A4030078002803D0DFF8EC
S3150800E7405004FCF709FADFF84C040078FF2803D0D8
S3150800E7500120DFF844140870FDF737FB4DE1DFF8B8
S3150800E7607C030078002803D0DFF83004FCF7F4F9BE
S3150800E770DFF820040078FF2803D00120DFF82014F2
S3150800E7800870FDF73FFB38E1DFF8500300780028F2
S3150800E79003D0DFF81004FCF7DFF9FDF74FFB2CE197
S3150800E7A0DFF838030078002803D0DFF8FC03FCF70D
S3150800E7B0D3F9FDF761FB20E1DFF8F00300780028C4
S3150800E7C00CD1DFF818030078002803D0DFF8E0033F
S3150800E7D0FCF7C2F90220FDF761FC0EE16078DFF86C
S3150800E7E0D4130880DFF8CC030088A17850EA01200A
S3150800E7F0DFF8C0130880E078DFF8BC130880DFF87C
S3150800E800B8030088217950EA0120DFF8AC130880A4
S3150800E8100120DFF8A8130870B0480078002809D04E
S3150800E820DFF894030288DFF88C030188DFF8900389
S3150800E830FCF792F90120FDF731FCDEE0DFF86C0306
S3150800E840007800280BD1A5480078002803D0DFF807
S3150800E8506003FCF781F90220FDF734FCCDE09F4800
S3150800E8600078002803D0DFF85C03FCF775F901206F
S3150800E870DFF8541308700120FDF724FCBDE0DFF82B
S3150800E8802C03007800280BD194480078002803D080
S3150800E890DFF81C03FCF760F90220FDF729FCACE061
S3150800E8A08E480078002803D0DFF82003FCF754F9D7
S3150800E8B00120C74908700120FDF71AFC9DE0BB48F6
S3150800E8C0007800280AD185480078002802D0B84880
S3150800E8D0FCF742F90220FDF723FC8EE07F4800781A
S3150800E8E0002802D0BB48FCF737F90120BA4908705E
S3150800E8F00120FDF715FC80E0B848007800280AD109
S3150800E90076480078002802D0B548FCF725F9022099
S3150800E910FDF71CFC71E06078B2490880B1480088B0
S3150800E920A17850EA0120AF490880E078AE4908800E
S3150800E930AD480088217950EA0120AB4908800120BA
S3150800E940AA49087065480078002806D0A6480288B3
S3150800E950A4480188A648FCF7FFF80120FDF7F6FB56
S3150800E9604BE0A448FCF7F8F86078FDF717FC6078E8
S3150800E970002803D10120A0490870FFE73DE09F4821
S3150800E980FCF7EAF8A078E17851EA002189B29C48B8
S3150800E99001602079617951EA002189B299480160BC
S3150800E9A0A0799949087098480678E71DDFF85C82CF
S3150800E9B0320039004046FEF709F81EE09448FCF795
S3150800E9C0CBF801209349087017E0444800780028DE
S3150800E9D002D09148FCF7C0F8FDF712FC0DE03F485D
S3150800E9E00078002802D08D48FCF7B6F8FDF74CFCF5
S3150800E9F003E021788A48FCF7AFF8BDE8F08770B5E0
S3150800EA0004000D002078FFF705FC012862D02900D4
S3150800EA10C9B289B22000FCF784FA2078401E09D0D2
S3150800EA20C01E50D0401E38D00A3820D0801E02287A
S3150800EA3049D94BE07B48FCF78FF87B4881787B48BF
S3150800EA4004F05DF87848C178784804F05EF87849AB
S3150800EA50764804F00BF8764804F04DF8060074483A
S3150800EA6004F047F8B6B23100FFF726FB32E07148EA
S3150800EA70FCF772F80120704908706D496E4804F079
S3150800EA8015F86B4804F037F80600694804F031F8C1
S3150800EA90B6B23100FFF710FB1CE06848FCF75CF8DB
S3150800EAA0FEF74CF8FEF762F8614804F013F8604880
S3150800EAB004F021F806005E4804F01BF8B6B23100EF
S3150800EAC0FFF7FAFA06E05E48FCF746F821785D4853
S3150800EAD0FCF742F870BD0000001001407D010020DF
S3150800EAE090510108584D0108804D0108D465010868
S3150800EAF0DC6501088F6C0020406C0020426C002009
S3150800EB00446C0020466C0020486C00204A6C0020AB
S3150800EB104C6C00204E6C0020F8690020186A002012
S3150800EB20906C0020506C0020526C0020546C002021
S3150800EB30566C0020586C0020386A0020876C00202C
S3150800EB408A6C0020886C00208B6C0020896C002061
S3150800EB508C6C002060490108FC4B0108796C002088
S3150800EB607A6C00207B6C0020904901088C470108CC
S3150800EB70A84D01087D6C00207C6C0020C049010866
S3150800EB80956C0020284C0108786C002094440108F4
S3150800EB90544C0108800100208D6C0020F0490108C2
S3150800EBA08E6C002074460108C0470108916C00204D
S3150800EBB0204A0108306C0020326C00207E6C002050
S3150800EBC0504A0108804A01087F6C0020B04A0108B3
S3150800EBD0806C0020E04A0108836C00209D6C0020B0
S3150800EBE0F4470108346C0020366C0020846C002041
S3150800EBF028480108D04401089F6C0020104B0108E2
S3150800EC00B86B0020BC6B0020A26C0020B068002006
S3150800EC10404B0108A06C0020D04D0108F84D0108B2
S3150800EC20304F0108B051010800F80B082C6C002081
S3150800EC30745D0020D05101086E6C0020D055010883
S3150800EC40544F0108F05101080100002070470100E7
S3150800EC500020704780B5DFF8F004FFF74BF8DFF8BF
S3150800EC60E804FFF70EF8DFF8E004FEF724FF01BD1D
S3150800EC7080B500F059F9FBF760FF01BD80B5DFF8F4
S3150800EC80CC04FFF737F8DFF8C404FEF7FAFFDFF81D
S3150800EC90BC04FEF710FF01BD80B500F089F9FCF74A
S3150800ECA018F801BD80B5DFF8A804FFF723F8DFF8E8
S3150800ECB0A004FEF7E6FFDFF89804FEF7FCFE01BDA8
S3150800ECC080B500F00FF9FCF7F5F901BD2DE9F84F0D
S3150800ECD0AAB0DFF88004DFF88014086062B603F093
S3150800ECE019FF00F0B5F800F0C0F900F084F900F05B
S3150800ECF0E6F800F019F900F039F900F059F900F0D2
S3150800ED00F1F8FBF71AFFFBF7E4FFFFF74FFAFCF7FA
S3150800ED10D1F900208DF8000003221021DFF83C0409
S3150800ED2003F00CFF040000208DF8000003221121D7
S3150800ED30DFF82C0403F002FF05005FF0000B032246
S3150800ED401421DFF8200403F0F9FE06005FF0000A3C
S3150800ED5003221021DFF8100403F0F0FE07005FF02D
S3150800ED60000903221821DFF8040403F0E7FE8046B1
S3150800ED70DFF8FC23D2E90001CDE90501012105A848
S3150800ED80FEF7CBFDDFF8EC130860DFF8EC23D2E9D9
S3150800ED900001CDE90301012103A8FEF7BEFDDFF856
S3150800EDA0DC130860DFF8D823D2E90001CDE90101B8
S3150800EDB0012101A8FEF7B1FDDFF8C813086023A8F2
S3150800EDC0DFF8C4131C22FDF711FE2100C9B223A8DF
S3150800EDD0FEF765FDDFF8B41308601CA8DFF8B0136A
S3150800EDE01C22FDF703FE2900C9B21CA8FEF757FD31
S3150800EDF0DFF8A013086015A8DFF89C131C22FDF79E
S3150800EE00F5FD3100C9B215A8FEF749FDDFF88C13E8
S3150800EE1008600EA8DFF888131C22FDF7E7FD390005
S3150800EE20C9B20EA8FEF73BFDDFF87813086007A8FD
S3150800EE30DFF874131C22FDF7D9FD4146C9B207A8AD
S3150800EE40FEF72DFDDFF864130860FEF723FDFEE7E5
S3150800EE5000B58FB005A8282103F082FF6846142163
S3150800EE6003F07EFF092005905FF4803006900020AD
S3150800EE7007900120099001200B9002200C905FF466
S3150800EE8080300D9000200E9005A802F003FA0028A5
S3150800EE9001D000F0A7F90F20009002200190002071
S3150800EEA0029000200390002004900121684602F099
S3150800EEB032FC002801D000F095F90FB000BD80B5EE
S3150800EEC0BB48BC4908600520BA49486040F2AA30E8
S3150800EED0B8498860B74803F046FF002801D000F01B
S3150800EEE081F901BD80B5B448994908605FF4E130FD
S3150800EEF09749486000209649886000209449C86070
S3150800EF000020934908610C209149486100209049E6
S3150800EF10886100208E49C8618D48FEF791FD00285A
S3150800EF2001D000F05FF901BD80B5A44886490860A4
S3150800EF305FF4E130844948600020834988600020F6
S3150800EF408149C8600020804908610C207E494861D3
S3150800EF5000207D49886100207B49C8617A48FEF710
S3150800EF606FFD002801D000F03DF901BD80B5944839
S3150800EF70944908605FF4E13092494860002091495D
S3150800EF80886000208F49C86000208E4908610C20DF
S3150800EF908C49486100208B49886100208949C861ED
S3150800EFA08848FEF74DFD002801D000F01BF901BD89
S3150800EFB080B58548654908604FF41650634948602E
S3150800EFC04FF480506149886000206049C86000207D
S3150800EFD05E4908610C205D49486100205B498861EB
S3150800EFE000205A49C8615948FEF72AFD002801D071
S3150800EFF000F0F8F801BD80B57448006850F00100CB
S3150800F000724908607148006810F001000090009885
S3150800F0106E48006850F002006C4908606B4800684A
S3150800F02010F0020000900098002205210D2003F040
S3150800F03045FF0D2003F057FF002205210F2003F09E
S3150800F0403DFF0F2003F04FFF00220521102003F09B
S3150800F05035FF102003F047FF002205213A2003F070
S3150800F0602DFF3A2003F03FFF01BD00B585B001A88A
S3150800F070102103F075FE5648006850F020005449E8
S3150800F08008605348006810F0200000900098504827
S3150800F090006850F010004E4908604D48006810F0AE
S3150800F0A01000009000984A48006850F0040048494B
S3150800F0B008604748006810F004000090009844482B
S3150800F0C0006850F00800424908604148006810F09E
S3150800F0D008000090009800220F213E48FDF737FBF4
S3150800F0E001224FF480513C48FDF731FB0F20019077
S3150800F0F001200290002003900320049001A93548BE
S3150800F100FDF760F94FF4805001900120029000202D
S3150800F11003900320049001A92F48FDF753F905B081
S3150800F12000BD38B5040025002C492D48FBF714FD11
S3150800F13003F0B4FD2800C0B203F08FFD4FF47A70D7
S3150800F140FEF7DDFBF4E70000F0670020706800209A
S3150800F150B06700200030000808ED00E0E05C010818
S3150800F160F45C0108B8590108085D0108EC55010866
S3150800F170EC650108A46B0020F4650108A86B002063
S3150800F180FC650108AC6B002008560108906B00204E
S3150800F19024560108946B002040560108986B0020FD
S3150800F1A05C5601089C6B002078560108A06B00206D
S3150800F1B0003000404C6B0020004C004000380140F5
S3150800F1C00044004030680020004800401410024007
S3150800F1D01810024000100140000C0140E4650108C7
S3150800F1E01C5D0108704768002DE9F04F85B00600E0
S3150800F1F00F0090469946DDF838A00F9C109D002C0C
S3150800F20007D1502080F31188BFF34F8FBFF36F8F5C
S3150800F210FEE7002D07D1502080F31188BFF34F8FEA
S3150800F220BFF36F8FFEE7542000900098542807D04C
S3150800F230502080F31188BFF34F8FBFF36F8FFEE71F
S3150800F240002D19D0002C17D0AB46CBF83040022041
S3150800F2508BF8510000200390CDF808B004A801905F
S3150800F260CDF800A04B4642463900300000F047F87A
S3150800F270584600F0A7F801E000200490049805B06D
S3150800F280BDE8F08F2DE9F84F84B006000F009046D0
S3150800F2909946DDF838A0DDF83CB0404680B28000DB
S3150800F2A003F03EFE0500002D0BD0542003F038FE77
S3150800F2B00400002C01D0256304E0280003F0BDFEFD
S3150800F2C000E00024002C15D0002084F8510000200E
S3150800F2D003900294CDF804B0CDF800A04B46424600
S3150800F2E092B23900300000F00AF8200000F06AF8FF
S3150800F2F0012001E05FF0FF3005B0BDE8F08F2DE991
S3150800F300F84F05000E0017009846DDF828900B9C6C
S3150800F310DDF830A0DAF8300000EB8700001FC008DF
S3150800F320C0000090009810F0070F07D0502080F317
S3150800F3301188BFF34F8FBFF36F8FFEE75FF0000BA7
S3150800F340BBF1100F0CD216F80B000AEB0B0181F873
S3150800F350340016F80B00002802D01BF1010BEFE76A
S3150800F36000208AF84300B9F1070F01D30620814629
S3150800F370CAF82C90CAF844900020CAF848001AF136
S3150800F380040003F018FF1AF1180003F014FFCAF876
S3150800F39010A0D9F10700CAF81800CAF824A000205E
S3150800F3A0CAF84C0000208AF8500042462900009806
S3150800F3B003F040FFCAF80000002C01D0C4F800A0F2
S3150800F3C0BDE8F18F10B5040003F0AAFFDFF8F004DA
S3150800F3D00068401CDFF8E8140860DFF8E8040068F5
S3150800F3E000280AD1DFF8DC040460DFF8D4040068DA
S3150800F3F0012811D100F0DCFA0EE0DFF8CC04006831
S3150800F400002809D1E06ADFF8BC140968C96A88428D
S3150800F41002D3DFF8B0040460DFF8B0040068401CCB
S3150800F420DFF8A8140860DFF8BC0401680122E06A66
S3150800F43082401143DFF8AC040160211DDFF8A824DF
S3150800F440E36A1420434302EB030003F0B7FE03F01C
S3150800F45084FFDFF87404006800280FD0DFF864041E
S3150800F4600068C06AE16A884208D25FF08050DFF817
S3150800F47054160860BFF34F8FBFF36F8F10BD38B5B2
S3150800F48005000024002D15D0DFF8200500680028A7
S3150800F49007D0502080F31188BFF34F8FBFF36F8FCB
S3150800F4A0FEE700F05DF80021280000F085FC00F07A
S3150800F4B05FF80400002C08D15FF08050DFF80416CE
S3150800F4C00860BFF34F8FBFF36F8F31BD10B586B09D
S3150800F4D0002004900020039005AA03A904A803F0BD
S3150800F4E0BDFF049802900398019000200090002325
S3150800F4F0059ADFF89C180FF28D40FFF775FEDFF8C6
S3150800F50094180860DFF88C080068002801D00124E8
S3150800F51000E00024012C16D1502080F31188BFF397
S3150800F5204F8FBFF36F8F5FF0FF30DFF86C180860FE
S3150800F5300120DFF8941308600020DFF860180860DF
S3150800F54003F09DFE0AE014F1010F07D1502080F365
S3150800F5501188BFF34F8FBFF36F8FFEE706B010BD5C
S3150800F560DFF848040068401CDFF84014086070475C
S3150800F57070B500250026DFF834040068002807D196
S3150800F580502080F31188BFF34F8FBFF36F8FFEE7CC
S3150800F59003F0C6FEDFF814040068401EDFF80C14FA
S3150800F5A00860DFF80804006800285DD1DFF810035A
S3150800F5B00068002858D0DFF8D407006800282BD048
S3150800F5C0DFF8C807C068C068050015F1180003F021
S3150800F5D01CFE281D03F019FEDFF808030168012246
S3150800F5E0E86A82401143DFF8FC020160291DDFF852
S3150800F5F0F822EB6A1420434302EB030003F0DEFD16
S3150800F600E86ADFF8C0120968C96A8842D3D30120BC
S3150800F610DFF88C170860CEE7002D01D000F03BFA22
S3150800F620DFF880070468002C0ED000F021F80028C7
S3150800F63003D00120DFF868170860641E002CF4D197
S3150800F6400020DFF860170860DFF854070068002814
S3150800F6500AD0012006005FF08050DFF868140860C1
S3150800F660BFF34F8FBFF36F8F03F077FE300070BD87
S3150800F6702DE9F0410027DFF83403006800287CD123
S3150800F680DFF818070468641CDFF810070460002C0C
S3150800F69024D1DFF8140700680068002807D0502036
S3150800F6A080F31188BFF34F8FBFF36F8FFEE7DFF844
S3150800F6B0F806D0F80080DFF8F4060068DFF8E816E8
S3150800F6C00860DFF8E806C0F80080DFF8E40600689E
S3150800F6D0401CDFF8DC16086000F0DDF9DFF8B80634
S3150800F6E0006884423DD3DFF8C00600680068002839
S3150800F6F005D15FF0FF30DFF8A016086031E0DFF8CB
S3150800F700A8060068C068C068050068680600B442B4
S3150800F71003D2DFF88406066023E0281D03F075FD92
S3150800F720A86A002803D015F1180003F06EFD6D488D
S3150800F73001680122E86A824011436A480160291D6E
S3150800F740694AEB6A1420434302EB030003F036FDD3
S3150800F750E86A5C490968C96A8842C4D30120070077
S3150800F760C1E7584800686049C26A1420424388586D
S3150800F770022809D30120070006E0DFF828060068FA
S3150800F780401CDFF820160860DFF814060068002819
S3150800F79001D0012007003800BDE8F08183480068E1
S3150800F7A0002804D00120DFF8F81508602CE00020B6
S3150800F7B0DFF8EC1508604B480068B0FA80F1D1F123
S3150800F7C01F014948142202FB01F28058002807D17C
S3150800F7D0502080F31188BFF34F8FBFF36F8FFEE77A
S3150800F7E04148142202FB01F2104442685268426002
S3150800F7F0426810F108039A4202D142685268426090
S3150800F8004068C0682F4A1060704738B504000D007C
S3150800F810002C07D1502080F31188BFF34F8FBFF318
S3150800F8206F8FFEE7DFF81006006810F11801200058
S3150800F83003F0D0FC0121280000F0BEFA31BD38B52E
S3150800F8400500E868C468002C07D1502080F31188A9
S3150800F850BFF34F8FBFF36F8FFEE714F1180003F065
S3150800F860D4FC52480068002814D1201D03F0CDFCB2
S3150800F8701C4801680122E06A824011431948016068
S3150800F880211D194AE36A1420434302EB030003F0DF
S3150800F89095FC05E014F11801DFF8F00403F08EFC7E
S3150800F8A008480068C06AE16A884205D20120012139
S3150800F8B0DFF80025116000E0002032BD00000000DE
S3150800F8C0F86B0020E86B0020046C0020146C002004
S3150800F8D0DFF8DC1409680160DFF860150968416023
S3150800F8E070470000006C0020386400202DE9F041C4
S3150800F8F004000D00002C07D1502080F31188BFF3B7
S3150800F9004F8FBFF36F8FFEE7002D07D1502080F38E
S3150800F9101188BFF34F8FBFF36F8FFEE703F000FD2B
S3150800F920DFF8780406686768F71B286810F1010F86
S3150800F93002D15FF000081BE0DFF874040068216854
S3150800F940884205D06068864202D35FF001080FE05E
S3150800F9502868874208D22868C01B28602000FFF75D
S3150800F960B7FF5FF0000803E0002028605FF0010899
S3150800F97003F0F3FC4046BDE8F0810120DFF83414BB
S3150800F9800860704710B5040000F03EF8DFF8B004D0
S3150800F99000680228F8D35FF08050DFF8A8140860E2
S3150800F9A0BFF34F8FBFF36F8FEEE70000206C002088
S3150800F9B010B50024072C09D2DFF88404142101FBB2
S3150800F9C004F1084403F0E8FB641CF3E7DFF8780465
S3150800F9D003F0E2FBDFF8740403F0DEFBDFF8AC03A8
S3150800F9E003F0DAFBDFF8680403F0D6FB714803F08E
S3150800F9F0D3FBDFF85404DFF8B0130860DFF84C04D3
S3150800FA00DFF85014086010BD10B5DFF84C04006824
S3150800FA1000281DD003F084FCDFF83404C068C068F1
S3150800FA200400201D03F0F1FBDFF830040068401ED7
S3150800FA30DFF828140860DFF820040068401EDFF8A5
S3150800FA401814086003F089FC200000F002F8DCE7CF
S3150800FA5010BD10B5040094F85100002806D1206B9B
S3150800FA6003F0EBFA200003F0E8FA13E094F85100EB
S3150800FA70012803D1200003F0E0FA0BE094F85100C6
S3150800FA80022807D0502080F31188BFF34F8FBFF3A9
S3150800FA906F8FFEE710BDDFF81003006800680028C6
S3150800FAA005D15FF0FF30DFF8F022106009E0DFF8DB
S3150800FAB0F8020068C068C06801004868DFF8D82204
S3150800FAC01060704704ED00E0DFF894030068002832
S3150800FAD001D1012007E0DFF88C030068002801D176
S3150800FAE0022000E00020704770B5040025000026BB
S3150800FAF0002C5CD0E86ADFF840130968C96A8842B6
S3150800FB004CD2A869002806D4DFF82C030068C06A1E
S3150800FB10D0F10700A8616969DFF82423EB6A14208D
S3150800FB20434302EB0300814230D1281D03F06DFBED
S3150800FB30002811D1DFF80813EA6A142042438858CE
S3150800FB40002809D1DFF8200301680122E86A82400B
S3150800FB509143DFF814030160DFF8DC020068C06A2D
S3150800FB60E862DFF8040301680122E86A824011436B
S3150800FB70DFF8F4020160291DDFF8C422EB6A1420BD
S3150800FB80434302EB030003F019FB04E0DFF8A80285
S3150800FB900068C06AE8620120060008E0686CDFF8C1
S3150800FBA098120968C96A884201D201200600300005
S3150800FBB070BD0000A86A002070B504002500002664
S3150800FBC0002C54D0DFF870020068854207D0502018
S3150800FBD080F31188BFF34F8FBFF36F8FFEE7A86CD2
S3150800FBE0002807D1502080F31188BFF34F8FBFF349
S3150800FBF06F8FFEE7A86C401EA864E86A696C8842A5
S3150800FC0035D0A86C002832D1281D03F0FEFA00284A
S3150800FC1011D1DFF82C12EA6A1420424388580028CA
S3150800FC2009D1DFF8440201680122E86A824091435B
S3150800FC30DFF834020160686CE862E86AD0F1070010
S3150800FC40A861DFF8240201680122E86A82401143AC
S3150800FC50DFF814020160291DDFF8E421EB6A14209D
S3150800FC60434302EB030003F0A9FA01200600300023
S3150800FC7070BD00002DE9F84304000F00A0465FF0B0
S3150800FC800109002C71D0D8F84800002807D1502067
S3150800FC9080F31188BFF34F8FBFF36F8FFEE7D8F855
S3150800FCA04400B84201D23E0002E0D8F844000600FB
S3150800FCB0D8F82C00B04258D0D8F84800484554D156
S3150800FCC0DFF874010068804507D1502080F3118859
S3150800FCD0BFF34F8FBFF36F8FFEE7D8F82C000500F0
S3150800FCE0C8F82C60D8F81800002803D4D6F1070005
S3150800FCF0C8F81800D8F81400DFF84411142202FBDB
S3150800FD0005F21144884230D118F1040003F07DFA57
S3150800FD10002813D1DFF82811D8F82C2014204243E4
S3150800FD20885800280AD1DFF8400101680122D8F86E
S3150800FD302C0082409143DFF830010160DFF828018A
S3150800FD4001680122D8F82C0082401143DFF8180117
S3150800FD50016018F10401DFF8E820D8F82C301420E7
S3150800FD60434302EB030003F029FABDE8F183DFF809
S3150800FD70C8000068002805D0DFF8BC000068816C60
S3150800FD80491C8164DFF8B00000687047806A00206B
S3150800FD90A46601081C6C0020186C0020FC6B00206F
S3150800FDA00C6C0020086C0020EC6B0020F06B002027
S3150800FDB0106C00200C6C0020F8B505000C001F48DC
S3150800FDC007681D480068001D03F01FFA002809D1BE
S3150800FDD019480068244909680122C06A824091438B
S3150800FDE02148016015F1010F08D1002C06D01248F0
S3150800FDF00068011D1D4803F0E1F91BE0E81906003B
S3150800FE000D4800684660BE4207D20B480068011DCF
S3150800FE101048006803F0DEF90CE007480068011D89
S3150800FE201348006803F0D6F912480068864201D2E2
S3150800FE3010480660F1BD0000E86B0020FC6B00204E
S3150800FE403864002004ED00E0586A00206C6A00203F
S3150800FE50946A0020F06B0020F46B0020F86B0020F9
S3150800FE60046C0020206C0020006C0020A86A00208A
S3150800FE70EC6B0020186C002070B506000C003500ED
S3150800FE80002D07D1502080F31188BFF34F8FBFF3A1
S3150800FE906F8FFEE703F044FA2968EA6B286C424341
S3150800FEA001EB020068600020A8632868A86029683A
S3150800FEB0EA6B521E286C424301EB0200E8605FF0D1
S3150800FEC0FF3085F844005FF0FF3085F84500002CC8
S3150800FED012D12869002817D015F11000FFF7AFFCDA
S3150800FEE0002811D05FF08050DFF87C150860BFF35A
S3150800FEF04F8FBFF36F8F07E015F1100003F04CF931
S3150800FF0015F1240003F048F903F027FA012070BD23
S3150800FF102DE9F84306000C0015001F00DDF82090B7
S3150800FF20002E07D1502080F31188BFF34F8FBFF3FF
S3150800FF306F8FFEE7002F07D1502080F31188BFF39B
S3150800FF404F8FBFF36F8FFEE7002D01D0002C01D035
S3150800FF50012000E00020C0B2002807D1502080F31D
S3150800FF601188BFF34F8FBFF36F8FFEE7002D01D1C6
S3150800FF70002C01D1012000E00020C0B2002807D1E2
S3150800FF80502080F31188BFF34F8FBFF36F8FFEE7C2
S3150800FF90482000900098482807D0502080F3118800
S3150800FFA0BFF34F8FBFF36F8FFEE7B846B8F1000F68
S3150800FFB00BD0012088F84600CDF800804B46DBB20E
S3150800FFC02A002100300000F031F84046BDE8F283EF
S3150800FFD02DE9F84304000D001700002C07D1502026
S3150800FFE080F31188BFF34F8FBFF36F8FFEE7002DA5
S3150800FFF002D15FF0000901E005FB04F919F1480098
S3150801000002F08EFF0600002E0DD016F1480080463C
S31508010010002086F8460000963B00DBB242462900DE
S31508010020200000F003F83000BDE8F2832DE9F04125
S3150801003005000C0016001F00DDF81880002C02D1FF
S31508010040C8F8008001E0C8F80060C8F83C50C8F854
S31508010050404001214046FFF70FFFBDE8F0812DE939
S31508010060F74380460D00994600244646002E07D1DF
S31508010070502080F31188BFF34F8FBFF36F8FFEE7D0
S31508010080002D02D1306C002801D1012000E00020AA
S31508010090C0B2002807D1502080F31188BFF34F8FD3
S315080100A0BFF36F8FFEE7B9F1020F02D1F06B01289A
S315080100B001D1012000E00020C0B2002807D150205C
S315080100C080F31188BFF34F8FBFF36F8FFEE7FFF7FA
S315080100D0FBFC002802D10298002801D1012000E08A
S315080100E00020C0B2002807D1502080F31188BFF341
S315080100F04F8FBFF36F8FFEE703F012F9B06BF16B09
S31508010100884202D3B9F1020F27D14A4629003000A5
S3150801011000F00EFA0700706A00280FD016F12400C5
S31508010120FFF78DFB002814D05FF08050DFF83813F5
S315080101300860BFF34F8FBFF36F8F0AE0002F08D017
S315080101405FF08050DFF820130860BFF34F8FBFF3CD
S315080101506F8F03F002F9012052E00298002803D1BB
S3150801016003F0FBF800204BE0002C04D16846FFF7AA
S31508010170AFFB0120040003F0F0F8FFF7F1F903F0F3
S31508010180CFF896F9440010F1010F02D1002086F844
S31508010190440096F9450010F1010F02D1002086F8B6
S315080101A0450003F0DAF802A96846FFF79FFB002825
S315080101B020D1300000F067FA002815D0029916F10F
S315080101C01000FFF722FB300000F016FAFFF7D0F90E
S315080101D0002891D15FF08050DFF88C120860BFF3D8
S315080101E04F8FBFF36F8F87E7300000F005FAFFF7EF
S315080101F0BFF981E7300000F0FFF9FFF7B9F90020F0
S31508010200BDE8FE832DE9F84306000C003500002DF4
S3150801021007D1502080F31188BFF34F8FBFF36F8F3B
S31508010220FEE7286C002807D0502080F31188BFF319
S315080102304F8FBFF36F8FFEE72868002802D16868E1
S31508010240002801D1012000E00020C0B2002807D112
S31508010250502080F31188BFF34F8FBFF36F8FFEE7EE
S3150801026003F0A8F8EFF31187502080F31188BFF344
S315080102704F8FBFF36F8FD5F83880E86B80451DD255
S3150801028095F9459018F10100A863484640B210F166
S31508010290010F0DD1686A00280ED015F12400FFF769
S315080102A0CEFA002808D0002C06D00120206003E0F1
S315080102B019F1010085F84500012000E0002087F3C7
S315080102C01188BDE8F2832DE9F34182B08046002406
S315080102D047460025002F07D1502080F31188BFF328
S315080102E04F8FBFF36F8FFEE7386C002807D0502079
S315080102F080F31188BFF34F8FBFF36F8FFEE7FFF7C8
S31508010300E3FB002802D10398002801D1012000E06F
S315080103100020C0B2002807D1502080F31188BFF30E
S315080103204F8FBFF36F8FFEE702F0FAFFBE6B002E09
S315080103301CD0701EB8633868002802D1FFF717FD74
S315080103407860386900280DD017F11000FFF777FAA1
S31508010350002807D05FF0805043490860BFF34F8FEC
S31508010360BFF36F8F02F0F9FF01207AE003980028A6
S315080103700DD1002D07D0502080F31188BFF34F8F80
S31508010380BFF36F8FFEE702F0E8FF002069E0002C5B
S3150801039004D16846FFF79CFA0120040002F0DDFF4C
S315080103A0FFF7DEF802F0BCFF97F9440010F1010FE0
S315080103B002D1002087F8440097F9450010F1010F92
S315080103C002D1002087F8450002F0C7FF03A9684655
S315080103D0FFF78CFA00282AD1380000F046F90028E0
S315080103E01FD03868002807D102F09AFF7868FFF70E
S315080103F07BFB050002F0B1FF039917F12400FFF713
S3150801040004FA380000F0F8F8FFF7B2F800288BD1A3
S315080104105FF0805014490860BFF34F8FBFF36F8FA9
S3150801042082E7380000F0E8F8FFF7A2F87CE7380021
S3150801043000F0E2F8FFF79CF8380000F016F90028FA
S315080104403FF472AF002D0BD002F06AFF380000F0BE
S3150801045064F8060031007868FFF70CFC02F07DFFAE
S31508010460002004B0BDE8F08104ED00E02DE9F04775
S3150801047080460C0015004646002E07D1502080F311
S315080104801188BFF34F8FBFF36F8FFEE7002C02D1A0
S31508010490306C002801D1012000E00020C0B20028FC
S315080104A007D1502080F31188BFF34F8FBFF36F8FA9
S315080104B0FEE702F07FFFEFF31189502080F31188E0
S315080104C0BFF34F8FBFF36F8FB76B002F20D096F90D
S315080104D044A02100300000F077F8781EB06350463A
S315080104E040B210F1010F0DD1306900280ED016F176
S315080104F01000FFF7A4F9002808D0002D06D0012026
S31508010500286003E01AF1010086F84400012000E0A2
S31508010510002089F31188BDE8F0870100486A0028A0
S3150801052004D0086B0068D0F1070000E0002070478E
S315080105302DE9F04707000E0014005FF00008BD6BB7
S31508010540386C002809D13868002838D17868FFF74F
S3150801055033FB80460020786031E0002C13D1D7F8B0
S315080105604090D7F808A04A4631005046FCF72EFAC3
S31508010570B868396C0844B860B868796888421ED387
S315080105803868B8601BE0D7F84090D7F80CA04A46FF
S3150801059031005046FCF71AFAF868396C49420844A2
S315080105A0F860F8683968884204D27868396C494233
S315080105B00844F860022C02D1002D00D06D1E681C7B
S315080105C0B8634046BDE8F087F8B504000D00206C15
S315080105D0002810D0E068216C0844E060E068616892
S315080105E0884201D32068E060266CE768320039004A
S315080105F02800FCF7EBF9F1BD70B5040002F090FE96
S3150801060094F94550280040B201280CDB606A00289D
S3150801061009D014F12400FFF712F9002801D0FFF7D9
S31508010620ACF96D1EEEE75FF0FF3084F8450002F085
S3150801063094FE02F075FE94F94460300040B2012838
S315080106400CDB2069002809D014F11000FFF7F7F830
S31508010650002801D0FFF791F9761EEEE75FF0FF302B
S3150801066084F8440002F079FE70BD38B5040002F042
S3150801067057FEA06B002801D1012500E0002502F0F4
S315080106806CFE280032BD38B5040002F049FEA06BA5
S31508010690E16B884201D1012500E0002502F05DFEEB
S315080106A0280032BD80B5DFF8C803006850F00100A4
S315080106B0DFF8BC130860DFF8B803006810F0010022
S315080106C000900098DFF8AC03006850F08050DFF81E
S315080106D0A4130860DFF89C03006810F080500090AE
S315080106E0009800220F217FF0010002F0E7FBDFF8F6
S315080106F08803006830F0E06050F00070DFF8781386
S31508010700086001BD18B585B004006846102102F0DD
S3150801071027FB2068DFF86413884259D1DFF85403B0
S31508010720006850F40020DFF84C130860DFF8440332
S31508010730006810F4002004900498DFF83403006878
S3150801074050F01000DFF828130860DFF8240300686A
S3150801075010F01000049004984FF480600090022075
S315080107600190032003906946DFF81403FBF72AFE7C
S315080107704FF4006000900020019000200290694625
S31508010780DFF8FC02FBF71EFEBE48BF4908600020E1
S31508010790BD4948600020BC4988608020BA49C860C4
S315080107A00020B94908610020B74948612020B649A7
S315080107B088610020B449C861B34800F083F900286C
S315080107C001D0FEF70FFDB0486063AF48446200E10F
S315080107D02068AE49884251D1A548006850F4804046
S315080107E0A3490860A248006810F480400490049860
S315080107F09F48006850F004009D4908609C480068BD
S3150801080010F00400049004984FF400700090022040
S3150801081001900320039069469D48FBF7D3FD4FF4E9
S315080108208060009000200190002002906946984857
S31508010830FBF7C8FD97489849086000209649486023
S3150801084000209549886080209349C8600020924914
S31508010850086100209049486120208F49886100205D
S315080108608D49C8618C4800F02DF9002801D0FEF7A2
S31508010870B9FC8948606388484462AAE020688749C8
S3150801088088424FD17B48006850F4003079490860A6
S315080108907848006810F40030049004987448006899
S315080108A050F00400724908607148006810F00400AD
S315080108B004900498042000900220019003200390DC
S315080108C069467348FBF77EFD0820009000200190D9
S315080108D00020029069466E48FBF774FD704871491D
S315080108E0086000206F49486000206E4988608020B2
S315080108F06C49C86000206B49086100206949486154
S3150801090020206849886100206649C861654800F069
S31508010910D9F8002801D0FEF765FC62486063614892
S31508010920446256E020686049884252D151480068BD
S3150801093050F480204F4908604E48006810F4802022
S31508010940049004984A48006850F00800484908602D
S315080109504748006810F00800049004984FF4806036
S315080109600090022001900320039069464F48FBF747
S3150801097029FD4FF4006000900020019000200290AC
S3150801098069464A48FBF71EFD49484A49086000205E
S315080109904849486000204749886080204549C86021
S315080109A04FF48070434908614FF4806041494861BA
S315080109B020204049886100203E49C8613D4800F031
S315080109C081F8002801D0FEF70DFC3A4860633948E2
S315080109D0446206B010BD10B5040020682749884254
S315080109E00ED12448006830F40020224908604FF4EB
S315080109F040612348FBF708FE606B00F0AAF836E071
S31508010A002068224988420ED11948006830F480408E
S31508010A10174908604FF4C0611D48FBF7F5FD606B87
S31508010A2000F097F823E020681C4988420DD1114847
S31508010A30006830F400300F4908600C211448FBF7B0
S31508010A40E3FD606B00F085F811E0206816498842DD
S31508010A500DD10848006830F48020064908604FF433
S31508010A6040611248FBF7D0FD606B00F072F810BDCB
S31508010A70181002401C10024004000140004C0040BE
S31508010A800010014030040240A066002000380140F1
S31508010A900008014058000240E46600200044004076
S31508010AA06C0002402867002000480040000C014005
S31508010AB0300002406C67002001480068704700BF9B
S31508010AC0E46B002010B401000022002901D10120A5
S31508010AD03DE00868DFF8B83398420CD20B68DFF8B6
S31508010AE0B403C3181420B3FBF0F080000864DFF8E0
S31508010AF0A803C8630BE00B68DFF8A003C31814202A
S31508010B00B3FBF0F080000864DFF89403C8630220A1
S31508010B1081F82100086803686FF30D134C6888682B
S31508010B200443C86804430869044348690443886957
S31508010B300443C869044323430868036000208863A3
S31508010B40012081F82100002081F82000002010BC36
S31508010B5070470100002901D1012045E008680068B5
S31508010B60400840000A68106000200A6810600020EA
S31508010B700A68506000200A68906000200A68D06000
S31508010B800868DFF80C2390420CD20A68DFF80403E0
S31508010B9082181420B2FBF0F080000864DFF8F8022E
S31508010BA0C8630BE00A68DFF8F40282181420B2FB66
S31508010BB0F0F080000864DFF8E802C8630122086CD7
S31508010BC08240C86B4260002088620020C86200200B
S31508010BD008630020486300208863002081F821000B
S31508010BE0002081F82000002070472DE9F04104001B
S31508010BF00D0016001F005FF0000894F82000012878
S31508010C0001D102203BE0012084F8200094F821005C
S31508010C1001282DD1022084F821000020A063206834
S31508010C20006840084000216808603B00320029003E
S31508010C30200000F017FBE06A002806D0206800684B
S31508010C4050F00E00216808600BE02068006830F05B
S31508010C500400216808602068006850F00A002168CD
S31508010C6008602068006850F001002168086004E007
S31508010C70002084F82000022080464046C0B2BDE824
S31508010C80F0810100002291F82100022806D00420F3
S31508010C908863002081F82000012018E008680068B0
S31508010CA030F00E000B6818600868006840084000BC
S31508010CB00B6818600123086C8340C86B43600120E8
S31508010CC081F82100002081F820001000C0B2704789
S31508010CD038B50400002594F82100022804D0042020
S31508010CE0A06301200500CFE02068006830F00E00FF
S31508010CF0216808602068006840084000216808608B
S31508010D002068DFF8A011884259D32068DFF89811C6
S31508010D10884201D101204EE02068DFF8901188420F
S31508010D2001D1102047E02068DFF88411884202D1FA
S31508010D304FF480703FE02068DFF87811884202D1CD
S31508010D404FF4805037E02068DFF86C11884202D1F1
S31508010D505FF480302FE02068DFF86011884202D105
S31508010D605FF4801027E02068DFF85411884202D129
S31508010D705FF080701FE02068DFF81411884201D106
S31508010D80012018E02068DFF83C11884201D11020C3
S31508010D9011E02068DFF83011884202D14FF48070E3
S31508010DA009E02068DFF82411884202D14FF4805007
S31508010DB001E05FF48030DFF81811086058E0206818
S31508010DC0DFF8E410884201D101204EE02068DFF8FF
S31508010DD0DC10884201D1102047E02068DFF8D010E6
S31508010DE0884202D14FF480703FE02068DFF8C410D2
S31508010DF0884202D14FF4805037E02068DFF8B810F6
S31508010E00884202D15FF480302FE02068DFF8AC1009
S31508010E10884202D15FF4801027E02068DFF8A0102D
S31508010E20884202D15FF080701FE02068DFF8601009
S31508010E30884201D1012018E02068DFF8881088422D
S31508010E4001D1102011E02068DFF87C10884202D118
S31508010E504FF4807009E02068DFF87010884202D1EB
S31508010E604FF4805001E05FF48030DFF8C01308606A
S31508010E70012084F82100002084F82000606B0028F6
S31508010E8002D02000616B88472800C0B232BD00003D
S31508010E9008040240F8FFFDBF00000240F8FBFDBF51
S31508010EA00004024081000240080002401C00024082
S31508010EB03000024044000240580002406C000240E3
S31508010EC0800002401C0402403004024044040240EF
S31508010ED00404024070B50400E06B056820680668E2
S31508010EE00421206C81400D4200F0C080700740F15A
S31508010EF0BD8020680068800605D42068006830F047
S31508010F000400216808602068DFF82413884258D352
S31508010F102068DFF82013884201D104204EE02068BA
S31508010F20DFF81413884201D1402047E02068DFF832
S31508010F300C13884202D14FF480603FE02068DFF845
S31508010F400013884202D14FF4804037E02068DFF869
S31508010F50F412884202D15FF480202FE02068DFF87E
S31508010F60E812884202D15FF4800027E02068DFF8A2
S31508010F70DC12884202D15FF080601FE02068DFF84A
S31508010F80D012884201D1042018E02068DFF8C41283
S31508010F90884201D1402011E02068DFF8BC1288425E
S31508010FA002D14FF4806009E02068DFF8B012884268
S31508010FB002D14FF4804001E05FF48020A84908601F
S31508010FC04CE020689B49884201D1042044E020680E
S31508010FD09949884201D140203EE0206897498842D4
S31508010FE002D14FF4806037E020689549884202D1E2
S31508010FF04FF4804030E020689249884202D15FF47C
S31508011000802029E020689049884202D15FF4800057
S3150801101022E020688D49884202D15FF080601BE09A
S3150801102020688B49884201D1042015E02068894946
S31508011030884201D140200FE020688749884202D1C1
S315080110404FF4806008E020688449884202D14FF451
S31508011050804001E05FF4802074490860E06A002856
S3150801106000F0E3802000E16A8847DEE00221206C77
S3150801107081400D4200F0B980B00740F1B680206882
S315080110800068800608D42068006830F00A002168E4
S315080110900860012084F821002068654988424DD3FB
S315080110A020686449884201D1022044E020686249E7
S315080110B0884201D120203EE020686049884202D159
S315080110C04FF4007037E020685D49884202D14FF439
S315080110D0005030E020685B49884202D15FF4003055
S315080110E029E020685849884202D15FF4001022E0BD
S315080110F020685649884202D15FF000701BE02068DB
S315080111005349884201D1022015E020685149884295
S3150801111001D120200FE020684F49884202D14FF4BF
S31508011120007008E020684D49884202D14FF400500A
S3150801113001E05FF400304A4908604CE020683D4907
S31508011140884201D1022044E020683B49884201D106
S3150801115020203EE020683949884202D14FF40070C8
S3150801116037E020683649884202D14FF4005030E012
S3150801117020683449884202D15FF4003029E02068AA
S315080111803149884202D15FF4001022E020682F49D4
S31508011190884202D15FF000701BE020682C49884222
S315080111A001D1022015E020682A49884201D1202070
S315080111B00FE020682849884202D14FF4007008E000
S315080111C020682649884202D14FF4005001E05FF4B5
S315080111D0003016490860002084F82000A06A00281B
S315080111E023D02000A16A88471FE00821206C81408E
S315080111F00D421AD0300718D52068006830F00E0065
S31508011200216808600121206C8140E06B4160012062
S31508011210A063012084F82100002084F82000206BB7
S31508011220002802D02000216B884770BD04000240C7
S3150801123081000240080002401C00024030000240C2
S3150801124044000240580002406C00024080000240FF
S31508011250080402401C0402403004024044040240CF
S315080112600404024030B40125046CA540C46B6560D2
S31508011270046863604468102C04D10468A260046899
S31508011280E16003E00468A1600468E26030BC70476D
S3150801129070477047F8B50400002C01D1012039E2E6
S315080112A02078C00740F18480DFF8AC06006810F0AA
S315080112B00C0004280BD0DFF8A006006810F00C001B
S315080112C008280ED1DFF890060068C00309D5DFF8B3
S315080112D08406006880036BD56068002868D1012000
S315080112E018E26068B0F5803F08D1DFF86806006843
S315080112F050F48030DFF85C16086038E06068002832
S3150801130010D1DFF85006006830F48030DFF8441653
S315080113100860DFF84006006830F48020DFF83416EC
S31508011320086024E06068B0F5A02F10D1DFF8240624
S31508011330006850F48020DFF81C160860DFF81406F0
S31508011340006850F48030DFF80C1608600FE0DFF80B
S315080113500406006830F48030DFF8F8150860DFF815
S31508011360F405006830F48020DFF8E8150860606845
S3150801137000280ED0FFF7A0FB0500DFF8D8050068A6
S31508011380800315D4FFF798FB401B6528F5D3032086
S31508011390C0E1FFF791FB0500DFF8B8050068800397
S315080113A006D5FFF789FB401B6528F5D30320B1E174
S315080113B0207880075CD5DFF8A005006810F00C0FCF
S315080113C00BD0DFF89405006810F00C0008281AD134
S315080113D0DFF884050068C00315D4DFF878050068CE
S315080113E0800704D52069012801D0012092E1DFF8A0
S315080113F06405006830F0F800616950EAC100DFF859
S315080114005415086034E0206900281ED00120DFF851
S315080114105C150860FFF750FB0500DFF83805006822
S31508011420800706D4FFF748FB401B0328F5D30320A2
S3150801143070E1DFF82005006830F0F800616950EACC
S31508011440C100DFF81015086012E00020DFF81C154E
S315080114500860FFF731FB0500DFF8F804006880072C
S3150801146006D5FFF729FB401B0328F5D3032051E1D5
S31508011470207800072CD5A069002816D00120DFF8AE
S31508011480F0140860FFF718FB0500DFF8DC040068B4
S31508011490800706D4FFF710FB401B0328F5D303206A
S315080114A038E1012000F041FA12E00020DFF8C0140B
S315080114B00860FFF701FB0500DFF8AC040068800748
S315080114C006D5FFF7F9FA401B0328F5D3032021E1D6
S315080114D02078400740F1A8800027DFF898040068C3
S315080114E0C00010D4DFF88C04006850F08050DFF893
S315080114F084140860DFF87C04006810F080500090BE
S31508011500009801200700DFF870040068C00516D4AA
S31508011510DFF86404006850F48070DFF85C14086032
S31508011520FFF7CAFA0500DFF850040068C00506D4BB
S31508011530FFF7C2FA401B6528F5D30320EAE0E06805
S31508011540012808D1DFF83404006850F00100DFF8FB
S315080115502C14086037E0E068002810D1DFF81C0475
S31508011560006840084000DFF814140860DFF80C042E
S31508011570006830F00400DFF80414086023E0E0682E
S31508011580052810D1DFF8F403006850F00400DFF8ED
S31508011590EC130860DFF8E403006850F00100DFF897
S315080115A0DC1308600FE0DFF8D40300684008400048
S315080115B0DFF8C8130860DFF8C403006830F00400D8
S315080115C0DFF8B8130860E068002810D0FFF774FA4E
S315080115D00500DFF8A8030068800719D4FFF76CFA3D
S315080115E0401B41F289318842F3D3032092E0FFF789
S315080115F063FA0500DFF884030068800708D5FFF75A
S315080116005BFA401B41F289318842F3D3032081E01A
S315080116103800C0B2012807D1DFF85803006830F056
S315080116208050DFF850130860E069002871D0DFF8B0
S315080116302803006810F00C00082855D0E069022834
S315080116403FD10020DFF838130860FFF735FA0700A5
S31508011650DFF800030068800106D5FFF72DFAC01BE5
S315080116600328F5D3032055E0206AB0F5803F09D158
S31508011670DFF8E402016831F40031A0680143DFF8BC
S31508011680D8020160DFF8D002016831F47411206ACA
S315080116900143606A0143DFF8C00201600120DFF8F7
S315080116A0E0120860FFF708FA0500DFF8A8020068EB
S315080116B080012ED4FFF700FA401B0328F5D3032037
S315080116C028E00020DFF8B8120860FFF7F5F90500F1
S315080116D0DFF88002006880011BD5FFF7EDF9401B92
S315080116E00328F5D3032015E0E069012801D101207B
S315080116F010E0DFF864020068060016F48030216AFB
S31508011700884204D116F47010616A884201D001201A
S3150801171000E00020F2BD70B504000D00002C01D1D7
S315080117200120AFE0DFF85C02006810F00700A8426C
S3150801173011D2DFF850020068C008C0002843DFF85C
S3150801174044120860DFF83C02006810F00700A8425E
S3150801175001D0012096E0207880071FD52078400720
S3150801176007D5DFF8F401006850F4E060DFF8E81106
S3150801177008602078000707D5DFF8DC01006850F417
S315080117806050DFF8D4110860DFF8CC01016831F048
S31508011790F001A0680143DFF8C00101602078C007A5
S315080117A034D56068012806D1DFF8A80100688003EE
S315080117B010D4012066E06068022805D165480068F2
S315080117C0800107D401205DE062480068800701D4E2
S315080117D0012057E06048016889088900606801436B
S315080117E05D480160FFF768F906005B48006810F07C
S315080117F00C006168B0EB810F08D0FFF75DF9801B1B
S3150801180041F289318842F0D303203BE05D48006804
S3150801181010F0070085420ED25A480068C008C00079
S315080118202843584908605748006810F00700A8423D
S3150801183001D0012026E02078400707D546480168EF
S3150801184031F4E061E068014343480160207800070C
S3150801185008D54148006830F46050216950EAC10052
S315080118603D49086000F00FF847493B4A1268C2F340
S315080118700312895CC8403A4908603A48006801F091
S31508011880F9FD002070BD78B585B001A83F49102241
S31508011890FBF7ACF83E480088ADF8000000200021AF
S315080118A00022002300242C4D2D6815F00C06042E69
S315080118B002D0082E02D01CE036481BE001A8C5F369
S315080118C08346805D0300E8030DD56846224E3668D7
S315080118D0C6F34046805D01002E4800FB03F0B0FBCD
S315080118E0F1F0020003E02C4800FB03F002001000AF
S315080118F000E01A4806B070BD19480068704780B5FF
S31508011900FFF7FAFF2549144A1268C2F30222895CD5
S31508011910C84002BD80B5FFF7EFFF20490E4A12689D
S31508011920C2F3C222895CC84002BD81B00C4909686C
S31508011930C9084FF47A72B1FBF2F101FB00F100918B
S3150801194000BF00994A1E00920029F9D101B07047DB
S3150801195000000000001002400410024000127A0044
S315080119607801002074010020241002400000424240
S31508011970800442421C1002400070004020100240C0
S3150801198060004242002002402463010814630108F2
S31508011990C22701080024F40000093D009C660108DD
S315080119A02DE9F0439FB000BF66A6269CDFF8E48ABE
S315080119B002918DF83B4000210B914FF0FF37044609
S315080119C091461D460AE019F8011B0298A04700280E
S315080119D0029000F0A4800B98401C0B9099F8000027
S315080119E050B12528EFD100200021059006910790D6
S315080119F0089109900A9103E00B98A7E041F00101CB
S31508011A0019F8010F2028F9D023280CD02B2804D047
S31508011A102D2805D0302809D083E041F00201EFE7EF
S31508011A2041F00401ECE741F00801E9E741F0100152
S31508011A30E6E700200D900AE00D98404505DA00EB2F
S31508011A40800302EB4302303A0D9209F1010999F834
S31508011A500020A2F130000A28EED399F800002E28BA
S31508011A6018BF0C9726D119F8010F2A2808D128681A
S31508011A70286009F1010950F8042B28600C9219E035
S31508011A802D280CBF19F8010B002000220C920BE03F
S31508011A9040B90C9A424505DA02EB820203EB42038E
S31508011AA0303B0C9309F1010999F80030A3F1300292
S31508011AB00A2AEDD3ADF83810304699F8001001F02E
S31508011AC0FFFC08B119F8010B8DF83A009DF83A00A8
S31508011AD0682804BF99F80010682903D162208DF897
S31508011AE03A0008E06C2804BF99F800006C2804D174
S31508011AF071218DF83A1009F1010910A804902A46B6
S31508011B0019F8013B6946204600F060F838B910AA71
S31508011B106946204600F08CF900287FF55FAF384604
S31508011B2014E02A2885D12A682A6052F8040B2A600B
S31508011B3000280D9003D540420D9041F0040109F1AA
S31508011B4001098AE7686A6C747A4C00001FB0BDE81F
S31508011B50F083622820D0682811D06A2803D06C281F
S31508011B6027D0712825D10868C01D20F00700086014
S31508011B70D0E9002308300860194610467047002A44
S31508011B800A680A60106803D0121D0A6000B217E0DD
S31508011B90121D0A6080B217E0002A0A680A601068F6
S31508011BA003D0121D0A6040B20AE0121D0A60C0B2D3
S31508011BB00AE0002A0A680A60106803D0121D0A6042
S31508011BC0C1177047121D0A600021704770B51C467F
S31508011BD00D46B4F125002E69114600F017811C380F
S31508011BE06AD0001F022867D9133843D0093863D051
S31508011BF0801E16D0401E1ED0401E02285CD9001F2A
S31508011C0019D0401F00F08380401E33D0401E00F0DB
S31508011C10CD80C01E00F0D880801E2BD0C01E29D0D2
S31508011C20FAE06869421C6A610A680A6052F8043B6C
S31508011C300A603354FAE095F83A000122FFF789FF62
S31508011C40C5E900010023994204DA6869411C696102
S31508011C502D210DE0288F810704D56869411C69612A
S31508011C602B2105E0C00722D56869411C696120213D
S31508011C7031541CE095F83A000022FFF76AFFC5E9DE
S31508011C80000195F83800010711D5D5E90023002090
S31508011C90834208BF82420AD044F02000782806D140
S31508011CA0686930213154401C411C6961345421460C
S31508011CB068693044E86083E00868C01D20F00700C1
S31508011CC00860D0E9002308300860C5E90023D5E992
S31508011CD00001C80F04D06869411C69612D210DE016
S31508011CE0288F810704D56869411C69612B2105E0A4
S31508011CF0C00704D56869411C6961202131546869A6
S31508011D003044E8602146284600F0C4F98EE005F122
S31508011D103A02507820B14FF0FF340FF648205EE0C2
S31508011D201078622808D0682824D06A2812D06C282E
S31508011D302ED071280ED02BE00A680A6052F8040BDF
S31508011D400A6020B94FF0FF340FF6302047E0E96A00
S31508011D5001706BE00A680A6052F8040B0A6020B940
S31508011D604FF0FF340FF6142039E0EA6AD317C0E9B9
S31508011D7000235BE00A680A6052F8040B0A6020B97E
S31508011D804FF0FF340FF6F41029E0E96A01804DE0BF
S31508011D900A680A6052F8040B0A6020B94FF0FF344A
S31508011DA00FF6D8101BE0E96A01603FE00A680A608D
S31508011DB052F8040B0A600021C5E90001EE6078219A
S31508011DC0284600F0BBF831E00868086050F8044B73
S31508011DD00860EC603CB94FF0FF340FF6B81001F01B
S31508011DE07BFB201A70BD2E6B002E04D52046FAF710
S31508011DF045FE044608E032460021204601F08CFBE8
S31508011E00002814BF041B3446AC610FE06869411C05
S31508011E1069612521315409E06969481C68612522EF
S31508011E207254210002D0411C69613454002070BDEE
S31508011E302DE9FC410F460646796B7869BC6A091A91
S31508011E40386A091AB869091A786A091AF869091AF1
S31508011E5097F838000C1B410790460FD42021002C17
S31508011E608DF800100ADD254601236A4639463046B3
S31508011E7000F060FC00285DD16D1EF5D17B694246F4
S31508011E803946304600F056FC002853D130208DF8EB
S31508011E9000003D6A002D09DD01236A4639463046B0
S31508011EA000F048FC002845D16D1EF5D1BB69FA68DA
S31508011EB03946304600F03EFC00283BD130208DF8EB
S31508011EC000007D6A002D08DD01236A463946304641
S31508011ED000F030FC70BB6D1EF6D1F868B969FB6974
S31508011EE042183946304600F025FC18BB30208DF8DB
S31508011EF00000BD6A002D08DD01236A4639463046D1
S31508011F0000F018FCB0B96D1EF6D197F838004107F4
S31508011F100DD52021002C8DF8001008DD01236A4615
S31508011F203946304600F006FC20B9641EF6D1002079
S31508011F30BDE8F6814FF0FF30BDE8F6812DE9FC4793
S31508011F4007468A463E69BAF16F0F08BF082405D0CD
S31508011F504AF02001782914BF0A2410243C25D7E920
S31508011F600023BAF1640F18BFBAF1690F9046994672
S31508011F7006D100218B4203DAD8F1000869EB490939
S31508011F800020814508BF80451FD1386BE8B9082C68
S31508011F904CD197F83800010748D530203B2586F8FB
S31508011FA03B0043E000280ED597F8380000F01400EE
S31508011FB0102808D17A6B7869121A386A121A511AD6
S31508011FC00029C8BF3962BDE8F3878DF800A04046ED
S31508011FD049462246E31701F0CBFA3032D0B26D1EDC
S31508011FE03A28019504DB9DF80000A0F151018A18F1
S31508011FF07255404649462246E31701F0B9FA80462A
S3150801200089460020814508BF804503D0F8687119C3
S315080120108842DCD3082C09D197F83800010705D581
S31508012020715D302902D06D1E30207055C5F13C0115
S31508012030B9617019F860386B8142B3DA411A3962AD
S315080120404FF6EF70398F01403987BDE8F3872DE9DF
S31508012050D04306460F4614464FF00008DFF8389479
S3150801206012E0E00707D542464B463046394601F0AD
S3150801207097FB06460F464046494642464B4601F0FF
S315080120808FFB641080468946002CEAD130463946D2
S31508012090BDE8D0832DE9F34F054641F020048DB004
S315080120A0D5E90089612C02AE09D0286B002848BF02
S315080120B0062003D408BF672C01D101202863D5E97E
S315080120C0002358004015401C0ED119030CD00320DB
S315080120D0A8619DF8380061381A2802D20FF2D0613A
S315080120E011E00FF2D0610EE058004015401C0FD1E7
S315080120F019030DD10320A8619DF8380061381A2803
S3150801210014D30FF2B861E8680322FAF75FFCD3E14A
S31508012110194621F00043B3F5801F10460DD200275A
S31508012120BB4208BFBA42019703D111E00FF2886199
S31508012130E9E701AA01F006FC0AE0DFF8607307EB9C
S315080121401352DFF85C3301921940DFF8583319430B
S31508012150C5E90001612C0ED1E86830210170811CA6
S31508012160E9609DF8381061290CBF78215821417022
S315080121706869801C6861D5E900AB2BF00043002033
S315080121802AF00002834204BF8242002300F05A81EA
S31508012190612C40F0A980286B00284CBF2120401CE7
S315080121A000904046009F7F1C49460022002301F00B
S315080121B001FCD94601988DF8082038BF89F00049F5
S315080121C0001F0190002FD0460DF1090040F3498107
S315080121D040F2FF71DFF8D0B20C91064640464946F7
S315080121E00022002301F0FEFB80F03A814800400DF1
S315080121F000F11C0210D0002A0EDD0C98824205DB84
S3150801220009F0004040EA0B01002013E0A448084009
S3150801221040EA025140460DE029F00043002028F02B
S315080122200002834208BF82420FBF40461C22404635
S3150801223001F0F0FB8046894601F08AFCFF1F002F5A
S31508012240044609DD01F0A2FC02460B464046494612
S3150801225001F0AEFC80468946F01D072104E004F032
S315080122600F0200F8012D2411002C01DD491EF6D5B7
S31508012270491E5CBF002200F8012DF9D5ECE00020CB
S31508012280194602AA0A4400E05B1E12F80149491ED2
S315080122908442F9D00F2804D10DF10900425C521C81
S315080122A04254002904D50198001D02AE5B1C019019
S315080122B0591E12D49DF838007218147804F13008A2
S315080122C05FFA88F4392CC4BFA0F13A04A044491E28
S315080122D002F80189F1D58DF83800286B002840F1FC
S315080122E0B080591E2963ACE04046494600220023C6
S315080122F001F060FB019938BF89F0004947F2975010
S3150801230041436A4A91FBF2F20192D2F1070204DDD6
S3150801231040464946FFF79BFE0AE0524200206449BF
S31508012320FFF795FE02460B464046494601F0B2FCC8
S315080123308046662C286BDFF87CB106BF019F0A37F9
S3150801234006273F18142FC8BF142730208DF8080018
S3150801235089460DF1090000E03046002F34DD0646B6
S315080123604046494601F0BAFD01460A4606F1080308
S3150801237004200A26B2FBF6F606EB860EA2EB4E02FF
S31508012380303203F8012C0A22B6FBF2F202EB820E76
S31508012390A6EB4E063036401E03F8026DE9D1083F1A
S315080123A0002F03F10806D7DD084601F0ABFD02460A
S315080123B00B464046494601F0FBFB00225B4601F00D
S315080123C0EFF980468946CBE70DF10901401A0DF16F
S315080123D0090604E00199491E401E0191761C3178CF
S315080123E03029F7D0662C02D10199491C03E0652CE6
S315080123F00CBF012100212B6BCB189842B8BF431E95
S31508012400002B1ED4834204DAF05C3528A8BF392094
S3150801241000DA30201946721E02EB010800E05B1E45
S3150801242018F80199491E8145F9D0392802D1705CFD
S31508012430401C7054002904D50198401C16465B1CA3
S315080124400190019800B200901BB29DF838103246EF
S31508012450284600F035F82FE0C61D002F3FF7BEAE1F
S3150801246030460DF10901401A009903468842C8BF52
S315080124700B46002B0DF109063FF52FAF8342BFF638
S31508012480FEAE0DF10900C05C07287FF7F8AE0F20F4
S31508012490F6E60000CBCCCC0C0000244002FCFFFF82
S315080124A0FFFF0F800000E03F0000F07FA0860100DB
S315080124B00000F03F84D797410FB0BDE8F08F0000C8
S315080124C02DE9FC43054683B01F46D5F83080002F19
S315080124D0164602DC5FF00107B9A68946BDF9304008
S315080124E049F02000662808BF641C17D0672840F009
S315080124F0888014F1040FC0F28A80444580F28780EF
S3150801250095F83800641C010702D44745B8BFB84698
S3150801251020B2B8EB000848BF4FF000080FFA84F95B
S31508012520E868A969B9F1000F27DC4A1C302343542E
S31508012530B8F1000F03DC95F83800010703D5E86800
S315080125402E218154521C18EB090FB8BFC8F100049B
S3150801255024B260426862A044B845AA61B8BF47463A
S31508012560E868AB693FB2EF613A4631461844FAF773
S315080125702DFAA8EB0700A862C5E022B297420844E3
S3150801258019DA3A463146FAF721FAA8693818A9EB51
S315080125900707B8F1000FA8616F6203DC95F83810D8
S315080125A00A0705D5E9682E220A54E869401CE8613C
S315080125B0C5F82880A7E03146FAF708FAA8693F1B4B
S315080125C0B8F1000F484403DC95F838100A0703D51B
S315080125D0E9682E220A54401CA86138B28045E86889
S315080125E0AB69B8BF47463AB206EB09011844FAF790
S315080125F0EDF9A8693FB23818A8EB0707A8616F6219
S3150801260081E0B9F1610F16D14FF0700918E047451D
S3150801261004DA95F838100A0758BFB846B8F1010820
S3150801262048BF4FF00008B9F1670F14BF4FF04509CD
S315080126304FF0650904E0B9F1410F08BF4FF05009A1
S31508012640A969EB68481CA861B8F1000F16F8012BB7
S315080126505A5403DC95F838100A0719D5EA68431C59
S31508012660AB612E211154B8F1000F11DD7F1E38B26E
S315080126708045E868B8BF47463AB231461844FAF782
S31508012680A5F9A8693FB23818A861A8EB07006862DE
S31508012690E868A9690844002C80F8009003D42B2126
S315080126A04170811C03E02D2141706442811C002088
S315080126B06A460AE023460A2493FBF4F404EB8406EB
S315080126C0A3EB460302F8013B401C24B2002CF1DCC3
S315080126D0012806DC49F02002652A04BF302201F8E8
S315080126E0012B48B9302001F8010B07E0401E1DF8FF
S315080126F00020303201F8012B0028F7DCE868AA69C6
S315080127001044091AE96195F8380000F014001028F8
S315080127100DD16969A8694118686A4118E8694118BB
S31508012720A86A4118686B8142BCBF411A296205B083
S31508012730BDE8F083F8B505460E4617461C46002047
S3150801274074B117F8011BB068A847B06030B1F06AD8
S31508012750401CF0620020641EF3D1F2BD4FF0FF3039
S31508012760F2BD00007072696E74665F733A20256E59
S3150801277020646973616C6C6F776564007072696E49
S3150801278074663A2062616420256E20617267756DF0
S31508012790656E74007072696E74665F733A20626161
S315080127A06420257320617267756D656E740000007B
S315080127B06E616E004E414E00696E6600494E4600D6
S315080127C03000010210B40400002C02D15FF0FF3082
S315080127D018E0216000202071606830F48070606024
S315080127E000206062002084F8280000202074002060
S315080127F060610020A0610020207700206077A26038
S31508012800E360002010BC70472DE9F84304000D0071
S3150801281016005FF000080027002C02D0E0680028A7
S3150801282002D15FF0FF3063E01020414689B22144AE
S3150801283081F8290118F101080220414689B221448B
S3150801284081F8290118F101085FF0000948463100AD
S3150801285080B289B2884223D2484680B2285C414672
S3150801286089B2214481F8290118F10108484680B244
S31508012870285CC719484680B2285C10280DD14846FD
S3150801288080B2285C414689B2214481F8290118F1B0
S315080128900108484680B2285CC71919F10109D5E72C
S315080128A01020414689B2214481F8290118F101080D
S315080128B00320414689B2214481F8290118F101080A
S315080128C0F0191330414689B2214481F8290118F1DA
S315080128D00108404680B22062002060770020A0618E
S315080128E000202074216A04F22910E268904700202A
S315080128F0BDE8F28370B504000D001600002C02D164
S315080129005FF0FF30A5E03000461E0128C0F2A08026
S31508012910207902281DD194F82810606A411884F894
S31508012920281094F828002978884209D1A068002837
S315080129300AD0616AC9B214F12900A268904703E076
S3150801294002214548E2689047002020740020207142
S315080129507CE094F828102878411884F828106068D3
S31508012960C0F30020002858D0606830F48070606099
S315080129702878022807D100206062002084F8280000
S315080129800120207162E02878032808D120790128DE
S3150801299002D10220207159E00020207156E02878E2
S315080129A0102816D1207901280ED1606AB0F5807FEA
S315080129B007D2606A411C61622978204480F829108F
S315080129C044E00020207141E0606850F48070606046
S315080129D03CE02878152839D1207F002815D0607F5A
S315080129E0217F88420CD202202074607F401C6077C8
S315080129F00020A061216A04F22910E26890470BE0E1
S31508012A000020A0610320207406E000202074216ABA
S31508012A1004F22910E268904718E02878102804D1B2
S31508012A20606850F48070606010E0207901280DD14B
S31508012A30606AB0F5807F07D2606A411C61622978B5
S31508012A40204480F8291001E0002020716D1C5AE706
S31508012A50002070BD00000000B46601080288024427
S31508012A6091700288521C028000887047F8B50400EC
S31508012A700D004FF4817600273A0031002800F9F756
S31508012A80A5FE02212800FFF7E9FF200000F035F82E
S31508012A900100C9B22800FFF7E1FF200000F033F872
S31508012AA00100C9B22800FFF7D9FFF1BDF8B5040046
S31508012AB00D004FF4817600273A0031002800F9F716
S31508012AC085FE0F212800FFF7C9FF21782800FFF7A7
S31508012AD0C5FFF1BD70B504004FF4817500263200BB
S31508012AE029002000F9F772FE05212000FFF7B6FF3D
S31508012AF070BD801C704700887047007870470200D7
S31508012B00117001207047407870470200517001200A
S31508012B107047000080B50848006850F01000064963
S31508012B200860032000F0C4F90F2000F0A3FCFDF7AC
S31508012B30B9FD002002BD0000002002402DE9F84F32
S31508012B4004000D001600FF277C4800780C286FDA70
S31508012B502800C0B221280FDAA8465FFA88F8784912
S31508012B60764802782220424301EB020942462100B7
S31508012B704846F9F72BFF0DE05FF0200870496F48CA
S31508012B8002782220424301EB0209424621004846C7
S31508012B90F9F71CFF6A49694802782220424301EB8A
S31508012BA0020080F820606649644802782220424380
S31508012BB001EB020090F82010614A60480378222050
S31508012BC0434302EB030080F821105C4890F800802B
S31508012BD05A480078401C594908701D215948F7F789
S31508012BE08DFF5FF003095FF0000AEB46524649463E
S31508012BF05846F9F7EBFD4246D2B24DA16846FBF7B6
S31508012C00F9F96846F9F73AFF010089B26846F7F714
S31508012C1075FF022147A0F7F771FF2900C9B289B2EA
S31508012C202000F7F76BFF022143A0F7F767FF0FE0D4
S31508012C304FF0FF0834214448F7F760FF2900C9B26D
S31508012C4089B22000F7F75AFF02213BA0F7F756FF92
S31508012C505FFA88F84046BDE8F28F10B504002000F7
S31508012C6036490978C0B2884212D235492200D2B211
S31508012C702220424301EB020090F82010304A23003B
S31508012C80DBB22220434302EB030080F8211004E063
S31508012C902100C9B22D48F7F75FFF10BD38B50021ED
S31508012CA000242B480078002840D100252800234914
S31508012CB00978C0B2884230D221492A00D2B22220EC
S31508012CC0424301EB020090F82100002814D01C4968
S31508012CD02A00D2B22220424301EB020090F82100D9
S31508012CE0401E040016492A00D2B22220424301EBB3
S31508012CF0020080F821400EE011492A00D2B22220B2
S31508012D00424311441348F7F727FF1348F7F724FFFF
S31508012D1001200F4908706D1CC8E7F9F70FFFF9F78D
S31508012D2023FF002802D10D4800F045F831BD000007
S31508012D30256400005D2000000D0A0000C76C002014
S31508012D40DC5B0020D05401081C47010854470108E0
S31508012D50C86C0020044D0108F05401084C6B002092
S31508012D60002201F0DDB838B50400002C01D101209C
S31508012D7020E04CF6CC402168086045F255502168A0
S31508012D800860606821684860A06821688860FDF766
S31508012D9093FE05002068C068002806D0FDF78CFE62
S31508012DA0401B2728F6D3032004E04AF6AA20216807
S31508012DB00860002032BD01004AF6AA200A681060A0
S31508012DC00020704710F00703DFF834110A684FF640
S31508012DD0FF010A40DFF82C1151EA03210A43DFF803
S31508012DE020110A607047DFF818010068C0F3022055
S31508012DF07047010049B200290AD4012210F01F01C7
S31508012E008A40DFF8041103005BB25B0941F823200D
S31508012E10704710B4020052B2002A05D40A013B4B8E
S31508012E20040064B21A5508E00A01394B040064B279
S31508012E3014F00F04234403F8042C10BC704770B433
S31508012E40030013F00704D4F10700052801D3042071
S31508012E5001E0D4F10700251D072D01D2002500E068
S31508012E60E51E012616FA00F0401E0140A940012080
S31508012E7010FA05F56D1E2A401143080070BC70470B
S31508012E8010B50400601EB0F1807F01D301200EE069
S31508012E90601E204908600F215FF0FF30FFF7B9FF78
S31508012EA000201D49086007201C490860002010BD44
S31508012EB010B504002000FFF785FF10BD2DE9F0418C
S31508012EC004000D0016000027FFF78DFF804632002B
S31508012ED029004046FFF7B3FF0100200040B2FFF783
S31508012EE098FFBDE8F08110B50400200040B2FFF755
S31508012EF080FF10BD10B504002000FFF7C1FF10BD0B
S31508012F000CED00E00000FA0500E100E000E400E055
S31508012F1018ED00E014E000E018E000E010E000E041
S31508012F202DE9F04104005FF00008FCF719FB93480E
S31508012F300068002801D100F0BDF8914800680442F4
S31508012F406AD1002C15D08F480068041914F0070FB0
S31508012F500FD014F1080014F00704041B14F0070F2E
S31508012F6007D0502080F31188BFF34F8FBFF36F8FBF
S31508012F70FEE7002C50D084480068A0424CD3834811
S31508012F8006008248006805006868A04205D22868DC
S31508012F90002802D02E002D68F6E778480068854299
S31508012FA03AD030687749096808448046286830600D
S31508012FB07448006840006968091B884215D205EB08
S31508012FC00400070017F00700002807D0502080F3F7
S31508012FD01188BFF34F8FBFF36F8FFEE76868001B39
S31508012FE078606C60380000F098F86748016868688E
S31508012FF0091A654801606448006865490968884294
S3150801300003D2614800686249086069685C480068DB
S315080130100143696000202860FCF7AAFA18F0070046
S31508013020002807D0502080F31188BFF34F8FBFF3D4
S315080130306F8FFEE74046BDE8F08170B504002600B3
S31508013040002C36D04F48006840420644350068686F
S315080130504B490968084207D1502080F31188BFF30C
S315080130604F8FBFF36F8FFEE72868002807D05020DF
S3150801307080F31188BFF34F8FBFF36F8FFEE7686840
S315080130803F490968084214D02868002811D169689F
S315080130903B48006881436960FCF762FA3A4801686F
S315080130A06868411838480160280000F036F8FCF7CE
S315080130B05FFA70BD10B44FF4A041364A12F0070FFB
S315080130C005D0D21DD208D200891A324841182F4894
S315080130D0026000202D4B58608B182A4800681B1A7D
S315080130E0DB08DB00254803600020244C2468606067
S315080130F00020224C24682060981A50601F480068F6
S3150801310010605068224C206050681F4C20605FF0A8
S3150801311000401B4C206010BC704730B41B4A116834
S31508013120814201D21268FAE71400516821448142AA
S3150801313004D153684168CB185360100003004168F5
S3150801314019441568A94211D111680C4C2468A14289
S3150801315008D04468116849680C19446011680968FF
S31508013160016005E005490968016001E0116801602F
S31508013170824200D0106030BC70470000806B00208E
S315080131808C6B0020B8660108846B0020706B0020E8
S31508013190886B00208401002010F1080141605FF06E
S315080131A0FF31816010F10801C16010F10801016168
S315080131B000210160704700210161704742684A6039
S315080131C093688B60936859609160086103685B1C1A
S315080131D00360704710B40B6813F1010F01D102693E
S315080131E007E010F1080254682468A34201D3526823
S315080131F0F9E754684C604C68A1608A6051600861BF
S315080132000468641C046010BC7047010008698A6878
S315080132104B689A604A688B685A6042688A4201D14B
S315080132208A68426000220A610268521E02600068CA
S3150801323070470000001F5FF080730360001F4B0892
S315080132405B000360001F0FF20D0303601438026070
S31508013250203870476B48006810F1010F07D05020DD
S3150801326080F31188BFF34F8FBFF36F8FFEE75020AE
S3150801327080F31188BFF34F8FBFF36F8FFEE7E0B579
S31508013280614801780191FF21017001788DF80010DC
S315080132909DF8001011F050015C4A117007215C4A33
S315080132A011609DF8001009060AD559490968491E91
S315080132B0574A11609DF8001049008DF80010F0E793
S315080132C053490968D1F10701042907D0502181F32F
S315080132D01188BFF34F8FBFF36F8FFEE74C4909681B
S315080132E009024B4A11604A49096811F4E061484AE2
S315080132F01160019901704748006850F4700045490A
S3150801330008604448006850F070404249086000F07F
S3150801331089F800203B49086000F04FFE00200EBDE9
S31508013320502080F31188BFF34F8FBFF36F8F354855
S315080133300068401C334908603248006801280BD1EF
S3150801334035480068000607D0502080F31188BFF37E
S315080133504F8FBFF36F8FFEE770472A480068002832
S3150801336007D1502080F31188BFF34F8FBFF36F8FBA
S31508013370FEE724480068401E224908602148006883
S31508013380002802D1002080F31188704780B55020AB
S3150801339080F31188BFF34F8FBFF36F8FFCF768F97E
S315080133A0002803D05FF080501B490860002080F395
S315080133B0118801BDEFF30580102811D3174A126849
S315080133C0125C11000A00114B1B78D2B29A4207D23D
S315080133D0502282F31188BFF34F8FBFF36F8FFEE739
S315080133E00B4A12680E4B1B6813F4E0639A4207D224
S315080133F0502282F31188BFF34F8FBFF36F8FFEE719
S31508013400704700007001002000E400E0C06C002055
S31508013410E06B002020ED00E004ED00E0BC66010849
S315080134200CED00E000200949086000200849086001
S31508013430084800684FF47A71B0FBF1F0401E06495E
S315080134400860072001490860704700BF10E000E0E6
S3150801345018E000E07801002014E000E0034B036067
S31508013460034B0B6080231360704700BF4C66002036
S31508013470DC57002010B504004FF47A700D4909781D
S31508013480B0FBF1F00C490968B1FBF0F0FFF732FD2A
S31508013490002801D001200CE0102C09D200222100BD
S315080134A05FF0FF30FFF70AFD04480460002000E0E2
S315080134B0012010BD8201002078010020740100203E
S315080134C00278C9B28A421AB11CBF10F8012FF9E76E
S315080134D018BF00207047000080B500B906A005494D
S315080134E00B681BB122220021984701E000F076FD06
S315080134F0222002BD286C0020636F6E7374726169A5
S315080135006E742068616E646C65723A20626164202B
S315080135106D65737361676500C9B2830706D0521E6C
S3150801352022D310F8013B9942F7D11FE0083A13D389
S3150801353002F1040241EA012141EA014150F8043B42
S31508013540121F21BF4B40A3F1013C2CEA030C1CF0CE
S31508013550803FF3D0C9B2001F083210F8013B521E52
S3150801356028BF91EA030FF8D818BF0120401E7047FB
S31508013570B3BBD9B1B2F5803F7DD2022A1ED98C469A
S31508013580B1FBF2F102FB11C31B0443EA1043B3FB7F
S31508013590F2FC02FB1C3380B240EA0343B3FBF2F0B0
S315080135A002FB103240EA0C4000237047022A05D973
S315080135B08446B0FBF2F002FB10C270474AB105D14E
S315080135C000F0010249085FEA300070470022002333
S315080135D0704700F007BD0B0002000021002070476C
S315080135E0904271EB030CF6D3B3F5803F2FD2F0B5B9
S315080135F0B3FA83F7B1FA81F4A7F10F0E3D1B5340D5
S31508013600CEF1200602FA0EF2F3415340B5F10F0747
S3150801361046D80F3C2C444140C4F12006A040F14154
S315080136204140B1FBF3F603FB1611A2FB0645001B4D
S31508013630A94102D2761E8018594180EA010221FA6F
S315080136400EF362FA0EF200215A403046F0BD30B44C
S31508013650B1FBF3FC03FB1C11A2FB0C45001BA941A2
S3150801366003D2ACF1010C8018594130BC02460B4615
S31508013670604600217047B2F1807F65D3F0B5B2FA92
S3150801368082F7B1FA81F4C7F10F063D1B22FA06F358
S3150801369007F1110EF24120355A40B5F10F07B8D995
S315080136A04140C4F12006A040F1414140B1FBF3FC81
S315080136B003FB1C11A2FB0C45001BA94103D2BCF15B
S315080136C0010C801859410F2F12D30F3FC90341EA44
S315080136D05041B1FBF3F603FB1611A2FB0645D4EBE9
S315080136E0C030A94102D2761E8018594146EACC3C1F
S315080136F007B34140C7F12006B840F1414140B1FB4B
S31508013700F3F603FB1611A2FB0645001BA94102D2DB
S31508013710761E8018594180EA010221FA0EF3C7F193
S31508013720200462FA0EF20CFA07F05A402CFA04F158
S315080137303043F0BD80EA010221FA0EF3002162FA54
S315080137400EF260465A40F0BD8C46B1FBF2F102FB1F
S3150801375011C31B0243EA1063B3FBF2FC02FB1C33E1
S315080137601B024CEA002043EA1063B3FBF2FC02FB9E
S315080137701C331B024CEA002043EA1063B3FBF2FC3C
S3150801378002FB1C331B024CEA002043EA1063B3FB1D
S31508013790F2FC02FB1C324CEA0020002370470000B1
S315080137A0B0B581EA030C0CF0004C40F2FF7515EA3E
S315080137B011541DBF15EA1357AC42AF4239E0E4195B
S315080137C023EA455343F48013C90241F0004141EA13
S315080137D0505EC7021100A7FB020200284FF0000045
S315080137E0EEFB01204FF00001E3FB072118BF42F071
S315080137F00102401800214941E3FB0E01A4F580644A
S315080138000F0302D252004041494154F101046CDDD3
S31508013810470872F1004250F1000051EB0451A1F53D
S3150801382080115CBF41EA0C01B0BD4CEA055100208C
S31508013830B0BD05EA1357AC4214BFAF4241E050EAA6
S31508013840410E1CBF52EA430E02E061460020B0BD9C
S3150801385024423C441BD15FEA070EF6D0090302BF96
S3150801386001460020AEF1140EB1FA81F7AEEB07045A
S3150801387001FA07FE0C37C7F1200100FA07F7C8401D
S315080138804EEA000E23EA455343F48013A2E733F0C8
S315080138900043B3FA83F704BFB2FA82FE77440B3FBB
S315080138A0E41BB7F1200E2FBF02FA0EF3BB40C7F196
S315080138B0200E22FA0EFE38BF43EA0E03BA40641CF4
S315080138C082E750EA410E14BF52EA430E6FF0000137
S315080138D04FF4001717EB430F8ABF194617EB410F31
S315080138E0B5E74CEA05510020B0BDD4F10104B4F1A5
S315080138F020070FDAC4F12007520828BF42F0010257
S3150801390010FA07F501FA07F7E1BF2A43E040384301
S31508013910E1400FE0352C98DCC7F1200452EA400259
S3150801392020FA07F218BF42F0010231FA07F0A14066
S315080139300A43002172F1004250F1000051EB0C01DB
S31508013940B0BD000010B5144600F002F8226010BDA3
S31508013950C1F30A5343B14A0012F5001F28D2A3F254
S31508013960FE32A1EB0251704750EA410C20D001F01A
S31508013970004C31EA0C01B1FA81F204BFB0FA80F3C6
S31508013980D2180B3AB2F120032CBF00FA03F1914089
S3150801399041EA0C013EBFC2F1200C20FA0CF319438F
S315080139A09040524240F2FD33D21A01EB035170475F
S315080139B0002270474FF4001C1CEB410F94BF1CEB0F
S315080139C0430F09E041EA030C50EA4C0C52EA0C0C8D
S315080139D003D2994208BF9042704714BF8B42824274
